:020000040800F2
:100000000000022075C0050889910008E91E020859
:1000100025C1050825C1050825C105080000000007
:10002000000000000000000000000000C5AD000856
:10003000C7AD000800000000C9AD0008190901089B
:1000400025C1050825C1050825C1050825C10508E4
:1000500025C1050825C10508BBEE0008BFEE000854
:1000600025C10508C3EE0008C7EE00089D990008E9
:10007000B1990008C5990008D9990008ED990008C0
:10008000019A0008159A000825C105080000000023
:10009000000000000000000000000000CBEE00089F
:1000A000D5980008FD98000825990008BF98000819
:1000B0004D990008619900087599000825C1050847
:1000C00025C1050825C1050825C1050825C1050864
:1000D00025C10508159400082194000800000000BF
:1000E000CFEE000825C10508CBAD000800000000D8
:1000F000000000000000000000000000299A000835
:100100000000000025C105088999000825C10508DF
:1001100000000000000000000000000000000000DF
:100120003D9A0008519A0008659A0008799A0008DB
:100130008D9A000800000000000000000000000090
:100140000000000000000000000000001DAE0008DC
:10015000A19A0008B59A0008C99A000825C10508A7
:1001600025C1050825C105080000000000000000A9
:10017000000000000000000000000000000000007F
:100180000000000025C1050800000000000000007C
:0801900025C1050825C1050881
:0801980008BC05000100000095
:1001A000A4FD0020020100000300141EC4FD002075
:1001B000010B000000007700E4FD0020010C0000AE
:1001C0000000760004FE0020011000000000760010
:1001D00024FE0020010D01000000770044FE0020F5
:1001E000011200000000760064FE002001140000EF
:1001F00000001E0084FE0020011A000000000D0017
:10020000A4FE00200116000000000C00C4FE002027
:10021000011B000000000E00E4FE0020011C000095
:1002200000001E0004FF00200117000000000C0069
:1002300024FF00200118000000000E0044FF0020F1
:100240000119000000000C0064FF002001280100DB
:100250000000180084FF002001200000000048007A
:10026000A4FF00200121000000004900C4FF00207D
:100270000122000000004A00E4FF002001230000EA
:1002800000004B00040001200124000000004C008D
:10029000240001200125000000004D004400012041
:1002A0000126000000004E0064000120012700002C
:1002B00000004F0084000120012B000000002900F5
:1002C000A4000120012C010000002900C40001202D
:1002D000012D010000007000E4000120012E01004A
:1002E0000000520004010120012F0100000028003D
:1002F000240101200229010000012C0044010120F9
:100300000132000000003C006401012001350000C2
:1003100000002000840101200136000000002900B7
:10800000D0E907239A422FBFD01AC0688018C01A3F
:108010007047D0E9092300699A4238BF1218D31A71
:108020000138C01A7047D0E90902131A5842584162
:108030007047036A41690246C85CD16801338B42CC
:1080400028BF002313627047436A8269D154436A90
:1080500002690133934228BF0023426B4362D36815
:1080600043F08003D3607047436B188810F0100012
:108070001EBF1A889B8801207047436B99891A8814
:10808000890610B592B2044607D5900605D5E26A76
:1080900022B39888216B80B29047636B99891A88C4
:1080A000090692B20FD510060DD5D4E909128A42FD
:1080B00022D0A169895C998021690132B2FBF1F07B
:1080C00001FB1022A262998A1A88C90592B204D5CE
:1080D000D20744BF4FF6F7721A8010BD9B88E26941
:1080E0006169DBB28B54E369E2680133B3FBF2F1FF
:1080F00002FB1133E361D0E7DA6822F08002DA6034
:10810000E1E770477047036941681F2B30B54FF0B6
:10811000200285BFA3F120054C680C68AA4098BFD7
:108120009A4022421ED0826900201074D068846870
:10813000206820F0010020605468206865790A4CAE
:10814000828934F8154092B21F2B22EA0402828100
:1081500088BF203B4FF020028BBF9A4002FA03F306
:10816000CA608B6030BD00BF901A06080E4BDA68FB
:10817000D20310D4DA68D1060FD4DA68D2050ED44F
:10818000DA6812F0E00F0CD1DB6813F0020F14BFB5
:108190000820092070470120704706207047022000
:1081A00070470720704700BF003C024007B5092315
:1081B0008DF80730FFF7DAFF8DF807009DF80730DC
:1081C000012BF7D09DF8070003B05DF804FB838A0C
:1081D000028B9BB243EA024331EA03030CBF012046
:1081E0000020704782B00023019300930123009088
:1081F0000193019B63B1009A21F07F4314320092F6
:10820000009A12681A4214BF0120002002B0704781
:10821000009A1832F3E77047704701207047044B0B
:10822000D3E90003984288BF03F50063181A70472A
:10823000E0150020054AD2E900318B42FDD0D1186B
:108240000133C3F30A03087A13607047E015002076
:10825000044BD3F8080820B1D3F80808431F58424C
:1082600058417047E0150020012380F849307047DD
:1082700010B5D0F8E83504461B699847032384F805
:108280001231002010BD08B590F8123180F813317A
:10829000042380F81231D0F8E835DB6898470020D5
:1082A00008BD08B5D0F8E435DB6903B19847002074
:1082B00008BD08B5D0F8E4351B6A9847002008BD12
:1082C00008B5D0F8E4355B6A9847002008BD10B5C2
:1082D000074C2068FF2808D00649D1F80C2801F582
:1082E000016100F035F8FF232360002010BD00BFBE
:1082F00000000020E0150020432301480B80704758
:1083000004000020122301480B8070474700002022
:10831000042301480B8070475900002070477047C4
:108320007047704770477047044B00200522C3F820
:108330000828C3F81808C3F81C087047E015002087
:10834000024B0020C3F80808704700BFE01500206A
:10835000212838B50C461BD022282BD0202815D137
:10836000A1B1072A12D11A4DD5F81C3813B10968EA
:10837000002098472368C5F82038237985F82438E9
:10838000637985F82538A37985F82638002038BD2B
:108390000029FBD0072AF9D10D4BD3F820280A6019
:1083A00093F824280A7193F825284A7193F82638FF
:1083B0008B71EBE70029E9D0022AE7D1044BD3F80F
:1083C0001838002BE2D0098800209847DEE700BF6C
:1083D000E0150020074AD2F82838D2F82C2893421A
:1083E00003F1FF338CBF002001209B1A03EBC02058
:1083F000704700BFE0150020ECE730B50F4CD4E922
:1084000000239A4286BF03F50065AA1A9A1A0A4405
:10841000B2F5006F10D801440022814203D102B1AD
:108420006360002030BDE21810F8015B1572013363
:10843000C3F30A030122F0E70220F3E7E01500206E
:10844000007970470079C0F3401070470079400907
:10845000704700BF704700BF704700BFD0ED007A83
:10846000D0ED036A30EE677AE6EE877AB0EE670AFF
:10847000C0ED007A704700BFD0ED017A80ED021A9E
:10848000F5EE407AF1EE10FA04BF9FED0C7AC7EEDC
:10849000207A31EE277A08BFC0ED017AC1EE076A73
:1084A000D0ED007AC0ED036A30EE677AE6EE877AA7
:1084B000B0EE670AC0ED007A704700BF83F9223E34
:1084C0009FED047AC7EE007A77EEA07A80EEA70AD5
:1084D000704700BF72C7D13D00230360436080ED49
:1084E000020A704790ED017AD0ED036AD0ED027A6E
:1084F00030EE470AA6EE807A90ED000A80ED017A10
:1085000037EE676AE6EE867A37EEC07AC0ED027A19
:10851000A6EE870A80ED000A704700BFD0ED056A1D
:10852000D0ED017A90ED007A90ED066AD0ED025A16
:1085300090ED035A80ED050A66EEA77AC0ED066A53
:10854000E7EE007A90ED077AE5EE867A90ED086A1C
:10855000D0ED045A80ED087AE5EE477AE5EEC67A6A
:10856000B0EE670AC0ED077A704700BFD0ED057A1C
:1085700090ED006A90ED067AD0ED035AE6EE007AAF
:1085800090ED016AF0EE406AA6EE267AB0EE670A38
:10859000D0ED047A90ED026A67EEC07AA5EEC07A5B
:1085A000E6EE267A80ED057AC0ED067A704703681C
:1085B0005A1C02601970704703690133012B036173
:1085C0001CD0D0ED005AD0ED026A07EE903A30EEA2
:1085D000656AF8EEE77A86EE277A77EE257AB0EECE
:1085E000667A30EE670AC0ED017AA6EE007AC0ED39
:1085F000007A80ED037A80ED027A7047002380EDE7
:10860000010A80ED000A8360704703685A1C02600B
:10861000197070472DE9F347038A8689B6B205467B
:108620000C461E404FF0004901F14C0701F134089F
:1086300016B902B0BDE8F087B6FA86F329FA03F25C
:10864000D24391B2298216401B3B002C40D0042B10
:10865000EED8DFE803F039342E280300E368D5F8BC
:108660002CA02BB19B681BB11FFA8AF1201D9847E3
:10867000636A33B19B6823B11FFA8AF104F11C00CD
:108680009847E36B2BB19B681BB11FFA8AF14046F8
:108690009847636D002BCBD09B68002BC8D01FFA86
:1086A0008AF1384603E0E368696B5B68201D9847F0
:1086B000BEE7636AA96B5B6804F11C00F7E7E36B34
:1086C000E96B5B684046F2E7636D296C5B68E8E73D
:1086D000042B06D8DFE803F00D0B09070300EB6A53
:1086E0000193019BA4E76B6BFAE7AB6BF8E7EB6BCD
:1086F000F6E72B6CF4E790F84820531C0244DBB2F9
:1087000080F8483082F8341090F849200AB1132BD1
:1087100001D952F094BB7047002280F8492052F0F2
:108720008EBB70B50F4E96F83038002BFBD1044647
:108730004518AC4201D1002070BDD6F82C3814F891
:10874000011BF2180133C3F30A0382F83118C6F88B
:108750002C38FFF73FFE0028EBD101200AF07DFA0C
:10876000F7E700BFE015002038B50C461146FFF7CB
:108770006FFD48B1054D002A55F8C43C04DD204684
:10878000FFF7CFFF55F8C43C38BD00BFD826002006
:10879000F0B590F8CF5590F8CE1590F8D12590F817
:1087A000D03590F8CC7590F8CDC501EB05218DB290
:1087B00003EB022390F8D31590F8D22585B002EB95
:1087C000012207F01F06012192B29BB28E4204469D
:1087D0008DF808708DF809C0ADF80A50ADF80C306E
:1087E000ADF80E20C0F8402180F8111100F00C8186
:1087F000022E00F01D81002E40F09B81BCF1090F7C
:108800005ED8DFE81CF0B600F4005D00C8005D0033
:1088100057000A005D00A90076002E0A022EADF86E
:1088200006200BD0032E25D0012E49D1D0F8EC35EF
:108830001B68A0780DF10601984709E0D0F8E435EF
:1088400080789B6A0DF1060198474670C4F8F005E0
:10885000BDF80620002A47D0BDF80E30002B43D0CB
:108860009A4228BF1A46ADF806200146204652F02B
:10887000EBF939E0E9B2052922D8DFE801F0030776
:108880000B0F1317D0F8EC355B68D2E7D0F8EC3556
:108890009B68CEE7D0F8EC35DB68CAE7D0F8EC355A
:1088A0001B69C6E7D0F8EC355B69C2E7D0F8EC3558
:1088B0009B69BEE71A4303D190F81231032B03D111
:1088C000204652F015F90FE0016905F07F0680F8A7
:1088D00014610B6865F30A121A430A6052F0C8F972
:1088E0002EB1022384F81231002005B0F0BD01231F
:1088F000F8E7E9B2904D012905F8C01CE0D890F8DE
:108900001231022B0FD0032BDAD1C1B9022380F828
:108910001231D0F8E43580F810115B689847204692
:1089200052F0A6F9E0E70029F9D00121032380F8ED
:10893000101180F81231204652F09DF8EFE790F8C0
:1089400010110129EBD0D0F8E4355B68984715F891
:10895000C01C84F81011EEE7012AB1D190F8123151
:10896000022B04D0032BABD100F588717EE773494D
:108970007CE790F81231023B012BA1D86E4B00220C
:1089800043F8B82CD0F8182112B1022243F8B82CC1
:108990006B4902226AE7012D08D1C0F81851D4F8BA
:1089A000E43502A99B6820469847B8E7022D9BD181
:1089B000DAB2002A98D102691B0A023B5268032BE3
:1089C00003D8DFE803F00C0E1012012363F3061244
:1089D000594B43F8B42C012384F816319FE7022346
:1089E000F4E70323F2E70423F0E70523EEE790F82A
:1089F0001231023B012B3FF663AF012D7FF474AFC0
:108A00000023C0F81831CAE790F81221032A7FF436
:108A100057AFDBB2012B3FF653AFD0F8E43502A9D4
:108A20009B689847BDF80E30002B7FF45DAF76E76A
:108A300007F06007202FD9B205D1D0F8E43502A99C
:108A40009B68984750E7BCF1010F31D0BCF1030F90
:108A50001ED0BCF1000F7FF447AF90F81221022A1C
:108A60005AD0032A7FF42CAF13F0800F4FF0280266
:108A7000314B59D001F07F0102FB010191F81E2119
:108A8000002A4FD0012243F8B02C2E490222EDE6F5
:108A900090F81231022B3FD0032B7FF411AF002D41
:108AA0007FF47DAF4A063FF47AAF51F0F0FF76E7EE
:108AB00090F81221022A2FD0032A7FF401AF002D53
:108AC0007FF412AF11F07F003FF429AF5BB2002BAF
:108AD0004FF02802B5BF02FB004102FB014101F546
:108AE0008E7101F55D710022DB0F08708A704B708A
:108AF00004EB8000C9786BB18269136802396FF3A7
:108B0000555301298CBFC3F30071012161F31C731C
:108B1000136044E7426DF0E74B063FF4E5AE51F0D9
:108B2000B6FFE1E60022AEE702FB010191F87623F1
:108B3000A6E707F08001F2E7D82600201C260020D7
:108B4000202600202826002010B5044671BB90F88E
:108B50001131032B1BD1D0F89023D0F87C339A42EB
:108B600017D9C178012908BFD0F88013A2EB0302FE
:108B700004BFC918C0F88013934228BF1346C0F839
:108B800090239BB2D0F88023002152F021F90020DD
:108B900010BDD0F8E4351B6923B190F81221032AE7
:108BA00000D19847204652F063F8F0E7D0F8E4355A
:108BB0009B69002BEBD090F81221032AE7D198474C
:108BC000E5E770B50A7812F0600406460D462AD033
:108BD000202C2FD1CC884B78FCB112060CD51F4924
:108BE00022461846FFF7B4FBEA881C49304652F08B
:108BF0002BF80024204670BD194A1360194A03233C
:108C0000C2F80C4880F81131C0E9E444234602F56B
:108C10000162002152F0DCF8EBE702221144184611
:108C2000FFF796FBE6E74B780A2B08D00B2B0BD00F
:108C3000062BDFD1304651F05BFF0224DAE70A4908
:108C4000012252F001F8D5E78B781BB9074B43F8A6
:108C5000AC4CCFE751F04CFFCCE700BFF01D00203B
:108C600000000020E01500202C260020D82600203F
:108C700010B5282303FB0101074AB1F88C13044601
:108C80001046FFF7BAFB2046034A4023012152F069
:108C90009FF8002010BD00BF30260020002310B533
:108CA00019460446402251F031FF402280212046DF
:108CB000002351F02BFF012384F81231D4F8E8355A
:108CC000A0785B689847002010BD38B54022044664
:108CD0000223812151F01AFF204602234022012164
:108CE00051F014FF204603230822822151F00EFF89
:108CF000084B0222002583F84B2083F84C50FFF7E5
:108D000013FB01212046044A402352F061F8284613
:108D100038BD00BF000000203026002038B50122F9
:108D2000044640F20113A0F844310125114652F0E7
:108D30006DF829462046A4F89C53002252F066F8AC
:108D40004FF48173A4F86C3120462A46022152F078
:108D50005DF8FFF7F5FA002038BD38B5254C94F8DA
:108D60003028012A034633D1234850F8682C1AB919
:108D700084F83028002038BD402AD4F8281819D9A2
:108D8000403A01F1400540F8682CC4F828584022C8
:108D90001A4810FA81F1C3E9541140F20110002180
:108DA000C3E95621A3F8440103F5A271184651F016
:108DB00076FFDFE702EB0105C4F828584FF0000505
:108DC00040F8685C0ABF022092B284F83008DFE7FE
:108DD000022ACFD1002540F20112C0E95455C0E962
:108DE0005655A0F8442100F5A27151F058FF84F8BF
:108DF0003058BFE7E0150020D8260020111E0020C3
:108E000038B52A4C54F8643C0F2B03F1010203D00F
:108E100044F8642C002038BD254A002344F8643C03
:108E200092F83038002BF5D1D2F82818B1F5006F40
:108E300008BFC2F82838D2F82818D2F82C3899423E
:108E400003D1002382F83038E4E78CBFC1F500631A
:108E50005B1A402B1BD9403B01F1400544F8683CAC
:108E6000012382F83038C2F828584023114A12FAF8
:108E700081F140F20112A0F844210022C0E954110E
:108E8000C0E9563200F5A27151F009FFC2E701EBCB
:108E90000305C2F828584FF0000544F8685C0EBF7F
:108EA000022401249BB282F83048DFE7D826002054
:108EB000E0150020111E002008B502484FF0AEFF5B
:108EC000014808BDF9A706087826002008B5024821
:108ED0004FF0A4FF014808BD05A806087826002029
:108EE00008B502484FF09AFF014808BD0AA80608D5
:108EF0007826002008B502484FF090FF014808BDD1
:108F000014A806087826002008B502484FF086FF0E
:108F1000014808BD1FA80608782600200068F02236
:108F2000FF2107F057BD0068B422FF2107F052BDB2
:108F3000CA4341EA02120068D2B2D22107F04ABD08
:108F40000A460068A52107F045BD5521F8E70068ED
:108F50009622FF2107F03EBD0A460068872107F0F0
:108F600039BDC90101F080020068782107F032BDE7
:108F7000F8B504460E461546071D20683A46FF21FF
:108F800008F0ECFA30B116B12379DB07F5D40DB156
:108F900023792B70F8BD00220121E9E710B50446C2
:108FA000FFF7C1FF18B12046BDE81040F3E710BD40
:108FB00010B50446FFF7C4FF18B12046BDE81040C5
:108FC000E9E710BD73B50546CDE90023FFF7E6FFDD
:108FD000A8B12846FFF7B9FF88B12846FFF7DBFFA5
:108FE00068B16E46082416F8011B2846FFF7E0FF1B
:108FF00028B1013C14F0FF04F5D102B070BD00208F
:10900000FBE7CC21D4E770B506460C468D18AC4280
:1090100001D1012006E014F8011B3046FFF7C8FF1C
:109020000028F4D170BD38B505461446FFF794FF0B
:109030002846FFF7B0FF20B11CB12B79C3F34013D2
:10904000237038BD10B50446FFF7A8FF38B120469D
:10905000FFF7D7FF18B12046BDE810409BE700207E
:1090600010BDC90138B501F0800104461546FFF76F
:1090700078FF08B9002038BD002201212046FFF703
:1090800077FF0028F6D023795B092B70F3E710B542
:10909000021D0446FF21006808F060FA18B120792B
:1090A000C04300F0010010BD38B504461546006805
:1090B0000A46E12107F08EFC30B120682A46FF21E4
:1090C000BDE8384008F04ABA38BD0A46C321EBE78C
:1090D00038B5021D0D46F0210446FFF7E5FF08B143
:1090E00023792B7038BD0A46E121DDE738B5044607
:1090F0000D46FFF72CFF40B12046FFF74CFF20B193
:1091000029462046BDE83840EDE7002038BD70B55F
:1091100006460C468D18AC4201D1012006E02146DE
:109120003046FFF7E3FF01340028F4D170BD024B55
:10913000D3F8A00007F0F9BAD82600200E49D1F8DC
:10914000883043F47003C1F888300C4B1A68002053
:1091500042F001021A6098601A6822F0847222F4C8
:1091600080321A60064A5A601A6822F480221A6015
:10917000D860044B8B60704700ED00E0003802407F
:10918000103000240000000870472DE9F0414769C5
:1091900006468846002F59D10368C3F30D0515B361
:1091A000D8F800803568FFF701F8092840F087807B
:1091B000444C236923F440732361236943F400730F
:1091C0002361236943F001032361C5F80080FEF7A2
:1091D000EDFF2369092823F0010323616FD1336870
:1091E0000433336032E0384A934229D302F5804297
:1091F000934224D302F5804293422AD3334A9342C6
:1092000029D902F58032934227D902F500329342E0
:1092100025D902F50032934223D902F50032934258
:1092200021D902F5003293421FD902F580229342E0
:109230001DD9B3F1016F1CD3052009F0C7FE082525
:10924000FEF7B4FF092816D04FF0FF373846BDE8C7
:10925000F0811025F4E71825F2E72025F0E728250E
:10926000EEE73025ECE73825EAE74025E8E7482532
:10927000E6E75825E4E7134C236923F440732361A0
:10928000236943F400732361236923F0F803236106
:1092900023691D4345F002052561236943F48033AA
:1092A0002361FEF783FF236923F00203236123690F
:1092B000092823F0F80323613FF472AFC4E76FF08D
:1092C0000107C3E7003C024000400008FFFF000820
:1092D000002808DB4209012300F01F0003FA00F018
:1092E000014B43F82200704700E100E00028ACBFCA
:1092F00000F16040064B4FEA0111ACBF00F5614040
:1093000000F00F00C9B2B4BF195480F800137047C1
:1093100014ED00E02DE9F04798463C4B914603EBF5
:10932000800205469468002C45D02833636004F120
:109330003E03A36104F59F73E3614FF48073C4E9B6
:109340000433236894F83D00E160A36306F002F85B
:10935000064694F8440294F83CA0271D08B14FF04B
:10936000DFFF94F8450208B14FF0DAFFD4F840323D
:109370001BB1274A116B0B43136318F0080F23D05E
:109380000135EDB21EB14FF4E163F380357218F090
:10939000100F94F8462211D00221304605F0ECFE61
:1093A00094F94702D4F84812FFF7A0FF94F9470256
:1093B000FFF78EFF3C462046BDE8F08718F0200FEF
:1093C00014BF12213221E8E719F0020F0CD06B1CF8
:1093D000DBB21EB14FF4A162F280337294F84622E0
:1093E0000221304605F0C8FE19F0010FD8D05046D2
:1093F00005F0B0FF0135EDB218B14FF4C163C38081
:10940000057294F846220221C8E700BF901A0608A8
:10941000003802400148FEF730BE00BF6400002063
:109420000148FEF72ABE00BFB0020020024B586F71
:10943000C0F30070704700BF0038024070B50028CC
:1094400028D04C684CB9426815685679AB8902221D
:109450009BB2B24023EA0203AB818A683AB94368FF
:109460001D68AB8923F001031B041B0CAB818160D9
:1094700044B14468216864798D890223A3402B4359
:109480009BB28B8132B143681A6893899BB243F0D7
:109490000103938170BD0B4B30B51A4600241D7932
:1094A000854208D1DD68294203D0142000FB042046
:1094B00030BD0029F9D001340A2C03F11403EED198
:1094C0000020F5E7F804002038B503681B681C6825
:1094D000254B03F5B86393ED007A07EE902AB8EEBA
:1094E000477AF8EE677A013987EE270A8DB2DFED09
:1094F0001F7A30EE270A55F007F81D4A23880138F5
:10950000944280B29BB212D002F5806294420ED097
:10951000B4F1804F0BD0A2F58032944207D002F50F
:109520008062944203D002F58062944202D123F01B
:1095300070039BB20F4A944206D002F580629442B7
:109540001CBF23F440739BB22380094BE5629C420D
:10955000208503D003F580639C4201D1002323863C
:109560000123A38238BD00BF000000200AD7233C9E
:1095700000000140001000402DE9F0434568A87943
:1095800010F0040300F002020BD0002017468046C2
:10959000042406466B79032B49D8DFE803F0094A17
:1095A00089C990464FF480701F461C460126F1E79A
:1095B0002D682B8C23F001031B041B0C2B84B5F8A6
:1095C00020C0B5F804902B8B23F073031B041B0CF5
:1095D00043F0600E2CF0020C6E4B4FEA0C4C4FEA3D
:1095E0001C4C48EA06069D421FFA89F94CEA060C13
:1095F00003D003F580639D420AD14FF6F3730CEA62
:1096000003033B4329F4407943EA040C40EA090987
:10961000A5F80490A5F818E06963A5F820C02B8B85
:1096200023F008031B041B0C43F008032B83BDE845
:10963000F0832D682B8C23F010031B041B0C2B8450
:109640002A8CB5F804E0B5F818C0524B2CF4E64C5F
:1096500022F020024FEA0C4C12044FEA1C4C120C70
:1096600048EA06069D421FFA8EFE4CF4C04C42EAC0
:10967000061203D003F580639D420BD122F08002D5
:1096800042EA071222F040022EF4406E42EA04122F
:109690004EEA800EA5F804E0A5F818C0A9632A8454
:1096A0002B8B23F400631B041B0C43F40063BDE706
:1096B0002D682B8C23F480731B041B0C2B842A8CA9
:1096C000B5F804E0B5F81CC022F400732CF0730C5C
:1096D000304A4FEA0C4C1B044FEA1C4C1B0C48EA66
:1096E000060695421FFA8EFE4CF0600C43EA0623F4
:1096F00003D002F5806295420BD123F4006343EA64
:10970000072323F480632EF4405E43EA04234EEAE9
:10971000001EA5F804E0A5F81CC0E9632B84AB8B00
:1097200023F008031B041B0C43F00803AB837EE704
:109730002C68238C23F480531B041B0C2384258C5E
:10974000A288A38B25F400552D0448EA06062D0CAB
:1097500023F4E64345EA06350E4E1B041B0CB442C7
:1097600092B243F4C04303D006F58066B44203D1FD
:1097700022F4804242EA8012A280A38321642584DD
:10978000A38B23F400631B041B0C43F40063A3832B
:109790004DE700BF0000014043685A79032A0FD803
:1097A000DFE802F00205080B1868343070471868CB
:1097B0003830704718683C30704718684030704740
:1097C0000020704710B543681A685879084B034465
:1097D000012093F85840138CA0409BB223EA000369
:1097E0001384138CA140194389B2118410BD00BFAA
:1097F000901A0608F0B5EFF31184102383F3128852
:10980000C5684668AA68136823F0010313603268CC
:109810007779104E938936F817609BB223EA0603D6
:1098200093812A696D681F2A4FF0200385BF203A73
:1098300093409340EB6098BFAB60E3B283F3118831
:10984000C3689B6859601A6842F001021A600123DC
:109850000374F0BD901A06080268137D012B04BF43
:109860000223137592F82C100CBF4FF400730023E1
:10987000012904BF022182F82C1092F8441008BF7D
:1098800043F48063012904BF022182F8441092F856
:109890005C1008BF43F4006301290DD1022182F856
:1098A0005C1043F480534268116800224A628A893E
:1098B00092B213438B8101E0002BF4D17047034B2C
:1098C0000348D3F8A410FEF7A5BE00BFD826002099
:1098D0000000014010B5064C0648D4F8A410FEF76D
:1098E00099FED4F8C4100448BDE81040FEF792BEBB
:1098F000D8260020000001400040014010B5064C71
:109900000648D4F8A410FEF785FED4F8C810044821
:10991000BDE81040FEF77EBED826002000000140C2
:109920000044014010B5064C0648D4F8A410FEF7D8
:1099300071FED4F8CC100448BDE81040FEF76ABEB2
:10994000D82600200000014000480140034B4FF0A2
:109950008040D3F8A810FEF75DBE00BFD8260020D7
:10996000024B0348D3F8AC10FEF754BED8260020B3
:1099700000040040024B0348D3F8B010FEF74ABE83
:10998000D826002000080040024B0348D3F8B4104A
:10999000FEF740BED8260020000C00400348D0F857
:1099A000D03513B100F2C4501847704700000020B2
:1099B0000348D0F8F03513B100F2E450184770476F
:1099C000000000200348D0F8103613B100F2046004
:1099D00018477047000000200348D0F8303613B114
:1099E00000F2246018477047000000200348D0F8B8
:1099F000503613B100F24460184770470000002051
:109A00000348D0F8703613B100F26460184770470D
:109A1000000000200348D0F8903613B100F28460B3
:109A200018477047000000200348D0F8B03613B143
:109A300000F2A46018477047000000200348D0F8E7
:109A4000D03613B100F2C460184770470000002000
:109A50000348D0F8F03613B100F2E46018477047BD
:109A6000000000200348D0F8103713B100F2047052
:109A700018477047000000200348D0F8303713B172
:109A800000F2247018477047000000200348D0F807
:109A9000503713B100F2447018477047000000209F
:109AA0000348D0F8703713B100F26470184770475C
:109AB000000000200348D0F8903713B100F2847002
:109AC00018477047000000200348D0F8B03713B1A2
:109AD00000F2A4701847704700000020036823F0CC
:109AE000010303600023036043608360C36003617C
:109AF000212343612A4B984203D13D2243F8082C8D
:109B00007047284B984204D14FF4746243F8202CDC
:109B10007047254B984204D14FF4741243F8382C07
:109B20007047224B984204D14FF0746243F8502C96
:109B300070471F4B984203D11E4A43F8642C70476C
:109B40001D4B984203D11D4A43F87C2C70471C4B97
:109B5000984203D11B4A43F8942C70471A4B984201
:109B600004D14FF03D5243F8AC2C17E0174B98420C
:109B7000C3D0174B9842C7D0164B9842CCD0164B47
:109B80009842D1D0154B9842D6D0154B9842DAD096
:109B9000144B9842DED0144B9842E2D0704700BF7D
:109BA000106002402860024040600240586002405D
:109BB000706002403D00002088600240400F00209D
:109BC000A060024000003D20B860024010640240E6
:109BD00028640240406402405864024070640240BD
:109BE00088640240A0640240B86402402DE9F0415C
:109BF0000022012603250B6806FA02FC3CEA030357
:109C000031D10368540005FA04FE23EA0E03036011
:109C10000B79D0F800806FEA0E0703FA04FE013BCF
:109C20004EEA080E012BC0F800E011D883681F40EF
:109C300087604B798768A3403B438360436823EA8E
:109C40000C0343608B79476893409BB23B4343606E
:109C5000C36805FA04F723EA0703C360CB79C76832
:109C6000A3403B43C3600132102AC4D1BDE8F08158
:109C7000F7B51C2005F06EFB1121044605F056FADD
:109C8000204605F045FAC82008F0E7FF204605F019
:109C90003AFA1B2005F05EFB20B140F21113C3809D
:109CA0000023037224B140F21123E38000232372C6
:109CB000CA4B502283F843230822C3F88820BFF3FD
:109CC0004F8FBFF36F8FC64CC64D236B43F001031C
:109CD00023634FF4C05040F20233CDE90003C24881
:109CE0006946FFF783FF436A23F470434362436A84
:109CF00043F420434362436A23F470234362436A7C
:109D000043F4202343623F2005F024FB002105F0AB
:109D10000DFA636C43F480436364636B43F0800328
:109D20006363B24BB24C01205861B24BC4F8C036E9
:109D300003F12C024833C4F8C836AF4BC4F8C4262C
:109D4000C4E93753022384F8E4304FF0A043C4F849
:109D5000E83003F50063C4F8EC3003F58073C4F811
:109D6000F43003F50073C4F83031A3F5F073C4F890
:109D7000F83003F50073C4F83431A3F5F073C4F878
:109D8000FC3003F50073C4F83831A3F5F073C4F860
:109D9000003103F50073C4F83C31A3F5EC63C4F85B
:109DA000F0304033C4F8A831C033C4F86C312033EC
:109DB000C4F870312033C4F874312033C4F87831DA
:109DC0002033C4F87C312033C4F880312033C4F808
:109DD00084312033C4F8883103F5226384F8E70026
:109DE000C4F8AC3103F58053C4F8B03103F58053A7
:109DF000C4F8B43103F58053C4F8B8314FF05023A0
:109E0000C4F8BC3103F58053C4F8C03103F5805366
:109E1000C4F8C43103F58053C4F8C831A3F5E44352
:109E20000022C4F8E83104F1DC0384F8EE0184F880
:109E3000F02119461546402681F81C21A1F822215F
:109E40000132042AC1E9496581F81D0181F81F51D9
:109E5000C1F8305101F12801EED100221146402015
:109E600083F87423A3F87A230132042AC3E9DF01BB
:109E700083F8751383F87713C3F8881303F1280365
:109E8000EED14FF0A04300259A6822F001029A60BB
:109E9000DA6842F04002DA604FF0B2FB94F8E53045
:109EA00094F8DF205B1B18BF01231B0143F0210343
:109EB00063F31745D4F8E830012A9D6307D19A6807
:109EC00022F03E0141F02A0161F307029A60DA684C
:109ED000C2F3076121F0600141F0400161F31F62AC
:109EE000DA60D4F8E82100201060D4F8EC20116882
:109EF00060F3CC21116094F8E710012912D11168A8
:109F000041F00301116080225A6202F580029A62D8
:109F100002F14012C3F804214FF4A072C3F80821E3
:109F2000C3F80C2110204FF04DFB00230093009B41
:109F300043F010030093D4F8E830009A1A612F4AD6
:109F400019690091013A02D00099C906F8D4D4F8F1
:109F5000EC1094F8DD502A4E00224FF0FF300A61D9
:109F600017464A614FF0FF0C8861CA61AA4251D37B
:109F70000022244E17464FF0FF0C95425CD80A6928
:109F800042F480720A6194F8DF20012A04BF1E485F
:109F90000863002199614FF0FF306FF080415961F3
:109FA0005860596119499961B2FA82F21849520907
:109FB00041EA021299690A439A619A6842F00102E1
:109FC0009A60D4F8C4361B689847044B502283F833
:109FD000432308229A6003B0F0BD00BF00E100E017
:109FE000003802400804010000000240003C01402B
:109FF000D8260020C407002040004001410D030086
:10A00000CC270020082800200301810000080080E0
:10A0100008383C0056F8040BD0F800E0BEF1000F01
:10A02000ACBF4FF0000E4FF0904EC0F800E0013290
:10A030000761C0F808C099E756F8040BD0F800E0B3
:10A04000BEF1000FACBF4FF0000E4FF0904EC0F8C5
:10A0500000E001320761C0F808C08EE7204A93682B
:10A0600003F00C03042B10B520D0082B20D01D4B7F
:10A070001B4C0360A3681C4AC3F30313134493F8F7
:10A0800028180368CB404360A168C1F382211144C2
:10A0900091F8281823FA01F18160A168C1F34231D7
:10A0A0000A4492F82828D340C36010BD0F4BDFE765
:10A0B0005368516813F4800F01F03F01536814BFD7
:10A0C0000A4A084AB2FBF1F1054A5268C2F301425A
:10A0D000C3F3881301324B435200B3FBF2F3C7E7DB
:10A0E000003802400024F4000000002000127A0032
:10A0F000F0B5446B8668A38923F400531B041B0C42
:10A10000A3818279278A0546BFB2100312F0040F9B
:10A110004FEA022100F400506A7927F4405740EAE0
:10A120000700208214BF4FF4805C4FF0000C12F047
:10A13000010F0CBF002304239207A28922F4B0521E
:10A1400001F4806122F00C0248BF43F0080341EAA9
:10A150000C0112040B43120C1A43A281A38A23F4AC
:10A1600040731B041B0C85B0A3826846FFF776FF83
:10A17000214B9C4203D003F580639C423AD1039B60
:10A18000A2891921170401FB03F34FF064014CBFAE
:10A190007600B600B3FBF6F3B3FBF1F001FB10332E
:10A1A0000201A08900044BBFDB001B0132333233B4
:10A1B0004BBFB3FBF1F3B3FBF1F303F0070303F081
:10A1C0000F0313439BB223816A6BAB7913F0080F23
:10A1D000938A0BBF23F008039BB21B0443F00803D0
:10A1E00008BF1B0C938293899BB243F40053938165
:10A1F00005B0F0BD029BC3E7001001402DE9F84314
:10A200001E46204B9DF820509DF8247098428946A8
:10A2100090462CD13B462A4631460020FFF77AF87B
:10A2200004460020C4E90700C4E90900C4E90B980A
:10A230006571A660A7712046FFF75AFFEA0707D5A8
:10A24000636B4FF6DF721A80DA6842F02002DA6040
:10A25000626BAB0742BFD36843F08003D36093893E
:10A260009BB243F4005393812046BDE8F883064B2C
:10A27000984204D13B462A4631460120CEE70024CD
:10A28000F2E700BF001001400044004081602FE76A
:10A2900041712DE72DE9F043654F07EBC00985B00B
:10A2A00005464FEAC00899F83C0805F053F8064601
:10A2B00099F83D0805F04EF8044699F83E084FF02D
:10A2C0002FF86B1CDBB21EB140F60E12F280337217
:10A2D0001CB140F60E22E280237204223A2130465D
:10A2E00004F04AFF204604223A2104F045FF07EB20
:10A2F0000803D3F838484F4B9C4263D103F5F2333F
:10A300001A6A42F400121A621A6A22F400121A62DD
:10A31000474497F83F38022B6ED0032B6ED0464E41
:10A32000464A012B08BF1646A78827F03F07684614
:10A330003F04FFF793FE3F0C029A414BB2FBF3F34D
:10A3400098B20743A780218821F001010904090C74
:10A3500021803C498E4253D13B4BB2FBF3F201309A
:10A3600092B2042A80B238BF04222084A2832388B8
:10A370009BB243F001032380238823F4816323F0FD
:10A3800002031B041B0C43F4806323804FF48043BF
:10A390002381238823F080031B041B0C2380238844
:10A3A0009BB243F001032380284B03EB45130122AA
:10A3B00083F8D126002283F8D05683F8D22605B040
:10A3C000BDE8F083224B9C4209D103F5F0331A6AB1
:10A3D00042F480021A621A6A22F4800297E71D4B47
:10A3E0009C4295D103F5EE331A6A42F400021A62D8
:10A3F0001A6A22F400028AE7124E95E7124E93E79A
:10A4000006EB4606B2FBF6F291B2C2F30B020AB9B2
:10A4100041F0010141F400424FF496714B434FF477
:10A420007A71B3FBF1F301339BB223849EE700BF43
:10A430000000002000540040801A060000350C0087
:10A4400040420F00A0860100400D0300D8260020E6
:10A4500000580040005C00402DE9F047B84E440130
:10A4600006EB401908F0BAFB99F9D026B54B88469F
:10A47000D10003EBC2020746D2F8385899F8D22629
:10A48000013A142A00F28380DFE812F07900890093
:10A49000A100BA00C700D100DC00F40001010A01EC
:10A4A000170168018601B8010F02220234023F023F
:10A4B0005F02820215005F184FF0090A97F83C0806
:10A4C00004F048FF054697F83D0804F043FFB6F84E
:10A4D000303701339BB207462846A6F8303704F0E0
:10A4E00012FE384604F00FFE1121284604F01EFE2D
:10A4F0001121384604F01AFE4FF0650803E00520EC
:10A50000002108F099FB284604F0ECFD10B9B8F1E1
:10A510000108F4D1284604F0FBFD0021052008F0D5
:10A520008BFB284604F0EFFD0520002108F084FB9A
:10A53000BAF1010AE0D1284604F0EAFD0021052025
:10A5400008F07AFB384604F0E3FD0021052008F00E
:10A5500073FB284604F0D7FD0520002108F06CFBB2
:10A56000384604F0D0FD331993F9D006431C01D0CE
:10A57000FFF790FE3319002283F8D22607E02B88DC
:10A5800013F4007340F0D081321982F8D2363319B7
:10A5900093F8D236002B7FF465AFBDE8F0872B88A7
:10A5A00023F400631B041B0C2B802B889BB243F409
:10A5B00080632B802B889BB243F480732B803319EC
:10A5C000032283F8D226604B2344C3E902785F4913
:10A5D0002846FDF7FCFD002800F0A681331993F80A
:10A5E000E2265AB993F8E326FF2A04D193F8E0262D
:10A5F0000AB10A22C0E733190422BDE70F22BBE7E4
:10A60000321992F8E13603F0FE032B82052382F81B
:10A61000D2364D4B2344C3E902784D492846FDF715
:10A62000D6FD002800F0788133190622A4E73319FB
:10A6300093F8E3262A82072283F8D226424B23444A
:10A64000C3E9027843492846FDF7C1FD002800F020
:10A6500063813219D2F8E43653B92B889BB243F4A4
:10A6600000732B80384B2344C3E9027801238CE725
:10A6700008238AE72B889BB243F480732B8033191D
:10A68000092283F8D226304B2344C3E902782F49AC
:10A690002846FDF79CFD002800F046813319A8E705
:10A6A000321992F8E13643F001032B820B2382F832
:10A6B000D236254B2344C3E9027827492846FDF7C3
:10A6C00086FD002800F028813219D2F8E436012BEB
:10A6D0001BD12B8823F480631B041B0C2B80EFF30E
:10A6E0001181102383F312882B8B2B889BB243F4A8
:10A6F00000732B80CBB283F311880C2382F8D236FF
:10A70000114B2344C3E9027841E7022B15D12B8872
:10A710009BB243F400632B80EFF31181102383F38A
:10A7200012882B8B2B8823F480631B041B0C2B803B
:10A73000CBB283F311880D23E0E72B8B0E23DDE7EB
:10A74000D826002000000020A82D002001000300D2
:10A750008200070084000700020003009449284695
:10A76000FDF740FD934B002800F0DF8031192344B2
:10A77000D1F8E826501CC1F8E806288A1070D1F8F4
:10A78000E426013AC1F8E4260122C3E9027881F8FF
:10A79000EC2681F8D226FAE687492846FDF722FD05
:10A7A000844B002800F0C180EFF3118C102282F35B
:10A7B00012882A88301992B2D0F8E81642F4007252
:10A7C0002A804A1CC0F8E8262A8A0A705FFA8CF2AE
:10A7D00082F31188D0F8E826511CC0F8E816298ABF
:10A7E00011706FF00102C0F8E42623440122C3E98E
:10A7F000027880F8EC2680F8D226C8E66E49284612
:10A80000FDF7F0FC6B4B002800F08F803219D2F876
:10A81000E41603292AD1298821F480610904090C4E
:10A820002980EFF3118C102181F31288D2F8E80609
:10A83000411CC2F8E816298A0170298889B241F4BE
:10A84000007129805FFA8CF181F31188D2F8E81643
:10A85000481CC2F8E806288A0870D2F8E4160239C3
:10A86000C2F8E4160C2182F8D2164AE702290FD862
:10A87000298821F480610904090C2980298889B27A
:10A8800041F400712980298A002182F8EC16EAE659
:10A89000D2F8E816481CC2F8E806288A0870D2F8F0
:10A8A000E4160139C2F8E4162BE72B8823F4806301
:10A8B00032191B041B0C2B8092F8E13603F0FE03C7
:10A8C0002B82102382F8D2363A4B2344C3E9027814
:10A8D0003A492846FDF77BFCF0B1331993F8E3269B
:10A8E000FF2A04D193F8E0260AB1132244E6331973
:10A8F000112241E6331993F8E3262A82122283F8C3
:10A90000D2262C4B2344C3E902782D492846FDF773
:10A910005EFC08B13319E8E72A492846FDF762FCD6
:10A9200010B13319142227E6224B2344D3E9020144
:10A9300042F21073381A68EB0108984278F100036C
:10A94000FFF425AE3319152216E63119194BD1F84B
:10A95000E4268AB1D1F8E806234410F801CBA5F823
:10A9600010C0013AC3E90278C1F8E806C1F8E4264C
:10A97000122381F8D2360AE62A8892B2234442F49E
:10A9800000722A80C3E90278012381F8EC36F0E7EF
:10A990002B889BB243F400732B804FF6FF33AB82BE
:10A9A000044B2344C3E9027801223319E4E500BFD4
:10A9B00040000010A82D00200400001082000700B5
:10A9C000840007000004001038B5114C04EB40145B
:10A9D00094F8D156D5B1C4F8E436049BC4F8E836EF
:10A9E000002384F8EC360223490084F8E32684F837
:10A9F000D23601229DF8143084F8E11684F8E2265C
:10AA000084F8E036FFF728FD94F8EC56284638BD68
:10AA1000D826002038B5114C04EB401494F8D156D8
:10AA2000CDB1C4F8E436049BC4F8E83602234900EB
:10AA300084F8E32684F8D23600229DF8143084F896
:10AA4000E11684F8E22684F8EC2684F8E036FFF775
:10AA500003FD94F8EC56284638BD00BFD8260020E8
:10AA6000F0B587B0002300930193744B1A6842F449
:10AA700080321A601A6802F400320192009A0132A0
:10AA80000092019A1AB9009AB2F5A04FF2D11B6850
:10AA900013F4003318BF01230193019B012B40F0F5
:10AAA000B180664B66491A6C42F080521A640A689B
:10AAB00042F440420A609A689A609A689A609A687A
:10AAC00042F480529A605F4A5A601A6842F080727B
:10AAD0001A601A689201FCD55B4A40F2027111605B
:10AAE0009A6822F003029A609A6842F002029A6021
:10AAF000524A936803F00C03082BFAD19368534C25
:10AB000003F00C03042B7FD0082B7FD0504BC4F8EC
:10AB1000C0354A4B4F4D9A684F48C2F30312224446
:10AB2000002692F85018D4F8C025CA40C4F8C025B1
:10AB30004A4AEA605A6F4A4AAA605A6B22F0800277
:10AB40005A635A6F42F080725A67196B454A0A433A
:10AB50001A635A6B5A631A6C42F0875242F4F61227
:10AB600042F41F6242F00F021A64596C3E4A0A43D3
:10AB70005A6402A948F2FF73CDE902364FF6FF7717
:10AB8000FFF734F800F580600297FFF72FF800F523
:10AB900080600297FFF72AF800F58060FFF726F83B
:10ABA00000F58060FFF722F80846FFF757FA029B8E
:10ABB0002E4AB3FBF2F32E4AC2F83437D5F8FC30F4
:10ABC0002C4A43F08073C5F8FC302B4BC3F8B02FF0
:10ABD0005E601A6842F001021A60D4F8C0354FF482
:10ABE0007A72B3FBF2F3013BB3F1807F08D24FF0EE
:10ABF000E0225361F02385F8233007239661136127
:10AC000007B0F0BD00BFFDE71C4B80E753685168FB
:10AC100013F4800F01F03F01536814BF174A0C4A28
:10AC2000B2FBF1F1054A5268C2F30142C3F3881343
:10AC300001324B435200B3FBF2F368E700380240A5
:10AC40000070004008304004003C0240000000203A
:10AC50000024F40000ED00E0000002400003FA05CB
:10AC6000000000081F9067003357070040420F00A4
:10AC7000D826002055CEACC5001000E000127A00A6
:10AC800082B000230193054B0193019B03EB8000ED
:10AC90000190019B196002B0704700BF502800402E
:10ACA000436D064A1A61C278012A06D100F2CC50DF
:10ACB00058611A684FF080221A60704718000860C7
:10ACC00038B5044600296FD190F81131022B2AD1F2
:10ACD000D0F83821D0F824118A4232D9C378012B18
:10ACE00004BFD0F828315B18A2EB010208BFC0F8FE
:10ACF00028314FF48071D0F82831C0F83821002570
:10AD000092B2A0F81C11C0F82C31C0F83451C0F830
:10AD1000302100F58E714FF045FF2B462A4629461B
:10AD2000204650F055F894F81631012B07D1244AEB
:10AD3000236952F8B42C5A60002384F8163100209D
:10AD400038BDD0F83C31B3FBF1F501FB1535A5B9A1
:10AD5000994212D8D0F8402193420ED24FF480731A
:10AD6000C0E94A55C0E94C55A0F81C3100F58E7178
:10AD70004FF018FFC4F84051CFE7D4F8E435DB6852
:10AD80002BB194F81221032A01D1204698470523BC
:10AD900084F81131002320461A46194650F018F85D
:10ADA0002046FFF77DFFBEE7D0F8E4355B69002B56
:10ADB000C5D090F81221032AC1D19847BFE700BF40
:10ADC000D826002070477047704710B5114C94F892
:10ADD000E630CBB14FF0E022D2F8103D23F006036D
:10ADE000C2F8103DFEF7AAF994F8E63063B1D4F842
:10ADF000EC309B68DB0707D5D4F8E821136823F013
:10AE0000030161F307031360034B4FF480225A617F
:10AE100010BD00BFD8260020003C01402DE9F04FB6
:10AE2000954CD4F8E8305A69D0078DB000F1A18272
:10AE30005A699B691340019300F09B82C3F3074357
:10AE40000293019B190311D5D4F8EC30DFF834924A
:10AE50009E69DB6904F1DC0B1E40360C04F5987723
:10AE60004FF00008DA46002E40F01281029B5A078C
:10AE70000FD5D4F8EC30814E9F69DB691F40BFB21B
:10AE8000A6F118054FF00009A6F1F408002F40F0D4
:10AE90004481019B9DF80470980741BF764BD3F81D
:10AEA000E83002225A61019B002B1BDA724D95F8A3
:10AEB000E6303BB1D5F8E821136823F0030161F3D4
:10AEC00007031360D5F8EC206D48536823F00103A5
:10AED00053606C4BD3F878389847D5F8E8304FF08A
:10AEE00000425A61019B1905C3F3072631D5624D13
:10AEF00000238DF81F3095F8EE318DF81F30614B2F
:10AF000005F1DC00D3F874389847D5F8E820D5F877
:10AF1000EC304FF400619B68516195F8E620C2B1B6
:10AF2000DA0716D595F8F131012B12D19DF81F30B3
:10AF3000032B0ED1D5F8E8311A6842F001021A60ED
:10AF40001A6842F003021A604F4A136943F006037D
:10AF500013613B070AD5484D4A4B05F1DC00D3F895
:10AF60006C389847D5F8E83008225A61FD0615D5A7
:10AF7000414BD3F8E800826922F010028261026A34
:10AF8000C2F34341022902F00F0500F08381062934
:10AF900000F0A781836943F010038361F00634D584
:10AFA000354DD5F8EC205368002723F0010353609A
:10AFB00038464EF007FBB84695F8DD003B46F435C1
:10AFC000FF218342C0F09B81D4F8EC302C484FF035
:10AFD000FF329A614FF00112DA610B2262F3070728
:10AFE00062F307085F61C3F810801A686FF30A12F2
:10AFF0001A60FFF755FED4F8E83021484FF480522C
:10B000005A61204BD3F870389847B10640F19381CC
:10B01000194CD4F8EC30D4F8F40099680268C1F304
:10B020004101022906BF032161F30A026FF30A02FC
:10B0300002605A6842F480725A6008A8FFF70EF85E
:10B04000D4F8E810D4F8EC00CB68099A6FF38D239C
:10B05000CB6085680D48C5F34105284490F85C0035
:10B06000032840F05381002284F8DE204FF4007260
:10B07000A4F8E020092258E1D8260020CC2700209F
:10B08000B42700200000002000ED00E0901A060820
:10B09000F2073BD55FFA88F104EB8103D3F8303136
:10B0A0009D68D4F8EC305B691D40EB0720D594F81F
:10B0B000DF003B680125A8429D6007D11869DBF8D5
:10B0C0007C33C0F312001B1ACBF88C33D9F86038EC
:10B0D0005046984794F8DF30012B09D1B8F1000FA2
:10B0E00006D194F8ED31052B02D15046FFF7D8FD7B
:10B0F000A80742BF3B6802259D60290706D5D9F8FD
:10B100006838504698473B6808229A6008F1010861
:10B11000760804370BF1280BA5E6FB0777D5D8F89E
:10B12000EC305FFA89FA1969586B08EB8A0220FA49
:10B130000AFBD2F8F4204FEACB1B92685FFA8BFB34
:10B140004BEA010B0BEA020B1BF0010F1ED05A6BEE
:10B15000A8484FF0010B0BFA09F122EA01025A63E9
:10B160003368C3F808B0A44B5146D3F86438984705
:10B1700098F8DF305B4509D1B9F1000F06D198F896
:10B18000ED31042B02D19B48FFF78AFD1BF0080F1D
:10B190001EBF33684FF0080BC3F808B01BF0100F48
:10B1A0001EBF33684FF0100BC3F808B01BF0400F00
:10B1B0001EBF33684FF0400BC3F808B01BF0020FFE
:10B1C0001EBF33684FF0020BC3F808B01BF0800FAE
:10B1D0001DD0D5E94C329B1AD5F82421D6F800E0D1
:10B1E00098F8DFB0DEF81800934228BF1346033307
:10B1F000D8F8EC2003920AF1320A9B0808EB8A0A7D
:10B2000080B2984203D9D5E94C03984205D809F198
:10B2100001097F080436283538E6C01AD5F82431EC
:10B22000984228BF1846C31C9B08BBF1000F1CD0D6
:10B23000D5F82811D5F834210144C5F82811D5F8DE
:10B24000301102448A42DEF81800C5F83421D7D103
:10B25000039A95F81C11526B4FF0010C0CFA01F196
:10B2600022EA010203994A63CAE7D5F82821049229
:10B2700082B2DAF8E410033292108C4605925946F5
:10B28000059A8A42D4D0049A52F82120CCF80020A2
:10B290000131F5E747F6F07111423FF47BAE28210A
:10B2A00001FB0531C2F30A12D71CD3F8ACE1D1F887
:10B2B0005CC4BF1000218F420DD1282101FB053352
:10B2C000D3F85C141144C3F85C14D3F868140A442E
:10B2D000C3F868245EE6DEF800804CF82180013176
:10B2E000E9E7D3F8AC110F68C3F8A8760968C3F88A
:10B2F000AC16282101FB0533C2F30A12E5E755F825
:10B30000042B9160AA6B013391605AE6012084F806
:10B31000DE004020A4F8E000A0F56400374CA0F562
:10B3200062401044A04227D80E2262F38D23CB60E6
:10B330004FF400534B61029BDA060BD5304C2E4B79
:10B3400004F1DC00D3F87C389847D4F8E8304FF4A7
:10B3500080125A61029B9B060BD5294C264B04F1A7
:10B36000DC00D3F880389847D4F8E8304FF4001266
:10B370005A610DB0BDE8F08F224CA2F57400A0F523
:10B380001050A04201D80D22CFE71F481F4C104497
:10B39000A04201D20C22C8E71D4CA2F18C70A0F58E
:10B3A0004340A04201D80B22BFE71A481A4C104470
:10B3B000A04201D20A22B8E71848194C1044A04212
:10B3C000FFF458AE174CA2F1B770A0F55850A04248
:10B3D00001D20822A9E71448144C1044A04201D21B
:10B3E0000722A2E712481044124A904234BF0622B4
:10B3F00005229AE7B4270020000000203F420F00FA
:10B40000D8260020DFC810002013FBFE20D6130032
:10B41000FF69180000D3CEFE40771B00C05BB3FE6F
:10B42000C091210040AC2700C01D6AFE40E13300FE
:10B43000803C36FEE09C41004A09012301F01F01D7
:10B4400003FA01F150F822300B4340F822307047E4
:10B450004A09012301F01F0103FA01F150F82230DB
:10B46000194214BF01200020704780EA0120082300
:10B4700041F2210210F4004F4FEA400018BF504043
:10B48000013B80B2F6D170474840082310F0800F8E
:10B490004FEA400018BF80F0D500013BC0B2F5D1A3
:10B4A000704710B50A440C46944200D110BD14F800
:10B4B000011BFFF7E9FFF7E738B50A4605680446C0
:10B4C0000020AA4203D36B1C2360287038BD12F8F9
:10B4D000011BFFF7D9FFF4E782B08DED010A019857
:10B4E00002B07047C31783EA400070479FED087AA7
:10B4F000C0ED020AC7EE007A0023036030EEA77A9F
:10B50000C0ED017AC0EE877AC0ED037A704700BFC4
:10B5100083F9223E80ED010A704700BF90ED017A69
:10B52000D0ED007AC0ED020A30EE877AC0EE876A6D
:10B5300030EE677AE6EE877AB0EE670AC0ED007A01
:10B54000704700BF80ED000A704700BF9FED047A8E
:10B55000C7EE007A77EEA07A80EEA70A704700BFA8
:10B560004E2DA63D002303604360836080ED030AF7
:10B57000704700BFF5EEC00AF1EE10FA06DCF0EEFF
:10B58000407A80ED000AB0EE670A704760EE810AEB
:10B5900090ED007A77EE607AF4EEC07AF1EE10FA70
:10B5A0000ADC77EE200AF4EEC00AF1EE10FA8CBF46
:10B5B000F0EE407AF0EE607AC0ED007AB0EE670A05
:10B5C000704700BFB4EEE00AF1EE10FA07D4B4EE13
:10B5D000C10AF1EE10FA88BFB0EE410A7047B0EE32
:10B5E000600A7047874BB3FBF2F399420DD30023F7
:10B5F0004FF07E52026043608360C36003610023AA
:10B60000836143610362C361704707EE902ADFEDF7
:10B610007E6AB8EE677A07EE901A27EE267AF8EE81
:10B62000677A27EE277AFDEEC77A17EE903A203335
:10B63000402B00F2D880DFED757AB4EEE77AF1EEB8
:10B6400010FAF0EE477A0CDDDFED715A9FED716A6A
:10B65000F0EE676AF4EEC66AF1EE10FA77EEE57A7C
:10B66000F6DCDFED6D6AF4EEE67AF1EE10FA0CD559
:10B67000DFED675A9FED696AF0EE676AF4EEC66A1D
:10B68000F1EE10FA77EEA57AF6D4DFED656AF4EE06
:10B69000E67AF1EE10FA00F39C80DFED626AF4EED8
:10B6A000E67AF1EE10FA03D5DFED5B6A76EEE77A23
:10B6B00027EEA76ADFED5C5ADFED5C6A9FED5C5A0E
:10B6C000DFED5C4AE6EE256ADFED5B5AA6EE265A10
:10B6D00027EE864AE6EE055AF7EE006AE4EE257A92
:10B6E000F0EE665AE7EEA45AE7EEE46A86EEA54A63
:10B6F000DFED4B6A77EE267ABDEEE76A16EE103A7A
:10B700002033402B68D8B4EEE67AF1EE10FA0CDD67
:10B710009FED3F6ADFED3F6AB0EE677AB4EEE67AFE
:10B72000F1EE10FA77EEC67AF6DC9FED3B7AF4EE96
:10B73000C77AF1EE10FA0CD59FED356ADFED376A66
:10B74000B0EE677AB4EEE67AF1EE10FA77EE867A2A
:10B75000F6D49FED337AF4EEC77AF1EE10FA47DDB6
:10B760009FED2A7A77EE677A67EEA76A9FED2E6AD9
:10B770009FED2E7ADFED2E4A9FED2F5AA6EE867AA8
:10B7800027EEA63AE6EE874AB7EE006AA6EEA45A7E
:10B79000B6EE007AE3EE057AF8EE003A36EE676A26
:10B7A00067EEA37A26EE077AB7EE005AC5EE256A51
:10B7B00080ED044A26EE877A26EE866A66EEA77A40
:10B7C00080ED007A80ED016A80ED027AC0ED037AA7
:10B7D00015E7DFED0E6A69E7DFED187AB6EE007A5D
:10B7E000B7EE006AE0E7B7EE004AF0EE445A7FE7B2
:10B7F0009FED0C7AF4EEC77AF1EE10FAB4D59FED16
:10B80000067AAFE720A1070027D4D236DB0F4940E4
:10B81000DB0FC940E4CB1641DB0F49C0E4CB16C1B6
:10B82000DB0FC93FDB0FC9BF9A7C2E36FAAF4FB989
:10B830003587083CF304353FA4AA2ABE0000000067
:10B84000FDEEC07A17EE903A2033402B51D8DFED51
:10B850002A7AB4EEE70AF1EE10FA0CDDDFED276A82
:10B860009FED277AF0EE407AF4EEC77AF1EE10FA07
:10B8700030EE660AF6DCDFED237AB4EEE70AF1EE8D
:10B8800010FA0CD5DFED1D6A9FED1F7AF0EE407ABD
:10B89000F4EEC77AF1EE10FA30EE260AF6D4DFEDB8
:10B8A0001B7AB4EEE70AF1EE10FA18DDDFED127A3A
:10B8B00037EEC00A60EE007A9FED157A9FED156AAB
:10B8C000DFED156AA7EE876A9FED147AE7EE866AC8
:10B8D00060EE275AA7EEA67AA5EE870A7047DFED3D
:10B8E000107AB4EEE70AF1EE10FAE3D5DFED057A4F
:10B8F000DEE79FED0C0A7047DB0F4940DB0FC940C4
:10B90000E4CB1641DB0F49C0E4CB16C1DB0FC93FC6
:10B910009A7C2E36FAAF4FB93587083CA4AA2ABEC6
:10B92000DB0FC9BF000000009FED2F7A70EE077A91
:10B93000FDEEE76A16EE903A2033402B51D8B4EE74
:10B94000C70AF1EE10FA0CDD9FED286ADFED286AD8
:10B95000B0EE677AB4EEE67AF1EE10FA77EEC67AD8
:10B96000F6DC9FED247AF4EEC77AF1EE10FA0CD5EE
:10B970009FED1E6ADFED206AB0EE677AB4EEE67ADC
:10B98000F1EE10FA77EE867AF6D49FED177AF4EEA0
:10B99000C77AF1EE10FA1ADD9FED187A77EE677A22
:10B9A00027EEA77ADFED166ADFED165A9FED166ACD
:10B9B000E7EE265ADFED156AA7EE256A27EE875ACD
:10B9C000E7EE066AE5EE267AB0EE670A70479FED6D
:10B9D000107AF4EEC77AF1EE10FAE1D59FED057A10
:10B9E000DCE79FED0C0A7047DB0FC93FDB0FC94056
:10B9F000E4CB1641DB0F49C0E4CB16C1DB0F494055
:10BA00009A7C2E36FAAF4FB93587083CA4AA2ABED5
:10BA1000DB0FC9BF00000000B5EE400AF1EE10FADE
:10BA200025D007EE902AF8EE670ADFED117A08B507
:10BA3000034660EEA70A0846F0EE406A4BB9FFF7EE
:10BA400055FDFCEEE66A16EE903A99B2BDE8084064
:10BA5000C8E5022B06D0032BF3D1FFF777FDBDE835
:10BA600008407FE5FCF72CFDFCF736FDE9E7704761
:10BA7000BD378635B5EE400AF1EE10FA02D1044B1F
:10BA80000B60704703280CBF024B034BF8E700BF65
:10BA900055840008E58400086D85000890ED0E7A55
:10BAA000B5EEC07AF1EE10FA00F3978030EE607ACE
:10BAB000D0ED015A037867EE255A002B5BD101F0D7
:10BAC0000103D0ED117A002B61D077EE677AF0EEAA
:10BAD000470AD0ED0F6AC0ED110AF5EEC06AF1EE2B
:10BAE00010FA87EE816A55DCD0ED037A26EE276ADC
:10BAF000D0ED056A90ED105A60EE266A76EE857AF2
:10BB000077EEA57A77EE867AF4EEE71AF1EE10FA80
:10BB100000F38480B4EEE72AF1EE10FA8CBFB0EEA9
:10BB2000670AB0EE420A70EE677A90ED044AD0EDF3
:10BB3000024AC0ED135A67EE847A4A07E7EE247A88
:10BB4000B0EE457AA1EE277A80ED125A80ED146AA4
:10BB5000C0ED156A80ED160A08D5F0EEC77AF0EE52
:10BB6000C56AF4EEE67AF1EE10FA6BD580ED107A44
:10BB70000B0756D4704711F001034FF000020CBFC1
:10BB8000F0EE607AF0EE477A0270002B9DD177EEEE
:10BB9000E07A9EE7D0ED0B7AD0ED034A80ED0C1AE7
:10BBA000F5EE407AF1EE10FA04BF9FED285AC5EE8B
:10BBB000267A71EE276A08BFC0ED0B7A81EE265A0D
:10BBC000D0ED0A7A80ED0D5A36EE676AE5EE067A18
:10BBD00024EEA76AC0ED0A7A8AE7D0ED077A80EDF5
:10BBE000081AF5EE407AF1EE10FA04BF9FED176ADD
:10BBF000C6EE077A70EE606A08BFC0ED077A71EE94
:10BC0000277A90ED067A81EE276A76EEC77A80ED84
:10BC1000096AA6EE277A80ED067A49E7B0EE610A56
:10BC200081E7F4EEC71AF1EE10FA08DCB4EEC72A89
:10BC3000F1EE10FA8CBFF0EE471AF0EE421AC0EDAA
:10BC4000101A7047B0EE457A92E700BF83F9223EA2
:10BC5000002301220270C3648364036503644364A8
:10BC60004365836283657047DFED1A7A80ED010AD0
:10BC7000F4EEE70AF1EE10FAC0ED020A80ED031AC5
:10BC8000C0ED051A12DC002383600361002301224A
:10BC900080ED0F2AC0ED0E2A0270C3648364036531
:10BCA000036443644365836283657047B4EEE70AC7
:10BCB000F1EE10FA0CDD81EE007AC0EE207AF0EEA3
:10BCC000006A77EE877A86EEA77A80ED047ADDE760
:10BCD0000023DAE7BD378635F0EEC07AB0EEE07AC1
:10BCE000B4EEE77AF1EE10FAB4BFB0EE676AB0EEE8
:10BCF000476AB5EE406AF1EE10FA46D0B4EEE77A44
:10BD0000F1EE10FA8CBFF0EE675AF0EE475AC5EE2E
:10BD1000866ADFED1F2ADFED1F3ADFED1F4A9FED38
:10BD20001F5A9FED1F3A9FED1F4ADFED1F5AE6EEA7
:10BD3000E23AA6EE834AE6EEA34AB7EE006AA6EE22
:10BD4000A45AA6EE846AE6EE855AC5EE866AB4EE7B
:10BD5000E77AF1EE10FA48BFDFED147AF5EEC00A8B
:10BD600048BF77EEE66AF1EE10FA48BFDFED107AD1
:10BD7000B5EEC00A48BF77EEE66AF1EE10FA48BFAA
:10BD8000F1EE666AB0EE660A7047DFED076ADEE73D
:10BD900039094E3DE3B59E3E88FA163E45FE7F3F8B
:10BDA00099FB243F69A2163EA7DFA834DB0FC93FE9
:10BDB000DB0F4940B7EE007AF0EEC07AF4EEC77AB6
:10BDC000F1EE10FA77EE676A1DD8B1EEE67ADFED94
:10BDD0000F5ADFED0F6A9FED0F6AE7EEA65ADFED0F
:10BDE0000E6AA7EEA56AE7EE866A67EE266AB5EEEA
:10BDF000C00AF1EE10FA44BF9FED087A77EE666A4A
:10BE0000B0EE660A7047DFED066AF0E72716983D48
:10BE1000306E99BC843459BEA40DC93FDB0F494034
:10BE200000000000B0FBF1F301FB130308463BB137
:10BE30001946B0FBF1F301FB13030846002BF7D1C1
:10BE4000704700BF44F25063984203DDA0F50C40F8
:10BE5000A0387047034B9842BCBF00F50C40A0309F
:10BE6000704700BFB0B9FFFF48F6A043984203DD1A
:10BE7000A0F50C40A03870470028B8BFC018704724
:10BE800080EAE073A3EBE0738B4203DB002803DD61
:10BE9000401A704700207047FDD00844704700BF2B
:10BEA000884203DB9042A8BF10467047084670479F
:10BEB00000230361704770B50378012B044635D128
:10BEC0000369214D23B9426812B955F8C42C426068
:10BED000D4ED067A77EE807A013304F11C062361F3
:10BEE000C4ED067A3046FCF767FB626855F8C43C3F
:10BEF0009B1AA268934219D9E06A94ED0A0A4EF09F
:10BF000087FDD4ED057AB4EEE70AF1EE10FA0EDD06
:10BF1000237B4BB955F8C42C236100236260A361D5
:10BF20003046BDE87040C3E70323237070BDD4EDF5
:10BF3000047AD4ED066AF8EE677A022386EEA77AD1
:10BF400084ED067AF1E700BFD82600202DE9F04104
:10BF500004461C30254604F16402064650ED017A81
:10BF6000B1EC010A77EE807A40ED017AFCF724FB10
:10BF700018309042F2D12369294F6268013323615E
:10BF800057F8C43C9B1AA268934246D904F1300882
:10BF9000E86A95ED0A0A4EF03BFDA845D4ED057A16
:10BFA0001CD0B4EEE70AF1EE10FA05F11805EFDD4A
:10BFB000237B83BB57F8C42C626000222361304688
:10BFC000A261FFF775FF04F134002263FFF770FFF1
:10BFD000A26404F14C00BDE8F04169E7B4EEE70A61
:10BFE000F1EE10FAE4DCD4ED047AD4ED066AF8EE52
:10BFF000677A022386EEA77AD4ED0C6A84ED067A7E
:10C0000086EEA77AD4ED126A84ED0C7A86EEA77AD2
:10C0100084ED127A00E003232370BDE8F08100BFB5
:10C02000D826002010B4019C401AA4EB030C00FB9E
:10C030000CFC511A5DF8044B9CFBF1FC0CEB03006B
:10C04000704700BF30EE600A32EE612A71EE600A7E
:10C0500022EE002A82EE200A30EE210A704700BF4D
:10C06000D1ED007ADFEDE16A37EEA67ABDEEC76A60
:10C0700016EE103A2033402B00F25882F4EEE67AA6
:10C08000F1EE10FA0CDDDFEDDB5A9FEDD96AF0EE30
:10C09000476AF4EEC66AF1EE10FA37EE657AF6DC1E
:10C0A000DFEDDE6AB4EEE67AF1EE10FA0CD5DFEDE4
:10C0B000D15A9FEDD16AF0EE476AF4EEC66AF1EE0E
:10C0C00010FA37EE257AF6D4DFEDC86AB4EEE67AD8
:10C0D000F1EE10FA40F30282DFEDC96A36EEC77A5C
:10C0E00067EE076A9FEDC76A9FEDC75ADFEDC75A33
:10C0F000A6EE865A9FEDC66AE6EE855A27EE264AD8
:10C10000A6EEA56AA4EE067AF0EE474ABDEEE77AFF
:10C1100017EE103A2033402B00F205829FEDB87ADB
:10C12000F4EEC77AF1EE10FA0CDD9FEDB26A9FEDE6
:10C13000B07AF0EE676AF4EEC76AF1EE10FA77EEC5
:10C14000C67AF6DC9FEDB57AF4EEC77AF1EE10FA16
:10C150000CD59FEDA86A9FEDA87AF0EE676AF4EE21
:10C16000C76AF1EE10FA77EE867AF6D49FED9F7AE1
:10C17000F4EEC77AF1EE10FA40F3DB819FEDA07A7E
:10C1800077EE677A27EEA77ADFED9E6ADFED9E5A9B
:10C190009FED9E6AE7EE265ADFED9D6AA7EE256ABF
:10C1A00027EE874AE7EE066AE4EE267AB0EE675A93
:10C1B00091ED017ADFED8D7A77EE276ABDEEE66AC2
:10C1C00016EE103A2033402B00F2A681B4EEE77A47
:10C1D000F1EE10FA0CDDDFED875ADFED857AB0EE77
:10C1E000666AB4EEE76AF1EE10FA76EEE56AF6DC1E
:10C1F000DFED8A7AF4EEE76AF1EE10FA0CD5DFEDA6
:10C200007D5ADFED7D7AB0EE666AB4EEE76AF1EE54
:10C2100010FA76EEA56AF6D4DFED747AF4EEE76AEA
:10C22000F1EE10FA40F39B81DFED757A77EEE66A66
:10C2300066EEA67ADFED735A9FED734A9FED736A3F
:10C24000A7EEA54ADFED725AA7EE846A66EEA73A1A
:10C25000E7EE865AE3EEA56A66EEC52A24EEA63A14
:10C26000B0EE666AFDEEC77A17EE903A2033402BA7
:10C2700000F24F81DFED627AB4EEE77AF1EE10FA68
:10C280000CDDDFED5C5ADFED5A7AF0EE476AF4EE32
:10C29000E76AF1EE10FA37EE657AF6DCDFED5F7AE9
:10C2A000B4EEE77AF1EE10FA0CD5DFED525ADFED7D
:10C2B000527AF0EE476AF4EEE76AF1EE10FA37EEE2
:10C2C000257AF6D4DFED497AB4EEE77AF1EE10FA8A
:10C2D00040F33A81DFED4A7A37EEC77A67EE077AA4
:10C2E000DFED485A9FED484ADFED486AA7EEA54AC0
:10C2F000DFED475AE7EE846A67EE273AE7EEA65A83
:10C30000A3EEA57AF0EE476AD1ED027ADFED375A57
:10C3100037EEA57ABDEEC74A14EE103A2033402B13
:10C3200000F2EC80F4EEE57AF1EE10FA0CDDDFEDD0
:10C33000313A9FED2F4AF0EE475AF4EEC45AF1EE2F
:10C3400010FA37EE637AF6DCDFED345AB4EEE57AB4
:10C35000F1EE10FA0CD5DFED273A9FED274AF0EE0B
:10C36000475AF4EEC45AF1EE10FA37EE237AF6D4B7
:10C37000DFED1E5AB4EEE57AF1EE10FA40F3FA80E2
:10C38000DFED1F5A35EEC77A67EE075A9FED1D4A5B
:10C390009FED1D2ADFED1D3AA5EE842A9FED1C4A74
:10C3A000E5EE823A67EE251AA5EEA34AA1EE847A5D
:10C3B00025EE072A64EE871A26EE821A26EE077A01
:10C3C00026EEA10AFDEEE75A15EE903A2033402BF7
:10C3D00000F28F80DFED0A5AF4EEE57AF1EE10FA02
:10C3E00027DDDFED043A9FED024A19E0DB0FC93F7C
:10C3F000E4CB1641DB0FC940E4CB16C1DB0FC93FCC
:10C40000DB0F49409A7C2E36FAAF4FB93587083C8E
:10C41000A4AA2ABE00000000DB0FC9BFDB0F49C081
:10C42000F0EE675AF4EEC45AF1EE10FA77EEE37AC2
:10C43000F6DC5FED065AF4EEE57AF1EE10FA0CD573
:10C440005FED143A1FED144AF0EE675AF4EEC45A49
:10C45000F1EE10FA77EEA37AF6D45FED185AF4EE07
:10C46000E57AF1EE10FA40F390805FED1B5A75EE1D
:10C47000E77A27EEA74A5FED1D5A5FED1D3A5FEDA3
:10C480001D0AE4EE253A67EE845AE4EE230A5FEDD6
:10C49000203AE4EE203AE5EEA37A64EEA74A65EE90
:10C4A000275AA6EEA42AE6EEE51A67EEC67A31EE22
:10C4B000241A75EEC05A80ED007AC0ED017AC0ED05
:10C4C000026A80ED031AC0ED041AC0ED052AC0ED22
:10C4D000065A80ED072A80ED083A70475FED326A10
:10C4E000B4EEE67AF1EE10FA7FF5FAAD5FED356A5B
:10C4F000F4E55FED385AF0EE657ADAE71FED3B2A96
:10C50000F0EE421AB0EE420AB0EE421AB0EE427AB3
:10C5100058E75FED406AF7E61FED423AF0EE432A36
:10C52000B0EE436A9EE61FED455A41E65FED474A8D
:10C53000ECE51FED477AF4EEC77AF1EE10FA7FF5DD
:10C5400021AE1FED4A7A1BE65FED4D7AB4EEE77A35
:10C55000F1EE10FA7FF5C2AE5FED507ABCE65FED0A
:10C56000527AF4EEE76AF1EE10FA7FF561AE5FED14
:10C57000557A5BE65FED585AB4EEE57AF1EE10FAC3
:10C580007FF502AF5FED5B5AFCE65FED5D5AF4EEBE
:10C59000E57AF1EE10FA7FF56CAF5FED605A66E771
:10C5A0000023036143618361C361036003624362EB
:10C5B0008362C3624360036343638363C3638360D3
:10C5C000036443648364C364C3607047D1ED017A3C
:10C5D00091ED007AD0ED044A90ED065AD0ED075A5D
:10C5E00090ED050AD0ED080AD0ED0A1AD0ED0C2A1C
:10C5F00090ED0D3AD0ED0E3A90ED091A90ED0B2A20
:10C60000F8EEE76AD1ED027AB8EEC77AF8EEE77A8B
:10C6100026EEA64AA7EE275AE7EE074AB0EE446A8E
:10C6200075EE875AA7EE076AE7EE272AE7EEA73AE4
:10C63000A7EE260AE7EE260AE6EEA71AA6EEA73A26
:10C6400031EE041AC0ED044A90ED0F4AD0ED104AC5
:10C6500080ED065AC0ED075A90ED115AD0ED125AEE
:10C66000C0ED0E3AA7EEA76A34EE274A74EE874A69
:10C6700075EEA75A35EE265A32EE262A80ED0F4A7D
:10C68000C0ED104A80ED115A80ED050AC0ED080A90
:10C6900080ED091AC0ED0A1A80ED0B2AC0ED0C2AB4
:10C6A00080ED0D3AC0ED125A90ED004A90ED025A1D
:10C6B000D0ED014AD0ED133AD0ED035AA7EE064A69
:10C6C000B0EE457AA7EE867AE6EE864AF7EE007A75
:10C6D00073EEA77A35EE866AC0ED137A80ED004AD4
:10C6E000C0ED014A80ED027A80ED036A704700BF19
:10C6F00010B50024034684468646002C00F00D81C8
:10C70000DEED006A9CED007AD3ED007AE6EEC77AA2
:10C71000012CC3ED007A00F00F81DEED016A9CED83
:10C72000047AE6EEC77A032CC3ED007A6CD1DEED15
:10C73000026A9CED087AE6EEC77AC3ED007AD2ED84
:10C74000007A90ED085AD0ED0C5AD0ED044A92EDE3
:10C75000017AD2ED026A92ED036AA7EEE47AE7EE7F
:10C76000C56AA7EEE56A90ED095AD0ED0D5AE7EEDD
:10C77000456AA5EEC76AD0ED0E5AA5EEE66A81EDD0
:10C78000036A90ED0F5AC1ED026AC6EE055AC1ED7B
:10C79000035A90ED0B6AE5EEC66AC1ED026A90EDB0
:10C7A0000A5A81ED017A86EE856A81ED026AD0ED42
:10C7B000066AA6EE667A81ED017AD0ED076AA5EEEB
:10C7C000E67A81ED017A90ED055AC1ED007AC7EE67
:10C7D000056AC1ED016A90ED017AE7EE667AC1ED76
:10C7E000007A90ED027AE7EE467AC1ED007A90ED9C
:10C7F000037AE7EE657AC1ED007AD0ED006A87EE44
:10C80000A67A81ED007A10BD9EED007ADCED016A1A
:10C81000D3ED017AE7EE667A022CB1EE476AC3EDFA
:10C82000017ADEED016A9CED057AE6EEC77AC3ED8A
:10C83000017A40F0AC80DEED046A9CED007AD3ED25
:10C84000047AE6EEC77A012CC3ED047A40F28780C1
:10C85000DEED056A9CED047AE6EEC77A032CC3EDA3
:10C86000047A7FD19EED066ADCED086A93ED007ACA
:10C87000E6EE667AC7EE876AC3ED046A9EED086A43
:10C88000DCED006AD3ED087AE6EE667A012CC3EDA2
:10C89000087A70D99EED096ADCED046AE6EE667AE4
:10C8A000032CC3ED087A07D19EED0A6ADCED086A15
:10C8B000E6EE667AC3ED087A93ED086AD3ED0C7A5A
:10C8C000C6EE076A032CC3ED086A9CED006ADEED34
:10C8D0000C6AE6EE667AC3ED0C7A9CED046ADEED36
:10C8E0000D6AE6EE667AC3ED0C7A07D19EED0E6A0C
:10C8F000DCED086AE6EE667AC3ED0C7AD3ED0C6ADD
:10C90000C6EE877AC3ED0C7A013414330EF1100EA3
:10C910000CF1040C002C7FF4F3AED3ED047A93ED0C
:10C92000007A93ED086AC7EE876AC6EE077AC3ED10
:10C93000046AC3ED087AE1E7DEED006A9CED016A66
:10C9400093ED017AD3ED027AA6EEC67A83ED017AF1
:10C950009CED027AE7EE667AC3ED027A6BE793ED1F
:10C96000007A87E793ED007AC7EE876A022CC3ED61
:10C97000046AC9D082E7C7EE876AC3ED086AC3D0EC
:10C980009CED006ADEED0C6AD3ED0C7AB2E79CED0B
:10C99000027AD3ED027AE6EE077A032CC3ED027A2F
:10C9A000DCED066A9EED017AE6EEC77AC3ED027A07
:10C9B0007FF441AFDEED026A9CED0A7AE6EEC77ABB
:10C9C000C3ED027ABBE600BF10B584B00C46024648
:10C9D00069461030FFF78CFEDDED006A9DED017AAF
:10C9E000DDED027AB6EE006A66EE866A27EE067A1A
:10C9F00067EE867A0120C4ED006A84ED017AC4ED09
:10CA0000027A04B010BD00BF20EE000AFEEE007AEC
:10CA100060EE277A60EEA00A9FED020AC7EEA00A38
:10CA200051F05ABF54F82D4008B54EF0DFFF07EE25
:10CA3000900AF5EEC07AF1EE10FAACBFB1EEE70A5B
:10CA40009FED010A08BD00BF0000000060EEA00AD3
:10CA5000E0EE000AB1EEE00A704700BF21EE011AD5
:10CA6000A0EEA01AA0EE001AB1EEC10A70472DE99F
:10CA7000F74F90469DF83020002A14BF4FF0300940
:10CA80004FF020090D9A1C1E05460F46BABF64429E
:10CA90000123002312F8011B01B12CB9A24663B196
:10CAA00000240D9EA41B12E0013CF3E7BD4204D21A
:10CAB000494628460193C047019BBAF1010AF5D2C5
:10CAC000EFE7BD4203D228460193C047019B06EB26
:10CAD000040B16F8011B0029F3D133B15446002C86
:10CAE00007DCBAF1000FA8BFD344584603B0BDE835
:10CAF000F08FBD4202D249462846C047013CEEE7CE
:10CB00000FB437B50B4D06ABD5F83C1753F8042BD3
:10CB1000D5F8380701934CF027FA0446D5F8A00061
:10CB200003F092FE0028F9D0204603B0BDE8304063
:10CB300004B07047D82600200EB403B503AB0849F3
:10CB400053F8042BCDE9003001A84CF00DFA019BFD
:10CB500000221A7002B05DF804EB03B0704700BF0A
:10CB60000B8600080CB430B5294CD4F84037A5B07A
:10CB70001BB9D4F84437002B38D094F84837994281
:10CB800006D9012303FA00F0D4F84C3718422DD00F
:10CB900054F8C41C4FF47A7304A8B1FBF3F203FBFE
:10CBA00012131C49FFF7C8FF04AB0344289A1A4923
:10CBB0000393054629AB03A802934CF0D5F9039BD8
:10CBC000591C03910A211970039B0246591CD4F881
:10CBD000400703910021197068B103681B6A03B113
:10CBE0009847D4F8400704A903F0FCFD25B0BDE840
:10CBF000304002B07047D4F84437002BF6D0022101
:10CC00002A4400910A44FD2004A924F00BFCEDE71E
:10CC1000D82600202DA80608AF85000830B54FF4AF
:10CC2000004087B022F0B2FD0446A0B34FF40041AB
:10CC300022F00EFF02281CD1226848F201039A421A
:10CC400029D1234C002584F8E4594FF400404BF0DF
:10CC5000F1FB00B3D4F8503783421ED0D4F82C38FF
:10CC600083422FD0D4F8083998422ED0C4F84457C4
:10CC700011E00023022294F90400CDE901234FF4CE
:10CC8000612200924FF400411A4622F03BFF104B04
:10CC9000C3F8400728B907B030BD04F5EA63C4F80B
:10CCA00044370C4B04930C4B03930C4B02930C4BEB
:10CCB00001930C4B00930C4A0C4B02210020FFF710
:10CCC00051FFE8E704F62C03E9E704F60813E6E76A
:10CCD000D826002039A8060842A806084BA806084E
:10CCE00057A806085DA806088DAE060805A8060820
:10CCF000174A38B5D2F8E849033004EB9003B3F58E
:10CD0000007F19D802F6EC15C2F8E839114A02EB97
:10CD1000810120F00300D1F8F420C3F50073104422
:10CD2000C1F8F4000C4A9B000421002005EB8404A8
:10CD3000FFF718FF204638BD0021084A0846FFF7D4
:10CD400011FF074A136843F0007313600024F1E7F2
:10CD5000D8260020D037002069A806088CA806082D
:10CD6000A80101202DE9F84F0268DFF8A4800646EB
:10CD7000002358F833108A420BD1DDB20D2D0CD9A7
:10CD8000204A00210520FFF7EDFE00242046BDE8E3
:10CD9000F88F01330E2BECD1F2E71B4F07EB850A1E
:10CDA0004FEA8509DAF8A4B0BBF1000F1AD10A21C5
:10CDB0006420FFF79DFF0446CAF8A40028B9014685
:10CDC000124A0520FFF7CEFEE0E76422594654F0F0
:10CDD000C2FDDAF8A43008EBC505C3E90053DB61F6
:10CDE0005B63DB644F447179D7F8A440182000FBE3
:10CDF000014300221C46C3E903229E601A750434D5
:10CE0000C4E700BF9AA80608D8260020BFA80608D5
:10CE1000F01A060803685A1C026019700368090AB0
:10CE20005A1C02601970704703685A1C026019701E
:10CE300003685A1C02600A0A1A7003685A1C0260CE
:10CE40000A0C1A700368090E5A1C026019707047A8
:10CE500003685A1C02600A0A1A7003685A1C0260AE
:10CE60001970704738B504460068154654F03AFB0F
:10CE700023682B44236038BD03685A1C026018786D
:10CE8000704703685A1C02601A4612F8021B0260BF
:10CE9000587841EA0020704710B502681146531CCB
:10CEA000036011F8024B0160D31C51780360937842
:10CEB0001B0443EA0123111D0160D078234343EA98
:10CEC000006010BDD1E900329A4206D05A1C0A60B7
:10CED00008B11B7803700120704700207047D1E92A
:10CEE00000239B1A012B10B50446084604DDFFF70A
:10CEF000C8FF2080012010BD0020FCE730B50A44A7
:10CF00000446914201D1002011E014F8013BA3F145
:10CF10004100192811F8010BA0F1410598BF2033F9
:10CF2000192D98BF20301B1A02D10028E9D130BD3D
:10CF30001846FCE76FF00042E0E710B50288C378BE
:10CF4000A2F5FA62910840F2B554013B04FB0133AB
:10CF500081780C24013902F0030204FB02120D490E
:10CF6000847901EB42021821B2F8D02013440279EF
:10CF700001FB0322437900893C2101FB0233064A6D
:10CF8000224401FB03224FF47A730021C2FB030108
:10CF900010BD00BF901A060880436D382DE9F0419E
:10CFA00090461F4605464FF47A72002340463946A4
:10CFB0004EF07AFE284B3C21034493FBF1F201FB37
:10CFC0001233AB7192FBF1F301FB13226A7140F251
:10CFD000B551182293FBF2F402FB143394FBF1F2E7
:10CFE00001FB1244B4F5896F2B714FEA82032EDAEC
:10CFF00040F2DA2294422CDCB4F5B77FB4BF0021B2
:10D000000121164A182000FB01220B2632F81600D7
:10D01000A04201DD013EF9D103F5FA630B442B80F8
:10D02000731CAB700C2303FB01660D4B03EB460630
:10D030000134B6F8D030E41AEC704FF47A72002361
:10D04000404639464EF030FE2A81BDE8F08103218A
:10D05000D7E70221D5E700BF80BC92C7601B060856
:10D06000901A0608F0B5274D06460F460FCD8DB035
:10D070006C460FC40FCD0FC495E80F0084E80F0075
:10D0800016F003033AD1642196FBF1F201FB126220
:10D0900042B94FF4C87296FBF2F302FB1363003BF4
:10D0A00018BF0123721EC3F11D03002A019340F231
:10D0B0006D13104606FB03F3B8BFB01C03EBA000D2
:10D0C0006FF0630392FBF3F318444FF4C87392FBC1
:10D0D000F3F210440630694600240725013F51F859
:10D0E000042BA74202EB000393FBF5F0C0EBC0005A
:10D0F000A3EB000004D1101A0DB0F0BD0123D1E75D
:10D100000134ECE7C01B0608084BD3E9621251EA70
:10D11000020309D0064B53F8C43C5B1842F10002ED
:10D12000C0E900320120704700207047D03700204E
:10D13000D826002037B505466846FFF7E5FF0446C8
:10D1400038B1DDE900232846FFF728FF204603B069
:10D1500030BD40F2011328806B80A880A87128811F
:10D16000F4E700BF8842F0B54FF0010461D301FB42
:10D1700004F4B0FBF4FC8C45F9D284B3002A45D00A
:10D18000002511E0BCF1090F2646CCBF3722302222
:10D190009444B14283F800C0744603F1010305F1E1
:10D1A00001051CD8B0FBFEFCB4FBF1FE04FB1C0027
:10D1B000002DE7D1BCF1000FE4DCA1420BD8B0FB9D
:10D1C000FEFCBCF1000F74460EFB1C00BEFBF1FE22
:10D1D000D8DCA142F3D90CF1300C03F801CB0022CA
:10D1E0001A70F0BDBCF1090F2646CCBF4FF0570EA8
:10D1F0004FF0300EF444B14283F800C02C4603F1E6
:10D20000010302F10102EAD8B0FBF5FCB4FBF1F531
:10D2100004FB1C00002AE5D1BCF1000FE2DCA142B6
:10D22000D9D8B0FBF5FC2C4605FB1C00B5FBF1F58D
:10D23000F2E78446002AA3D1E8E700BF0028BCBF7C
:10D240002D23404270B5B8BF01F8013B09280446C0
:10D250004FF0010307DD03EB83035B00B0FBF3F248
:10D26000092AF8D83BB3164D4FF0000C0AE0092A02
:10D270008CBF572130210A44092B0EF8012B16D9F7
:10D2800071460346A5FB0320B4FBF3F25CEA0206F9
:10D290008E464FEAD00003FB12440CF1010CE6D19C
:10D2A000092B01D9B446EBE730320EF8012B0023ED
:10D2B0008EF8003070BD8E4600238EF8003070BDB1
:10D2C000CDCCCCCC90422DE9F0410B46044615461E
:10D2D0000AD2B0FBF5F6134A05FB16441846135D57
:10D2E00000F8013BBDE8F081B0FBF2F69642B6FBD8
:10D2F000F2F706D20B4A05FB1767D15D03F8011B55
:10D30000EAE7BA42B7FBF2F807D9064A05FB1878F4
:10D3100012F8081003F8011BEDE74046FFF7D2FFB3
:10D320000346F2E790AA0608B5EEC00ADFED307AB0
:10D33000F1EE10FACCBF30EE270A30EE670ADFEDCF
:10D340002D7A20EE270A70B5FDEEC07A86B017EE72
:10D35000904A054684EAE470002303A9A0EBE47038
:10D36000CDE9003302934BF0FDFF002CACBF20232E
:10D370002D2303A88DF800304DF0A4FE01286E4641
:10D3800026D002282DD003281CD003A9304654F003
:10D39000EAFA30464DF096FE0338C4B222463146D2
:10D3A000284654F09FF800232B5528464DF08AFE5E
:10D3B0002E232B5401303119284454F0F0FA28461A
:10D3C00006B070BD302303A930468DF80130DEE78A
:10D3D00043F23002302303A9ADF801208DF8033069
:10D3E000D4E743F2300303A93046ADF80130CEE76D
:10D3F0006F12033A00007A440378202B024600F1B2
:10D400000100F9D0092BF7D02D2B25D02B2B00F0C4
:10D41000A280B7EE000AA3F13001C8B209289FED3F
:10D42000587A10D8F2EE046A07EE901AF8EEE77A0E
:10D4300012F8013FE7EE267AA3F13001C8B20928BD
:10D44000B0EE677AF0D92E2B62D003F0DF03452BC4
:10D4500007D020EE070A70475378BFEE000A024655
:10D46000D9E710B451782D297AD02B290BBF9178A8
:10D47000A1F13003A1F13003013208BF0232092BC0
:10D4800064D80024002303EB830301EB430312F869
:10D49000011FA1F130000928A3F13003F3D9B3F53E
:10D4A0009A7F1A4628BF4FF49A72072B64D9DFED92
:10D4B000356A1346F7EE007A083B072B67EEA67A2B
:10D4C000FAD802F00702DAB1F2EE046A012A67EE36
:10D4D000A67A15D0022A67EEA67A11D0032A67EE43
:10D4E000A67A0DD0042A67EEA67A09D0053A67EE2F
:10D4F000A67A05D067EEA67A012A18BF67EEA67A4B
:10D5000034B387EE277A5DF8044B20EE070A7047A4
:10D510005378A3F13001C8B2092802F1010294D86E
:10D52000F2EE046AF0EE665A07EE901AF8EEE77A29
:10D5300012F8013F87EEA66AA3F13001C8B20928AC
:10D5400066EEA56A37EE067AEED97EE7F7EE007A48
:10D5500027EE277AD7E75378B7EE000A02465AE754
:10D560009178A1F13003092B02F1020288BFF7EE96
:10D57000007AC6D8012485E7F7EE007AA3E700BF5A
:10D580000000000020BCBE4C0378202B024600F1B6
:10D590000100F9D0092BF7D0303BDBB2092B4FF05B
:10D5A00000000AD812F8011F00EB8000303903EBAD
:10D5B0004000CBB2092BF5D9704770470378202B78
:10D5C000024600F10100F9D0092BF7D02D2B0CBF3A
:10D5D0000246012092F800C0ACF13001CBB208BF86
:10D5E0004FF0FF30092B4FF0000302D903FB00F08E
:10D5F000704712F801CF03EB830301EB4303ACF157
:10D6000030015FFA81FCBCF1090FEEE710B5002391
:10D61000802804D893420AD2C854581C10BD9342A3
:10D6200005D060F07F04CC54C0090133F0E74FF01F
:10D63000FF30F3E738B50C468D18AC4200D138BD49
:10D6400014F8011BFDF711FFF7E770B51249134CF1
:10D65000134E01220020FFF7EDFF228862B1A31DC7
:10D66000B34217D2A518B54214D2052A12D92146C1
:10D67000FFF7E0FF2C46F0E721460222FFF7DAFF32
:10D6800063880849084AC31A641A5842A2F89041AC
:10D69000584170BD0020FCE7004000080140000830
:10D6A00000800008FC3F0008D037002003682DE907
:10D6B000F04104464068134483421AD80D468E1840
:10D6C00004F10C074FF00008B54202D16069BDE8D3
:10D6D000F08123695A1C2261234415F8011B197338
:10D6E000042AF1D139462046FBF74FFDC4E90480F6
:10D6F000EAE74FF0FF30EAE7034AD2F8943123EA31
:10D700000000C2F894017047D03700200346064954
:10D710000648884201D3002070470288C2F30B02FA
:10D720009342F9D01430F4E7A8090708BC040708AD
:10D7300013B542880B460446C2F30B02002118467B
:10D74000019254F008F9216903460A48814209D33D
:10D750000948019A814205D2184602B0BDE810403E
:10D7600053F0C0BE21B1184602B0BDE810400847D2
:10D7700002B010BDA8090708220E070810B4B0F9BE
:10D7800002404288002C0B4641685DF8044BBEBF46
:10D79000C2F30B02DBB203FB0211C9E730B5094B40
:10D7A000094CA34200D330BDB3F902205988002AA6
:10D7B00006DA5A68DD68C1F30B0100FB01222A601A
:10D7C0001433EEE7BC040708A809070830B5024681
:10D7D0000144002012F8015B082480EA050313F0DD
:10D7E000010F4FEA50001CBF80F08C03D8B2631EBB
:10D7F00013F0FF044FEA5505EFD18A42EAD130BD5C
:10D800002DE9F04F87B0CDE9021200258046049340
:10D810000195039B404603EBC50AFBF7BFFBEC00F9
:10D82000024600286DD0002201214046FBF7A0FBF4
:10D830000246002865D098F80430990761D5F02198
:10D840004046FBF7B5FB024600285AD0039BA4F1E3
:10D8500008024FF0000B012713443C465E46059337
:10D86000029B002B55D0082C53D804F1FF3943FA02
:10D8700009F909F0010949464046FBF772FB0246E7
:10D8800000283ED0002201214046FBF771FB0246F2
:10D89000002836D098F8041001F0600CBCF1600F3D
:10D8A0004FEAD11016D0029B1BB1082C01D881453C
:10D8B00027D1002841D01AF8061039437F000134DF
:10D8C00017F0FF070AF80610E4B2C9D10136F6B224
:10D8D000082E1CD1402C10D9072150460592FFF785
:10D8E00075FF9AF80710059A814206D10135EDB20D
:10D8F000BBF1000F05D0CDF804B0049B1B78AB4200
:10D9000087D8049B10461D7007B0BDE8F08F012733
:10D91000A6E75DB1019BA34208D9059B9A5D17421A
:10D9200014BF4FF001094FF00009A4E7019B1B1B36
:10D93000D3F1000949EB03099DE7880940EA511139
:10D9400011F0010F1AF8061008BFA34621EA0701DB
:10D95000B4E700BF0123037750F8043C0BB118383B
:10D960001847704790F83420034602F0FF0012B1C8
:10D97000002283F8342070474FF40063838170479E
:10D98000064A002352F8041B814204D00133042BC1
:10D99000F8D1002070470120704700BF605D002073
:10D9A0003248F0B5C38B058AB0F92840B0F916604B
:10D9B000B0F922C0B0F93070ED1A838B6B43B0F927
:10D9C000265004EBE334ED0295FBF4F505EBE3356B
:10D9D000A5F57A6E0EFB0EF42313B0F91840C5625C
:10D9E0000EFB06F60EFB04FEB0F920405C4303FB81
:10D9F0000CFCF612241406EBEC2C04EB6E34B0F99C
:10DA00001460438B02340CEB860CA410466B04F5B7
:10DA100000440CFA07FC63430CF1020C4CF250304A
:10DA2000DC0BA6EBAC0640FA07F3734355BF5B0073
:10DA3000B3FBF4F3B3FBF4F35B0071B1181240F6DF
:10DA4000DE34404360430A4C00145C4300EB244046
:10DA500000F6CF6003EB20130B6022B10A235D4375
:10DA600008352D1115600120F0BD00BF605D00205C
:10DA700043E3FFFF01207047012070472DE9F84381
:10DA80005E4F1546BC6BBA8FB7F84290C2EB2413B9
:10DA90005200C2EBE402B7F93E40624303FB03F4D9
:10DAA000B7F9403024135C43A41304EBE224B7F924
:10DAB00046307C650E46A4F5FA3181FB01CE4FEA73
:10DAC000E37803FB0EF20CFB0822A3FB0C38904416
:10DAD000B7F9442082FB01021B0A120343EA0863E0
:10DAE00042EA105200031B1842EB282202F50042C2
:10DAF000A3FB093809FB02884FEAE8734FEA680282
:10DB000053EA68084FF000006CD0B7F94C904FEA28
:10DB1000E97809FB0EFE0CFB08EEA9FB0C9CE64421
:10DB2000B7F94AC08CFB01814FEA414C4FEA4841AA
:10DB300011EB0909B96D4CEAD83C4EEB0C0CC1F560
:10DB4000801E0EF00048B7F9481048EA5E0810EB56
:10DB500009004FEACE7EBEEB00000CEBC10168EB82
:10DB6000010C40F63548A0FB080108FB0C114EF0F3
:10DB70009BF8B7F952304FEA613E4FEA503C4CEA0D
:10DB8000C14C03FB0EF24FEAE3790CFB0929A3FB1E
:10DB90000C324A4403FB0EFE0CFB02EEA3FB0C3CD2
:10DBA000B7F95020E6445B0E43EACE1313EB000CAA
:10DBB000804602FB01F34FEAE27941EB6E6EA2FB75
:10DBC000082809FB00314144D00C40EA41301CEBED
:10DBD0000000B7F94E304EEBE141000A40EA016027
:10DBE00000EB03100EB1000A306025B104EB840491
:10DBF000803424122C600120BDE8F883605D002091
:10DC000031B10A4BD3ED1D7AFDEEE77AC1ED007A12
:10DC100052B1064B9FED067AD3ED1E7A67EE877AF6
:10DC2000FDEEE77AC2ED007A01207047605D0020CA
:10DC30000000C8422DE9F74FCDE90012554AB2F86D
:10DC40008A30D16FB2F88660B2F88C701B02C91AA4
:10DC5000B2F888306EEB0E0EA3FB010403FB0E44FA
:10DC6000B2F88430C00940EA44601B04C018A6FB27
:10DC7000013506FB0E55B2F882604FEA132343EAE2
:10DC800005634FEAC6364FEAE41444F100049B19D9
:10DC9000A7FB012607FB0E664FEAD25242EA462254
:10DCA0004FEA252545F10005F61512F5FA6C46F107
:10DCB000000BBCF5FA6F7BF100074CDAA2FB02788F
:10DCC0004FF0050A02FB06F908EB4909A7FB0A78A1
:10DCD0000AFB09884FEA570949EAC879BF08B0EB3F
:10DCE000090047EA887764EB6804DB1B2A4F65EB81
:10DCF000A805BC454FF0FF377BEB070720DA40F65D
:10DD0000AC57D21946F100065643A2FB027202EB51
:10DD100046064FEAC608FA00BA1A48EA577866EB90
:10DD20000808101844EB08044FF00B08A7FB087212
:10DD300008FB06267F0847EAC677DB1B65EB66050E
:10DD400001FB0EFEA1FB011202EB4E0EC90F41EAD0
:10DD50004E01BCEB010C009A9AB10E4AD2F8901019
:10DD6000A1FB032301FB0535520D42EAC522121A1D
:10DD70004FEA6555009B65EB0404D20B42EA44422E
:10DD80001A60019B0BB1C3F800C0012003B0BDE8CD
:10DD9000F08F00BF605D002024FAFFFF0120704774
:10DDA0000A4B18680A4B10B5D3F89440001BFA28A8
:10DDB00009D811B1D3F89800086012B1D3F89C309B
:10DDC0001360012000E0002010BD00BF14260020D9
:10DDD000605D0020034B0022C3E92822C3E92A2208
:10DDE00001207047605D00200A4B1A680A4BD3F887
:10DDF000AC10521AFA2A9FBFD3F8A020C286D3F8DB
:10DE0000A420D3F8A8309DBF0287438701200020BB
:10DE1000704700BF14260020605D002090F85F323C
:10DE200030B53BB990F85D1290F85E320124DAB259
:10DE3000914200D830BDB0F8665204FA03F22A438A
:10DE4000A0F866220133F2E7437913F001031FBF04
:10DE5000D0E90732C0689B1A00F1FF3014BF1840A8
:10DE600018467047437913F002031FBFD0E9093207
:10DE700000699B1A00F1FF3014BF984318467047A1
:10DE800010B5437913F0010301460DD0FFF7DCFF15
:10DE900060B10A6A4B69C8689B5C0132B2FBF0F45E
:10DEA00000FB1422DBB20A62184610BD0346FBE7F2
:10DEB00043799B070AD5436A8269D154436A026950
:10DEC0000133B3FBF2F102FB11334362704741713E
:10DED0007047D0E90920131A584258417047024B45
:10DEE000D3F8B0305B681847605D0020024BD3F870
:10DEF000B03008309B681847605D002001207047F3
:10DF000001207047012070470120704731B10C4B50
:10DF1000D3ED2D7AF8EEE77AC1ED007A7AB1084BAD
:10DF2000DFED086AD3F8B830A3F5D543333B07EEED
:10DF3000903AF8EEE77A87EEA67A82ED007A70479B
:10DF4000605D00200000C842704700BF054B03EB36
:10DF5000C00040F2FF739942A8BF1946A0F8C01054
:10DF6000704700BF605D0020044B03EB8000D0F8D9
:10DF70001C310BB19B681960704700BF605D0020C9
:10DF8000084AD2F85C315BB140B19968B2F86021BF
:10DF9000054BB3FBF2F35B100B6070479B68186096
:10DFA000704700BF605D002040420F000C4A1378AC
:10DFB0007BB10C4B93F8621159B193F8631159B1CD
:10DFC00050680021FA2883F86311A8BF4FF0FF3092
:10DFD00070476FF0010070476FF00200704700BF9C
:10DFE00010090020605D00200B4B93F864216AB19A
:10DFF00093F865216AB1002283F86521074B986880
:10E00000B0F5967FA8BF4FF0FF3070476FF001006A
:10E0100070476FF002007047605D0020100900201B
:10E02000024BD3F868315B68184700BF605D002081
:10E03000024BD3F868319B68184700BF605D002031
:10E04000024BD3F86831DB68184700BF605D0020E1
:10E05000014BD868704700BF10090020044B93F8AB
:10E060006C3113B1034B186970476FF001007047B2
:10E07000605D00201009002010B54A4C94F86D3105
:10E08000C0B24BB1484BD4F870211B689B1A0A2BC5
:10E0900084BF002384F86D3194F86D31ABB9EE285C
:10E0A00009D1414A1268C4F87021012284F86D2117
:10E0B00084F8743110BDBB28FCD13B4B1B68C4F8FD
:10E0C0007031012384F86D31F2E7012B10D194F8FF
:10E0D000743123B984F8750184F86D31EAE7012BB6
:10E0E000E8D1002384F88C3184F88B010223F3E714
:10E0F000022BDFD194F88C31E218013382F87501DC
:10E1000094F88B21DBB29A4284F88C31D2D100236F
:10E1100084F86D3194F88D31012B31D1B4F9772128
:10E12000DFED226A224B9FED236A07EE102AB8EE3C
:10E13000C77AC7EE267AFDEEE77A17EE902A1A80A4
:10E14000B4F9792107EE102AB8EEC77AC7EE067A3D
:10E15000FDEEE77A17EE902A5A80B4F9752107EEA2
:10E16000102AB8EEC77AC7EE267AFDEEE77A17EEE8
:10E17000902A9A8020F0F4FF002384F88D3199E7EB
:10E18000022BF9D194F87531094A03F00301517259
:10E19000C3F381011172C3F301119B09D171937112
:10E1A000EAE700BF605D002014260020CDCCCC3F04
:10E1B000B8010120CDCCCCBF08B500684CF0F9FA0D
:10E1C000014BD867012008BD605D002008B50068DC
:10E1D0004CF0EFFA024BC3F89000012008BD00BFDD
:10E1E000605D002038B514460D46002943D0344BFD
:10E1F0009FED346AD3ED647AB3F9A821F8EEE77A9B
:10E20000C7EE866A07EE902AB3F9A42107EE102A1A
:10E21000F8EEE77AB8EEC77AB3F9A621A6EEA77AA8
:10E22000D3ED677AF8EEE77AE6EE877A93ED667AD1
:10E23000B8EEC70AA6EEA70A07EE902AB3F9A22104
:10E2400007EE102AF8EEE77AB3F9A021B8EEC77A04
:10E25000A6EEA77A07EE902AF8EEE77AE6EE877A3E
:10E2600093ED6B7AB8EEC77AC7EE066AA6EEA70AF8
:10E2700050F04AF928600CB3114BDFED126AD3ED70
:10E280006B7AB3F99421B3F99631F8EEE77A07EE99
:10E29000102A87EEA60A07EE903AF8EEE77AB8EE73
:10E2A000C77A60EE277AF6EE006AE7EE267A9FEDEF
:10E2B000060A27EE800A50F027F92060012038BDB9
:10E2C000605D00200000F04A0000C84210B50C4B11
:10E2D00003EBC00082B0D0F8BC4001916CB107EEF6
:10E2E000901A94ED047A94ED030AF8EEE77AA7EE1B
:10E2F000870A50F009F9A368186002B010BD00BF8A
:10E30000605D00202DE9F0410B4DDFF830802C6876
:10E310006B6901271C400CB9BDE8F081B4FA84F3A5
:10E32000C3F11F0307FA03F658F823000368984760
:10E3300024EA06046E61EEE7003C0140F43B002055
:10E340002DE9F04F9B4D002605F5D87C95F8F4118A
:10E35000A7B00A243246E646374605F5F67AA0E02D
:10E3600003EBC70305EB4300C3F30726B0F8F8013E
:10E3700001964607DFB25FFA80FE4FEA102B40F1AC
:10E38000C980480614D402F10209B9F18C0F41F09A
:10E39000400100F2008126A802F1010802444FF07A
:10E3A000040002F88C0C26AA90444A4608F88C1CFB
:10E3B000019802F10208B8F18C0F40F0020900F256
:10E3C000EA8026A8104400F88B9C4FF0050900F85D
:10E3D0008C9C02F10409B9F18C0F00F2DC8026AEAE
:10E3E000B0444FF0060608F88C6C02F106084FEABC
:10E3F0008E0EB8F18C0F00F8897C5FFA8EFE00F269
:10E40000CA8026AEB1444FF0070609F88C6C00F8BC
:10E4100087EC02F1080EBEF18C0F00F2BC8026AE34
:10E42000B0444FF00509019E08F88C9C00F8856CFB
:10E4300002F10A068C2E00F2AE800DF19809CE444E
:10E440004FF006080EF88C8C00F8837C02F10C0764
:10E450008C2F00F2A0804E444FF0070006F88C0C81
:10E460000B324846024402F88CBC3A465F09012050
:10E4700003F01F0600FA06F65CF82700013C20EACC
:10E4800006004CF8270000F089805E1CB6F5F07F8E
:10E4900080F0848073090CEB830ED6454FEA830726
:10E4A0007CD2DEF800004FF0FF3306F01F0603FABF
:10E4B00006F606EA000393FAA3F3B3FA83F3DBB29A
:10E4C000202B7FF44DAF0EF1040050451AD23A4B89
:10E4D000A3EB0E0727F003070EF1080E774401E0C7
:10E4E000B8420FD006460430336893FAA3F3B3FA68
:10E4F00083F3DBB2202BF3D0A6EB0C0613EBC603A1
:10E500007FF530AF85F8F4111046002A48D127B0C6
:10E51000BDE8F08F4E0603D401F03808F04515D061
:10E5200021F0780102F102080143B8F18C0FC9B261
:10E5300031D826A802F1010E02444FF0040002F87F
:10E540008C0C26AA964442460EF88C1C901C8C28F3
:10E5500021D826AE06EB020E019E0EF88B6C4FF012
:10E5600005060EF88C6C161D8C2E14D80DF198082B
:10E5700040444FF0060800F88C8C0EF8897C971DFB
:10E580008C2F08D826A806444FF0070006F88C0CFC
:10E59000053226A866E76FF0004267E785F8F411B8
:10E5A000D5F8EC0103A94CF08EFC012027B0BDE8A2
:10E5B000F08F00BF605D0020475F002037B58368A3
:10E5C0001C686379DB0724D5A57994F85C3205F0E3
:10E5D00001010D46FBB1E06B43681A68D36AC3F3CF
:10E5E0004E03536294F86D32012B07D094F86132D8
:10E5F00023B1B4F868320133A4F8683285F0010120
:10E600004AF02AFC0023A4F866324FF08073C4F865
:10E610005C3203B030BD94F85F320191012B04BF2E
:10E6200094F85D3284F85E322046FFF7F7FB94F8E9
:10E630005F32019953B9012384F85F3285EA0301FF
:10E64000E06B03B0BDE830404AF006BC002384F81C
:10E650005F32F5E710B5C14C04EB8003D3F81C31F1
:10E660000BB19B6819600F2822D8DFE810F0220058
:10E670003100480063007A009100AC00C300D5006F
:10E68000E400FB0016012D0144015F011000084663
:10E6900026F03AFA94F8CD3500F0070203F01F0394
:10E6A00043EA4213C0F3C70084F8CD3584F8CE05A1
:10E6B00010BD084626F028FA94F8BA3584F8B90552
:10E6C000C0F3022223F00703134384F8BA3510BDC8
:10E6D000084626F019FA94F8BA2594F8BB3500F0EC
:10E6E0001F0102F00702C0F3451023F03F0342EA86
:10E6F000C102184384F8BA2584F8BB0510BD08464A
:10E7000026F002FA94F8BB2594F8BD3500F0030119
:10E7100002F03F0242EA811223F00103C0F380219C
:10E720000B43C0F3870084F8BB2584F8BC0584F84C
:10E73000BD3510BD084626F0E7F994F8BD2594F8DC
:10E74000BE3500F07F0102F00102C0F3C31023F0D8
:10E750000F0342EA4102184384F8BD2584F8BE0540
:10E7600010BD084626F0D0F994F8BE2594F8BF35C0
:10E7700000F00F0102F00F02C0F3061023F07F0338
:10E7800042EA0112184384F8BE2584F8BF0510BD83
:10E79000084626F0B9F994F8BF2594F8C13500F081
:10E7A000010102F07F0242EAC11223F00303C0F329
:10E7B00041210B43C0F3470084F8BF2584F8C0050E
:10E7C00084F8C13510BD084626F09EF994F8C1259D
:10E7D00094F8C23500F03F0102F00302C0F3841048
:10E7E00023F01F0342EA8102184384F8C12584F80C
:10E7F000C20510BD084626F087F994F8C23500F02E
:10E80000070203F01F0343EA4213C0F3C70084F872
:10E81000C23584F8C30510BD084626F075F994F892
:10E82000C53584F8C405C0F3022223F0070313435F
:10E8300084F8C53510BD084626F066F994F8C5255C
:10E8400094F8C63500F01F0102F00702C0F345102E
:10E8500023F03F0342EAC102184384F8C52584F837
:10E86000C60510BD084626F04FF994F8C62594F861
:10E87000C83500F0030102F03F0242EA811223F0A2
:10E880000103C0F380210B43C0F3870084F8C62541
:10E8900084F8C70584F8C83510BD084626F034F959
:10E8A00094F8C82594F8C93500F07F0102F0010200
:10E8B000C0F3C31023F00F0342EA4102184384F867
:10E8C000C82584F8C90510BD084626F01DF994F83E
:10E8D000C92594F8CA3500F00F0102F00F02C0F309
:10E8E000061023F07F0342EA0112184384F8C92579
:10E8F00084F8CA0510BD084626F006F994F8CA2522
:10E9000094F8CC3500F0010102F07F0242EAC11216
:10E9100023F00303C0F341210B43C0F3470084F805
:10E92000CA2584F8CB0584F8CC3510BD084626F0FE
:10E93000EBF894F8CC2594F8CD3500F03F0102F0C7
:10E940000302C0F3841023F01F0342EA810218433C
:10E9500084F8CC2584F8CD0510BD00BF605D002093
:10E9600008B5202153F00EF8034620B11A78202A6A
:10E9700000F10100F8D0184608BD2DE9F0410D4620
:10E980001646044600274FF019082046FFF7E8FF17
:10E99000044690B1FEF712FE40F634024FF4617166
:10E9A000FDF77EFAA0F5617090FBF8F0302804D8EE
:10E9B0004FB9287033780133337017B12046BDE862
:10E9C000F0810127E1E76870F4E7244B1A6810B57D
:10E9D00013460446B3FBF1F0B0F5803F03D3012B9F
:10E9E000FAD95B08F6E781B22046FAF76DFD236895
:10E9F0001B68587990B1032140B2FAF777FC23687D
:10EA00001B685A7993F90530002B07DB02F01F01D0
:10EA100001228A405B09124941F8232023681B68C0
:10EA2000987990B1032140B2FAF760FC23681B6823
:10EA30009A7993F90630002B07DB02F01F010122BF
:10EA40008A405B09064941F8232063681A681388E5
:10EA50009BB243F00103138010BD00BFC00500202E
:10EA600000E100E08160C06BAFE7144951F820007D
:10EA700070B500B30C2202FB001292F9D535581C78
:10EA80001AD092F8DD05B0B1C818642590F8106668
:10EA900092F8DC45002014226B431D1901EB45055B
:10EAA000013AB5F81456344410FA85F0F5D1142320
:10EAB000B0FBF3F080B270BD0020FCE7605D002089
:10EAC00038B503200D461446FFF7CFFF07EE900A36
:10EAD0008DB19FED0B7AF8EE677AF0EE006A67EE83
:10EAE000877AB8EE047AA7EEA67ADFED067A67EEAB
:10EAF000277AC5ED007A0CB1034B236038BD00BF07
:10EB00006740533A00007A443313904310B5427A79
:10EB1000044632B10146406851F80A3B9847002349
:10EB2000637210BD10B4447A621C0444D2B24272C3
:10EB3000A172037A934202D85DF8044BE6E75DF8D0
:10EB4000044B7047EEE710B503681A79022A0446B1
:10EB500002D1987A4BF01EFE00232360237110BD72
:10EB600073B50279022A37D1032490F910308DF859
:10EB700003401B4C8DF80220142606FB0343194E5C
:10EB80005B6900250120B3428DF800508DF801002B
:10EB900024D0154DAB4203D0144883421CD11046FB
:10EBA00002AA11441A8811F8085C22F040021204EB
:10EBB000120C14211A8001FB00401A88016A22F00D
:10EBC000380231F825101204120C0A431A801A88F0
:10EBD00092B242F040021A8002B070BD2846DFE7D0
:10EBE000100900200030014000380040003C004087
:10EBF000C36910B5044623B90C211420FEF778F838
:10EC0000E061E06910BD10B504460068FFF7F0FF51
:10EC1000837853B183885BBAE381C3885BBA23826C
:10EC200003895BBA6382012010BD1846FCE710B56A
:10EC300000680C46FFF7DCFF83784BB14389222242
:10EC4000DBBA93FBF2F303F26D132380012010BDB6
:10EC50001846FCE738B500680D461446FFF7C8FFB4
:10EC6000D0F8013007EE103ACDB1D0F80530DFED25
:10EC7000176A9FED176A07EE903AF8EE677A77EE1B
:10EC8000E67A77EEA77AC7EE866AF7EE007A76EE36
:10EC9000E77ADFED106A67EEE67AC5ED007A9CB19F
:10ECA000DFED0D7ADFED0D6AB8EEC77A27EE277A31
:10ECB000C7EE267A9FED0A7A77EEC77A9FED097A3A
:10ECC00077EE877AC4ED007A38BD00BF9AC9CC448C
:10ECD0009AC94C460E76D7450000484300E0FF44F1
:10ECE00000004842339388430368DB6B13B5044646
:10ECF0002BB923685B6B3BB9FF23638202E0984723
:10ED00000028F6D102B010BD214601A8984700287E
:10ED1000F2D0BDF80630013B9BB2EEE710B50368B8
:10ED200004469B68984701236373FF23A37310BDB8
:10ED3000036810B504461B689847236820469B6803
:10ED40009847E37B0133E37310BD036810B50446B5
:10ED50005B689847236820469B689847E37B013BA4
:10ED6000E37310BDF0B585B0044618460D4616464F
:10ED700003934CF0A7F92268E67228440021A072A0
:10ED800000915769039B324629462046B84705B093
:10ED9000F0BD03689B6A184738B504468B6801606C
:10EDA0000D4698470B4BE360002323742B6B13B184
:10EDB000204698472074084B93F86C381BB1237C8D
:10EDC00023F001032374002363822046BDE838400A
:10EDD0008AE700BF0001FF00605D002003681B6838
:10EDE00003B11847704703685B6803B11847704761
:10EDF00003681B6A03B11847704703685B6A03B175
:10EE00001847704730B40468A46A14B1A44630BCF3
:10EE1000604730BC704730B40468E46A14B1A4465B
:10EE200030BC604730BC704703685B6C03B1184767
:10EE3000704703689B6C03B11847704703689B6F6A
:10EE400003B1184770470368D3F8803003B11847FF
:10EE500070470368D3F8843003B1184770470368DC
:10EE6000D3F8883003B11847704721B10B68D3F845
:10EE70008C3003B118470020704738B5094B052482
:10EE800004FB0030A0F1A00515F8010B013C4BF08C
:10EE900000FC14F0FF04F7D12046BDE838404BF0E9
:10EEA000F8BB00BF9C1E060810B5441E14F8010FE5
:10EEB00000B910BDFFF7E1FFF8E7FFF723BAFFF74E
:10EEC00021BAFFF71FBAFFF71DBAFFF71BBAFFF70A
:10EED00019BA30B1006800F13F4000F57E00800AA9
:10EEE00070474FF0FF30704728B18088B0FA80F04B
:10EEF000C0F11F0070474FF0FF307047F7B506466E
:10EF0000FFF7E7FF194B18440C4690F8A30215468B
:10EF10004AF006FA3046FFF7E7FF3768C0F3CC0344
:10EF200007EB830300F00702196A92000F2090405C
:10EF300021EA00011962196A95400D431D62B388E8
:10EF4000009304F003038DF80430C4F381038DF8BB
:10EF500005306946C4F30013384664098DF806305D
:10EF60008DF80740FAF742FE03B0F0BD9C1E06087C
:10EF70002DE9F04F87B099469DF84430BDF840B078
:10EF80000293CDE900019046FDF7ECFE064600280D
:10EF900000F098804E4F97F86D58052D00F28D8047
:10EFA0005C2303FB05730022C3F8702883F87428E0
:10EFB000009B1A79130905EB450A6C1C013BC5EB54
:10EFC000CA01E4B207F5076A032B87F86D4802F01F
:10EFD0000F020AEB810A3ED83E49039331F8130031
:10EFE00040FA02F1CB0736D5012101FA02F2013ACB
:10EFF00010404CF0C1FE3849039B384A0B444FF097
:10F00000020C93F8AC32184400EB400002EB800392
:10F01000019A9A71029A1C7283F807C000FA0CF4E4
:10F02000002A43D118460093FFF753FF084490F895
:10F03000A3024AF075F9009B284A998804914FF081
:10F0400001111059059104A9FAF7D0FD234A009B3C
:10F05000A2589B8853835C2303FB057542464946AF
:10F060003046C5F87068FAF72FFAD5F87008594697
:10F07000FAF782FAD5F8700843681A68B2F8443093
:10F080006FEA43436FEA53439BB2A2F844301388BC
:10F090009BB243F001031380FAF77EFB0023C5F80F
:10F0A00078080360504607B0BDE8F08F009A6146CB
:10F0B000127A1846FFF722FFCDE7094A0021042003
:10F0C000FDF750FD4FF0000A504607B0BDE8F08F45
:10F0D000605D0020F01B06089C1E060868390020B1
:10F0E000B8AA060830B1036882881B691A4214BFA7
:10F0F00001200020704728B10368828809B11A8373
:10F1000070475A83704710B1036882881A8370472A
:10F1100010B1036882885A8370478379806BDB075C
:10F1200048BF81F0010101B1EDE7F1E737B50C46C9
:10F130000546E8B1FFF7CDFE0E4B184490F8A30248
:10F140004AF0EEF8AB88009304F003038DF8043026
:10F15000C4F381038DF805302868C4F300136946B1
:10F16000C4F341148DF806308DF80740FAF73EFDE0
:10F1700003B030BD9C1E060800B1BFE6704710B555
:10F18000837913F0010F03F020020446C36B12D001
:10F190005B68002A1A7A14BF02214221606BFFF7D4
:10F1A000EBFF0121E06B84F86012A4F85C12BDE86B
:10F1B0001040FAF707BB5B68002A18BF02211A7AD1
:10F1C00008BF2221EAE7036C806B1BB15B68012159
:10F1D0001A7AD1E70121A9E770B583681C686379C1
:10F1E0009A0731D594F86152D5B194F962329BB146
:10F1F000B4F864124B08A4F86432204601F001010F
:10F20000FFF78BFF94F86232A279013B5BB25006A4
:10F2100084F8623218D5BBB9002384F8613213E058
:10F22000A36A626A94F860129A4226D161B9A379FE
:10F230001B0709D5236CA06BDBB15B681A7AFFF75B
:10F240009BFF2046FFF79BFF6379D90740F1818040
:10F2500094F85C32002B7CD194F85D320133DBB240
:10F26000092B84F85D3235D12046BDE87040FEF7A9
:10F27000D5BD1946FFF75AFFE3E75A1CA069A26201
:10F28000C35C26695B0043F40073A4F864320A236C
:10F29000B24234BF1046284684F862320123A0628D
:10F2A00084F8613291B1A3791E070FD5E06B29462E
:10F2B000FAF788FAE36B606B5B6829461A7AFFF706
:10F2C0005BFF84F860522046FFF77DFFA3795D065F
:10F2D0008BD4B9E70A2B3CD194F85F322BB9B4F840
:10F2E000663243F00103A4F86632B4F86602820580
:10F2F00001D4C3071AD4B4F86A320133A4F86A32CD
:10F3000094F85F5201239D42A4F85C3221D1A17987
:10F31000E06B002384F85F3201F0010149F09CFDAD
:10F32000E06B2946BDE87040FAF74CBAE36AC0F3D7
:10F33000470013B1216B9847E2E7E3696269D05453
:10F34000E369E2680133B3FBF2F102FB1133E361DD
:10F35000D6E770BD10B50409013C032C00F00F0284
:10F3600019D80E4B33F8141041FA02F313F00100D0
:10F3700010D0012303FA02F2013A02EA01004CF034
:10F38000FBFC074A14440C2294F8AC321844054B99
:10F3900002FB003010BD0020FCE700BFF01B060898
:10F3A0009C1E0608683900202DE9F04F3C220446D7
:10F3B0000021B74893B052F0CEFAB649621EE01C65
:10F3C0000C4612F8013F5D1E032D88BF00239042BA
:10F3D00041F8043BF5D10120FEF7D2FA38B12023E1
:10F3E00084F8E03594F81036013384F810360220A2
:10F3F000FEF7C6FA38B1212384F8EC3594F81036BC
:10F40000013384F810360320FEF7BAFA38B110231E
:10F4100084F8F83594F81036013384F81036042057
:10F42000FEF7AEFA38B1112384F8043694F810369A
:10F43000013384F81036984E954CDFF86C824FF00B
:10F440000F094FF0000A06F52C77207B38B394F9AA
:10F450000D50FFF77FFF28B107238371002380F849
:10F46000079003721321FFF761FE227B002317F838
:10F470003310914240F0DC8006EBC303D3F8B43282
:10F480002361182303FB0585AB6F23755A1C0723E3
:10F49000A3750123AA67637585F874309A4409F14E
:10F4A00001095FFA89F9B9F1130F04F10C04CCD109
:10F4B000BAF1000F00F0B980784CDFF8F0914FF00E
:10F4C0000008237C002B00F0A6806079704D49F085
:10F4D00027FF207949F024FFA068FAF7FFFA0023FC
:10F4E000CDE90E33CDE91033069308932368A06865
:10F4F000CDF814904C330493E368039363691422AA
:10F50000534307934FF480624FF40063CDE909231E
:10F510004FF400514FF48073CDE90B134FF40033D7
:10F5200003A90D9349F020FEA268136843F001037C
:10F5300013605B4A536823F4733323F4477323F057
:10F54000030343F440335360226863695168012B1D
:10F5500021F04071D4BF0020012021F4807141EAE4
:10F560000021516090684F49014041F002019160D3
:10F57000D16A013B21F47001DBB241EA0353D3624B
:10F580004FFA88F101239C4601914FF01F0E697DCF
:10F5900051B395F90D100198814225D1297CAE7D9A
:10F5A0005F1C0929FFB249D9A1F10A00D2F80CA0C9
:10F5B00000EB40004FF0070B0BFA00FB2AEA0B0AA6
:10F5C00006FA00F040EA0A00D060062B44D8013B5E
:10F5D000506B03EB83030EFA03F620EA060001FAF0
:10F5E00003F3034353633B460CF1010CBCF1050FDD
:10F5F00005F10C05CBD1936843F4007393609368D5
:10F6000043F480739360936843F0010393609368BD
:10F6100043F08043936008F10108B8F1030F04F14F
:10F62000180409F1C8097FF44CAF13B0BDE8F08F9E
:10F630000133102B7FF41BAF002321E7106901EB8E
:10F64000410A4FF0070B0BFA0AFB20EA0B0006FAFF
:10F650000AF630431061B8E70C2B0CD8073B106B4F
:10F6600003EB83030EFA03F620EA060001FA03F324
:10F6700003431363B7E70D3BD06A03EB83030EFA32
:10F6800003F620EA060001FA03F30343D362AAE774
:10F6900034630020605D00209C1E06087409002071
:10F6A00000230140FDF7FFC0100900207463002013
:10F6B0002DE9F74FAE4D0093AE4B9D4221D26C79B0
:10F6C0008C4240F06D812C79844202D0002840F0B9
:10F6D0006781EC79944240F063812C68DCB11C2294
:10F6E0000021201D52F037F925602B79237195F800
:10F6F0000690C4F808902A7AE260012B03D0022B0E
:10F700000DD0002407E0E87AFFF724FE6B7A23741B
:10F71000AB7AA0616374204603B0BDE8F08FE87A4D
:10F72000FFF718FE95F90960A0612674A87AFFF723
:10F7300011FE6061002800F02F818F4D4FF01408FA
:10F7400008FB0658D8F81430002B00F0258198F8F3
:10F750002630002B40F0C58098F81C0049F0E0FDF1
:10F7600098F81C3003F01F025B090121023B01FAEB
:10F7700002F2032B08D8DFE803F0726C02667F49BF
:10F780000B6923EA02020A61142303FB0653587E25
:10F79000FFF7E0FD731CDFB2834618B140F60D326F
:10F7A000C2800772142202FB0652D07EFFF7D2FD00
:10F7B000824618B140F60D52C2800772142202FB35
:10F7C0000652907EFFF7C6FD804618B140F60D4206
:10F7D000C2800772142303FB065319F004095A7FF1
:10F7E000019242D04A215846FFF7C6FC019A2A21CD
:10F7F0005046FFF7C1FC019A40460A21FFF7BCFCC6
:10F80000142303FB0653019A93F81880B8F1000FF4
:10F8100007D040460192FFF79DFD019A0921FFF7AD
:10F82000ABFC142303FB06535A69554B9A4223D170
:10F8300003F58433596A41F480515962596A21F4BD
:10F840008051596225E04D494B6923EA02024A6121
:10F850009AE74A490B6A23EA02020A6294E7474997
:10F860004B6A23EA02024A628EE70A215846FFF7F2
:10F8700083FC019A0A21BBE7424B9A4240D103F52F
:10F880000033196A41F480411962196A21F48041F8
:10F890001962B9F1000F67D00021084613880143AF
:10F8A00003F44153194341F445711180938B23F4C0
:10F8B00000631B041B0C93830723138213889BB2E2
:10F8C00043F040031380B8F1000F04D04046FFF727
:10F8D00041FDFFF718FC142303FB0655012385F8AF
:10F8E0002630606928B1009B83710E23C371002309
:10F8F00003720921FFF71AFC6069FFF704FC0AE7AD
:10F90000214B9A4209D103F5FE33196A41F40041B3
:10F910001962196A21F40041BAE71C4B9A4209D1D5
:10F9200003F58233596A41F400515962596A21F44E
:10F93000005186E7164B9A4209D103F56843596A8C
:10F9400041F480115962596A21F4801179E7114B11
:10F950009A429ED103F56443596A41F400115962F9
:10F96000596A21F400116CE70121022096E700BFDB
:10F97000A001000820030008100900200038024000
:10F980000030014000380040003C0040003401409D
:10F9900000500140005401402046FFF7D4F8B0E683
:10F9A0000C358AE6064B53F820303BB19A881B6829
:10F9B00059690A4201D05A8370471A83704700BFC1
:10F9C000F81B0608034B81F0010153F82000FFF7F4
:10F9D00092BB00BFF81B06082DE9F84F6A4FD7F815
:10F9E000980A037C03F0FF0C002B40F0CB8097F8C3
:10F9F0009E2A97F89F3A97F8A09AA7F89CCA07F60C
:10FA0000A22EE2463C259EF802109EF80360C1F14A
:10FA1000FF0189B2002900F0B180C1F1FF017143FB
:10FA2000BEF80040B4FBF5FB0912BBF1050F22D86C
:10FA3000DFE80BF0030E63748593731A6343B3FB23
:10FA4000F5F353FA81F35FFA81F9DBB2324610E045
:10FA5000B4FBF5F205FB124292B2C2F13C02741AF9
:10FA60006243B2FBF5F252FA81F25FFA81F9D2B247
:10FA700033464FF0010A160246EA034646EA0906F3
:10FA800000214FF001080CEB0104C1F1170B08FA3B
:10FA90000BFBA4B21BEA060F07EB8404414414BF1E
:10FAA0004FF0020BC3461829C4F824BBE9D10CF16E
:10FAB000180C1FFA8CFCBCF5407F0EF1040EA2D18D
:10FAC0003249A1F8D4C6BAF1000F05D087F89E2AB2
:10FAD00087F89F3A87F8A09A2023A7F89C3A91F8D4
:10FAE000D636002B4ED040F22A31F9F783FED7F8F4
:10FAF000980ABDE8F84FF9F7AFBEB4FBF5F305FB84
:10FB00001344A6EB0109A4B2CAB204FB09F9B9FB7C
:10FB1000F5F959FA81F15FFA81F9A9E7B4FBF5F338
:10FB200005FB13439BB2C3F13C03741A6343B3FB5D
:10FB3000F5F353FA81F3CAB2DBB2B14699E7B4FBED
:10FB4000F5F905FB1944721AA4B26243B2FBF5F24F
:10FB500052FA81F2CBB2D2B2EFE7B4FBF5F205FB79
:10FB6000124292B2C2F13C02741A6243B2FBF5F245
:10FB700052FA81F2CBB25FFA82F967E7B1463346B7
:10FB8000324676E7BDE8F88F605D0020586E0020B1
:10FB9000F8B500212A20F9F77EFC054650B3FDF7A1
:10FBA000E1F81B4F0446C7F8980A18B32A20FFF75C
:10FBB000D1FB184EC6F8D80620B140F21723C380F7
:10FBC000002303722A7A4A21FFF7D6FA124A032148
:10FBD0002046F9F779FCD7F8980A0021F9F7CCFC10
:10FBE0000E49D7F8980A40F22A3249F0E7FA10B9DC
:10FBF00086F8D606F8BD094840F6A842002151F023
:10FC0000AAFE012386F8D636BDE8F840E4E600BF38
:10FC1000605D0020586E0020009F24008468002052
:10FC2000084B93F8F1214AB193F8F33113F0400FE8
:10FC300014BF4FF4F0704FF4C37070474FF4F0707E
:10FC4000704700BF605D0020054B93F8F10130B1B3
:10FC500093F8F33113F0400F0CBF0D2010207047C4
:10FC6000605D0020104A70B5002302F5707E4FF4ED
:10FC70000056A2F14605012432F8020F4FEA531C48
:10FC8000B0F5005F1CBF55F82C00168003F01F0173
:10FC900004FA01F11CBF014345F82C10724503F131
:10FCA0000103E9D170BD00BF565F00204FF01E0C6C
:10FCB00043EA0223FF2A0CFB01011BB288BF43F079
:10FCC0000403B1F5F07F07DA0C4A02EB41009BB266
:10FCD000B0F8F8C19C4500D170474FEA511C02F5BD
:10FCE000D872A0F8F83101F01F0152F82C30012031
:10FCF00000FA01F10B4342F82C307047605D0020A0
:10FD00004FF01E0C0CFB0101B1F5F07F01DB002070
:10FD100070470B4800EB4101B1F8F811080AC9B26D
:10FD200010801970490709D5118841F4807111803C
:10FD30001A7822F0040201201A70704701207047DF
:10FD4000605D00202DE9F0471E2404FB01011478BA
:10FD50008CB31D282FDC194E0FFA83FE06EB410CE5
:10FD6000C1F10105483E012701E01D2B23DCB1F55F
:10FD7000F07F4EEA042405EB010313D2BCF800A087
:10FD80004FEA5119A24518BFACF8004001F01F0816
:10FD900018BF56F8294007FA08F81CBF44EA0804BF
:10FDA00046F8294012F8014FDBB20CF1020C034473
:10FDB0000131002CD9D1BDE8F08700BF585F002089
:10FDC0002DE9F04F012885B014BF292412240546DF
:10FDD0008B462046002199460292F9F75CFB9DF87C
:10FDE00038709DF83C8006462046FFF7B3FA07F0CE
:10FDF0000303032B08BF48F0080818F00803044663
:10FE0000019321D026B90026304605B0BDE8F08F19
:10FE1000B3795907F7D43046FCF7A4FF7A4B4FF477
:10FE20001C7202FB0533C3F818070028EBD0C3F897
:10FE30001447C3F810476B1CDBB2002C3DD040F2D6
:10FE40000672E280237238E017F001021BD00392A1
:10FE5000002ED8D0B3795A07D5D43046FCF782FFAC
:10FE6000694B4FF41C7101FB0533C3F818070028D8
:10FE7000C9D0C3F810476B1C039ADBB21CB140F227
:10FE80000661E1802372BB0717D55F4B4FF41C71ED
:10FE900001FB053ACAF81447002A40F09580002E6D
:10FEA000B1D03046FCF75EFFCAF818070028AAD088
:10FEB0006B1CDBB2002C40F0928053494FF41C7352
:10FEC0006B43CC1801F2DC625049C4F8DC1602998D
:10FED000C4F80C1703F15C011144C4F8F01603F5E3
:10FEE000AE714FF0000A11444FF4807CD4F818072B
:10FEF00084F8E17684F8E286C4F808B7C4F8E8C666
:10FF0000C4F8F416C4F8ECC64946C4F8E496C4F83C
:10FF1000FCA6C4F8F8A6C4F804A7C4F800A784F89F
:10FF20004859C4F844A9A4F83CA9D6180293FEF78E
:10FF30004CFD08F00101D4F81807DFF8DCB048F0F8
:10FF40008BFF029B324A03F1440817F0020F9044E2
:10FF5000304F47D0D4F81C07002843D0D4F81837C6
:10FF6000596843680968D3F800C08C453AD001212C
:10FF700084F849194946FEF728FDD4F81807C4F853
:10FF800020674146C4F82477C4F828A7C4F82C6732
:10FF9000C4F830A7C4F834B7F9F750FA029B1C4AEA
:10FFA000D4F81C0703F150011144F9F747FA019BFB
:10FFB00033B93046FFF707F901213046FFF7ADF8B6
:10FFC0003046FFF7DCF81FE73046FCF7CBFEDAF8E7
:10FFD0001837CAF81C07002B7FF46AAF13E740F20A
:10FFE00006522EE7084B4FF41C7000FB053500232A
:10FFF000D5F8180785F84939C5F82067C5F824777A
:020000040801F1
:10000000C5F828B74146D0E7586E0020CC21060835
:1000100034750020BDE50008D9F10008002ABCBFF6
:1000200080185242002BBCBFC9185B420028BCBFDD
:10003000121A0020F0B58518CC180029A5F11D056D
:10004000BCBF234600210F3C002DC8BF521B002C13
:10005000C8BF1B1B0A4E02440B443C274FF0200C28
:1000600090420CDC06EB40050C4604E007FB04FE66
:10007000013425F80EC09C42F8DD0130F0E7F0BDF8
:10008000585F0020154B07B51A6C42F080521A6475
:10009000134A01211162134AFF215162CA215162A0
:1000A000532151625B6FDB000AD5002301930E4B95
:1000B0000193019B0193019B1A680C4B9A420AD051
:1000C00000210120FAF7DCFD0849002003B05DF8AB
:1000D00004EBFAF7D5BD03B05DF804FB003802402D
:1000E00000000E42002800405028004076614E6912
:1000F000024B002283F8AC20704700BF100900209B
:10010000024B012283F8AC20704700BF1009002089
:10011000034A044B92F8BC2B03EB42035878704718
:10012000586E0020091C0608104A114B92F8BC2B8F
:1001300003EB42035B7803B970470E4B1978002933
:10014000FAD010B50C4C002304EBC00C4FF0010E9C
:1001500054F833202AB112791AB1984208BF8CF8AA
:1001600006E001339942F3D110BD00BF586E002064
:10017000091C0608E41101201C5E002010B5154C76
:10018000D4F8D02BD4F8D43BD4F8C81B82B002FBEF
:1001900003F38B428DF807001AD0D4F8C43BD4F88F
:1001A000CC0B0DF10701184451F09CF9D4F8C43B75
:1001B000D4F8D02BD4F8C81B1344D4F8D42BB3FBF9
:1001C000F1F0013201FB1033C4F8C43BC4F8D42B66
:1001D00002B010BD586E00200B4B10B4002203F685
:1001E000D83408200121C3F8CC4BC3F8C80B5DF804
:1001F000044BC3F8D01BC3F8C02BC3F8C42BC3F8FF
:10020000D42BC3F8E42B7047586E0020174B184AC4
:100210009B7982F8BC3B032B23D9191F02291CD8D8
:10022000052B10B41FD0062B14BF4FF47A604FF487
:100230007A501049104BB3FBF0F3002401F1100C7D
:100240004C60C2F8F03B00200C4B5DF8044BC2F848
:10025000E83B00214CE902017047094BC2F8E83B3A
:100260007047084BFAE74FF4FA50E2E7203E0020CF
:10027000586E0020487A002040420F004DDF0008F1
:1002800049DF0008CDE200080F4B93F8BC3B062B7A
:1002900017D8DFE803F00416070A0D1013004FF417
:1002A000C87070474FF4FA607047084B98887047E1
:1002B0004FF47A6070474FF4FA5070474FF47A5019
:1002C00070474FF47A707047586E0020203E00202F
:1002D0002DE9F041854B93F8BC3B82B00D46062BCF
:1002E00000F2FC80DFE803F02EC0669604040400F0
:1002F000052B00F0E7807E497E4C062B08BF214687
:100300004FF00008CDE9008214230A460421FEF7CD
:100310002FFE0646002800F0DF800746122257F81D
:10032000140B394648F04AFF0446002840F0CC80C0
:100330000124714901EBC501C1F8BC60204602B03F
:10034000BDE8F08101926D4A6D4B1468A3FB042156
:100350004FF6FF7202EBD112120CB4FBF2F4002242
:10036000A3FB04130092C3F3CF1322460421FEF72C
:10037000FFFD98B107EE904A9FED627ADFED626A69
:10038000F8EE677A012367EE877A037127EE877AA2
:10039000E7EE667A80ED047AC0ED037A5649041ED2
:1003A00001EBC50118BF0124C1F8BC00204602B012
:1003B000BDE8F0810192514A544B1468A3FB04211B
:1003C0004FF6FF7202EBD112120CB4FBF2F40022D2
:1003D000A3FB04130092C3F3CF1322460421FEF7BC
:1003E000C7FD0028DAD007EE904ADFED496A9FED9D
:1003F000467A9FED486AF8EE677A012367EEA66AAF
:10040000037127EE667AC0ED046AA7EE867A80ED66
:10041000037AC3E70192404B384A9B881268B2FBCB
:10042000F3F101F57F41FF31090CB2FBF1F200213C
:100430000091B2FBF3F40421A3B2FEF799FD00286A
:10044000ACD007EE904ADFED2F6A9FED2F7AF8EEE1
:10045000677A012367EEA67A037127EE677AC0ED0B
:10046000047A80ED037A99E70192244A274B1468B5
:10047000A3FB04214FF6FF7202EB9112120CB4FBA6
:10048000F2F40022A3FB04130092C3F38F1322465D
:100490000421FEF76DFD002880D007EE904ADFEDC5
:1004A0001F6A9FED187AF8EE677A012367EEA67A45
:1004B000DFED156A037127EE877AE7EE667A80ED45
:1004C000047A69E716491BE741463846482251F04D
:1004D00042FA012333712CE704462AE7064901EB6F
:1004E000C50100231C46C1F8BC3027E7586E002028
:1004F000C0C62D00001BB700605D0020C0050020B5
:100500001F85EB516F12833A00007A44D34D62107D
:1005100077CCAB32ACC5A736203E00206F12033932
:10052000808D5B00044B03EBC000D0F8BC0010B121
:1005300003685B6818797047605D002008B50A4B56
:100540001B7A012B06D0022B09D0084B084AC3F8AE
:10055000002C08BD49F0C0FD044B064AF7E749F0FE
:10056000BBFD024B044AF2E7383E0020586E0020E3
:1005700069DF0008ADCF020855E600082DE9F04F0D
:1005800087B09B469DF84030019381468A4690464D
:10059000FCF7E8FB0446002800F09D80504D95F8DC
:1005A0006D78052F00F292805C2303FB0753002235
:1005B000C3F8702883F8742899F8042007EB4701E2
:1005C00013097E1CC7EBC101013B05F50760F6B2BC
:1005D00000EB8101032B85F86D6802F00F02029198
:1005E0003BD84049039331F8130040FA02F1CB079E
:1005F00033D5012101FA02F2013A10404BF0BCFB65
:100600003949039B394A0B4440F2052C93F8AC322C
:10061000184400EB400002EB8003019A1E72A3F81D
:1006200006C08600002A4AD118460193FEF751FC05
:10063000084490F8A30248F073FE019B2B4A998866
:1006400004914FF001119059059104A9F9F7CEFAE0
:10065000264A019BB2589B8853835C2303FB0757B0
:10066000234AC7F87048B2FBF8F1204689B2F8F780
:100670002BFFD7F870085946F8F77EFFD7F87008B7
:1006800043681A68B2F844306FEA43436FEA534351
:100690009BB2A2F8443013889BB243F0010313804D
:1006A000F9F77AF80023C7F8780805EB8A050360A4
:1006B000029BC5F81C31012007B0BDE8F08F99F806
:1006C000082018460221FEF719FCC6E7094A002156
:1006D0000420FCF747FA002007B0BDE8F08F00BF08
:1006E000605D0020F01B06089C1E0608683900208B
:1006F00040420F00B8AA0608034BD3F8002C12B1F1
:100700000F2800D810477047586E002050B10138AC
:10071000002330F0FF019AB203F1010303D140EA54
:10072000022080B270474008F3E703681B6818474F
:100730002DE9F041134E144B07460C46D6F8040C35
:100740004FF00008AA21154683F86D81FFF7EDFFF1
:10075000D6F8040C4146FFF7E8FFD6F8040C3946FA
:10076000FFF7E3FF2946D6F8040CFFF7DEFF254428
:1007700014F8011BD6F8040CFFF7D7FFAC42F7D1F1
:10078000BDE8F081586E0020605D002007B50122B1
:100790008DF8041001A9FFF7CBFF03B05DF804FB4F
:1007A00070B50E4C0E4B002206460D46D4F8040CD4
:1007B00083F86D21AA21FFF7B8FFD4F8040C0121BA
:1007C000FFF7B3FFD4F8040C3146FFF7AEFFD4F8BF
:1007D000040C2946BDE87040A7E700BF586E002012
:1007E000605D002038B505460C4614F8011B01B9C0
:1007F00038BD2846FFF799FFF7E703685B6818479D
:1008000003689B6818470368DB6970B506460C46A9
:10081000154683B1BDE8704018473046FFF7F0FF3A
:100820000028FAD014F8011B3046FFF77EFF2B1B7F
:10083000002BF2DC70BD0D44F9E7E4E70368DB68E8
:10084000184703681B69184703685B691847036802
:100850009B6A03B1184770470368DB6A03B1184706
:100860007047074B9B7A01460BB1FDF789BB054BDF
:100870001868054B1B780BB981F00101FEF73BBCF2
:10088000143F00200C3F0020103F002072B60022D1
:100890004FF0FF31930003F1604303F561430132F0
:1008A000082AC3F88010C3F88011F3D1BFF34F8F2B
:1008B0000549064BCA6802F4E0621343CB60BFF3FC
:1008C0004F8F00BFFDE700BF00ED00E00400FA0518
:1008D000012108B50846FAF7D3F9FFF7D7FF07B5A6
:1008E0000B4B002101910193019B04330193019B68
:1008F0001868012808D1FAF7C3F9064B1A6882F381
:1009000008885B689847FEE703B05DF804FB00BF0A
:10091000502800400000FF1FEFF31183102282F3E4
:10092000128809490A6801320A604FF0E02207493B
:100930009069C1F8080C0020C1F80C0C1269DBB2F8
:1009400083F31188704700BF14260020586E0020E2
:10095000064A074B51681B6858434FF47A73B0FB43
:10096000F3F053685B1A8342FBD97047001000E034
:100970000C2E002010B504464FF4FA70FFF7E8FF84
:100980006069BDE81040FEF7BEBB73B5104B15465D
:1009900090F910200446142000FB02335E69A3681E
:1009A0009A0704D46069019149F0ECFE0199304640
:1009B0004AF0AEFA294630464AF0AAFAA3689B07E5
:1009C00002D42046FFF7D6FF012002B070BD00BF61
:1009D000100900207FB50379012B0D460AD0022BA8
:1009E00019D18368DB0758BF01F07F0104B0BDE86F
:1009F0007040CAE781688DF80F2001F001010DF108
:100A00000F0200920191417C90F910002A46F9F7FB
:100A1000DBFF04B070BD0020FBE700682E22F4214C
:100A2000D8E7044B00681A8E9201343202F0FC02BF
:100A3000F421CFE7605D002008B53122F421006881
:100A4000FFF7C8FF012008BD006801225821C1E757
:100A5000006801224821BDE7006802220821B9E7A9
:100A6000006801220821B5E710B5044600222121C3
:100A70000068FFF7AFFF2068FC222021FFF7AAFFE4
:100A8000206840222421FFF7A5FF20680C222321A3
:100A9000FFF7A0FF206800222221FFF79BFF012023
:100AA00010BD10B5012204460B210068FFF792FF2C
:100AB00020B120681D220921FFF78CFF00F0010002
:100AC00010BD044B0246D3F8100C08B1802181E719
:100AD000704700BF586E002010B5B020FFF7F1FF3F
:100AE0004020FFF7EEFF0020FFF7EBFF1020FFF79D
:100AF000E8FF4FF48064013C0020A4B249F0C9FD36
:100B0000002CF8D110BD503910B50446C8B2FFF71B
:100B1000D8FF04EB4400400004EB440400F00E0056
:100B2000FFF7CFFFC4F3C3001030BDE81040C8E7A3
:100B300008B55038C0B2FFF7C4FF0020FFF7C1FF6F
:100B4000BDE808401020BCE738B50022222332213E
:100B50000120FEF7ADFD3D4BC3F8100C10B9002489
:100B6000204638BDAE20FFF7ACFF04460028F6D083
:100B7000D420FFF7A6FF8020FFF7A3FFA820FFF7F0
:100B8000A0FF3F20FFF79DFFD320FFF79AFF002033
:100B9000FFF797FF4020FFF794FF8D20FFF791FFAD
:100BA0001420FFF78EFFA120FFF78BFFC820FFF76F
:100BB00088FFDA20FFF785FF1220FFF782FF8120F0
:100BC000FFF77FFFCF20FFF77CFFD920FFF779FFEA
:100BD000F120FFF776FFDB20FFF773FF4020FFF7E0
:100BE00070FFA420FFF76DFFA620FFF76AFFAF207C
:100BF000FFF767FFA620FFF764FFAE20FFF761FF56
:100C00002020FFF75EFF0020FFF75BFFB020FFF71B
:100C100058FF4020FFF755FF0020FFF752FF10203C
:100C2000FFF74FFF4FF48065013D0020ADB249F062
:100C300030FD002DF8D18120FFF743FFC820FFF7DA
:100C400040FFAF20FFF73DFF8AE700BF586E00204E
:100C500008B5FFF7BFFE014B187008BD1009002052
:100C6000F7B515461E4690F91020104B0446142087
:100C700000FB02335F69A3689A0704D4606901919D
:100C800049F080FD019938464AF042F933462A4638
:100C9000002138464AF0ECF8A3689B0702D42046AE
:100CA000FFF768FE012003B0F0BD00BF100900206F
:100CB000F7B50779012F16460AD0022F15D184689F
:100CC000E40758BF41F0800103B0BDE8F040C7E73A
:100CD000826802F00102CDE900620A46417C90F987
:100CE0001000F9F771FE03B0F0BD0020FBE707B577
:100CF000130A8DF804308DF80520022301AAFFF7AE
:100D0000D7FF024B187003B05DF804FB10090020F8
:100D100010B50A4C002384F8143C84F8151C84F8A0
:100D2000162C032304F61442FF21FFF7C1FF00280D
:100D30000CBF6FF00C00002010BD00BF586E0020EB
:100D400010B50B4C002384F8143C130A84F8151CCE
:100D500084F8163C84F8172C042304F61442FF216F
:100D6000FFF7A6FF00280CBF6FF00C00002010BD9D
:100D7000586E0020024A00680023512198E700BF06
:100D80006C7B0020F7B515461E4690F91020104BDD
:100D90000446142000FB02335F69A3689A0704D459
:100DA0006069019149F0EEFC019938464AF0B0F8CB
:100DB00033460022294638464AF05AF8A3689B0772
:100DC00002D42046FFF7D6FD012003B0F0BD00BFDE
:100DD00010090020F7B50779012F16460AD0022F17
:100DE00015D18468E40758BF41F0800103B0BDE825
:100DF000F040C7E7826802F00102CDE900620A46CE
:100E0000417C90F91000F9F705FE03B0F0BD002019
:100E1000FBE770B5066805463046FDF7E9FE0E2390
:100E20000446021D3B213046FFF7D4FFA07040B1BD
:100E3000A3895BBA2B84E3895BBA6B84238A5BBA90
:100E4000AB8470BD07B50223006801AAF621FFF745
:100E5000C1FF20B1BDF80430024A5BBA138203B06F
:100E60005DF804FB605D002007B50323006801AA5C
:100E7000F621FFF7AFFF80B19DF805309DF8042003
:100E800007491B0243EA02439DF806201343B1F9C8
:100E90003020C2F10802D3404B6303B05DF804FB7D
:100EA000605D002037B50623F7210068154C6A46BF
:100EB000FFF790FF1449E8B19DF801209DF800303C
:100EC0009DF80350120142EA03329DF8023042EAD3
:100ED00013129DF804308A651B0143EA05339DF81F
:100EE0000550C4F8142D43EA15138B63C4F8183D5C
:100EF00003B030BDD4F8143D8B65D4F8183D8B6336
:100F0000F6E700BF586E0020605D002007B50323A0
:100F1000006801AA1946FFF75DFFA0B19DF80430F3
:100F20009DF805109DF904201B0443EA01239DF858
:100F30000610002AB4BF4FF07F4200220B43134338
:100F4000024AC2F8AC3103B05DF804FB605D0020DA
:100F500007B50323006801AA0021FFF73BFFA0B1FA
:100F60009DF804309DF805109DF904201B0443EA08
:100F700001239DF80610002AB4BF4FF07F420022E3
:100F80000B431343024AC2F8903103B05DF804FBEF
:100F9000605D002013B5044600680379022B0CBF86
:100FA0004321032106236A46FFF714FF18B9E086A0
:100FB000A06302B010BDBDF800305BBAE386BDF897
:100FC00002305BBA6387BDF804305BBA2387F0E771
:100FD00013B5062304466A4600681121FFF7FAFE9E
:100FE00018B9E086A06302B010BDBDF9003007EE6D
:100FF000103AB8EEC77AF7EE086A27EE267ABDEE09
:10100000C77A17EE103AE386BDF9023007EE103AC0
:10101000B8EEC77A27EE267ABDEEC77A17EE103AF9
:101020002387BDF9043007EE903AF8EEE77A67EED1
:10103000A67AFDEEE77A17EE903A6387D3E713B509
:101040000023C38683630446062300686A4603219F
:10105000FFF7C0FE78B1BDF8003003EB4303E38631
:10106000BDF902305B4203EB43032387BDF8043034
:1010700003EB4303638702B010BD07B5012301AA48
:10108000FF210068FFF7A6FE03B05DF804FBF7B58B
:1010900005460068FDF7ACFD0023037004230446F9
:1010A0000DEB03022868FF21FFF794FE10B9002022
:1010B00003B0F0BD286804236A46FF21FFF78AFECB
:1010C0000028F4D09DF804108A09023A012AEED9CA
:1010D0009DF800209DF805309DF8015003EB012399
:1010E00005EB0225C3F30D03C5F30D055A1B002ABA
:1010F000B8BF5242FF2ADADC9DF806109DF807209F
:101100009DF8027002EB01229DF8031001EB07210C
:1011100049115611C1EB5212002AB8BF5242FF2AA0
:10112000C5DC01222B443144134111412270C4F823
:101130000530C4F80110BBE707B5022301AAFFF789
:1011400049FE044B1870BDF8040040BA80B203B0E9
:101150005DF804FB1009002038B515460D4A0B0A4E
:1011600082F8143C82F8151C022302F61442FF2177
:101170000446FFF79DFD10B96FF00C0038BD012348
:101180002A46FF212046FFF725FE0028F4D0002044
:10119000F4E700BF586E0020F8B5124D164685F8EA
:1011A000151C05F6144200240223FF21074685F88A
:1011B000144CFFF77DFD05F6144210B96FF00C00DA
:1011C000F8BD0223FF213846FFF704FE0028F5D0C2
:1011D00095F8142C95F8153C03EB02233380204638
:1011E000EEE700BF586E00202DE9F341754D04680D
:1011F000DFF8DC810023064685F864312D27B9B27B
:1012000018F8012B20460137FFF782FD882FF6D111
:10121000402287212046FFF77BFD00238DF8063012
:101220000DF10601204649F098F99DF80630002B93
:10123000F6D0012286212046FFF76AFD0022872191
:101240002046FFF765FD092208212046FFF760FDD3
:1012500000220B212046FFF75BFD002853D13768A1
:101260000DF106025E213846FFF796FFBDF8063005
:10127000B3F5D77F00F0A18055D8512B00F09B80AB
:1012800049D81D2B6CD01E2B00F095803068212191
:1012900049F0D2F834680DF10602DE212046FFF74E
:1012A0007BFFBDF806309FED487AC3F3090328227F
:1012B000ADF80630534307EE903AF8EEE77A434A2A
:1012C00067EE877A0021FCEEE77A82F8141C17EEAD
:1012D000903A6C2182F8151C190E82F8161C190C14
:1012E00082F8171C190A82F8181C82F8193CFF2191
:1012F00002F6144206232046FFF7DAFC306840224B
:101300008721FFF705FDB0FA80F0400985F86401F8
:1013100002B0BDE8F081AD2B4FD0D62B01D0602BB1
:10132000B4D121241DE040F2E132934247D00CD8E1
:1013300040F2D922934242D040F2E122934202D0BD
:10134000B3F5E67FA2D164240BE040F28F429342D2
:1013500003D040F29152934298D14FF4FA7400E0D6
:101360000F24002892D10A224B213846FFF7D0FCE7
:101370000F2260213846FFF7CBFC0D22632138464F
:10138000FFF7C6FCB82269213846FFF7C1FC40F6DA
:101390000D7278213846FFF7D3FC40F60E627A21B1
:1013A0003846FFF7CDFC00287FF470AF2146384661
:1013B00049F042F86AE71424D3E73224D1E7C8247D
:1013C000CFE700BF605D00209A99893F586E0020EA
:1013D000FC21060837B5124D95F864310446E3B197
:1013E00000680DF1050149F0B8F89DF805307BB1B2
:1013F0000DF1060220689621FFF7CEFE0A22BDF805
:101400000630B3FBF2F3074A9360012385F8653198
:10141000206801228621FFF77BFC03B030BD00BFAE
:10142000605D00201009002013B5022301AA0446C4
:1014300051210068FFF7CEFC114AF0B1BDF804302D
:101440005BBA9BB2D360D368B3F5C87F02DD4FF0BF
:10145000FF33D3600B4B0C4A1968D2F81C3D323372
:101460008B4208D2C2F81C1D2068002302F61452D9
:101470005121FFF71DFC02B010BD6FF00103E8E73A
:101480001009002014260020586E002007B5022302
:10149000006801AA0021FFF79DFC0F4B83F86C0147
:1014A000B0B1BDF804300D4A5BBA9BB2B3F5FA6F28
:1014B0003FBF0A21B3FBF1F307EE903AF8EEE77A6B
:1014C0002BBF4FF0FF33FDEEE77A1361C2ED047AD4
:1014D00003B05DF804FB00BF605D00201009002030
:1014E00013B502230C46006801AA0021FFF772FC25
:1014F00060B15CB19DF805309DF90420DB0903EB78
:10150000830302EB820203EB4203238002B010BD8F
:1015100073B5114B154690F910200446142000FBBA
:1015200002335E69A3689A0704D46069019149F0A7
:1015300029F90199304649F0EBFC012300222946A4
:10154000304649F095FCA3689B0702D42046FFF77C
:1015500011FA012002B070BD1009002073B50379A3
:10156000012B16460AD0022B15D18368DB0758BF22
:1015700041F0800102B0BDE87040C9E7826802F026
:101580000102CDE900620A46417C90F91000F9F7AA
:1015900041FA02B070BD0020FBE7F7B515460DF12A
:1015A00007021C4606460F46FFF7D8FF9DF8073096
:1015B00005EA0302A24209D023EA05022243394682
:1015C000304603B0BDE8F040FFF704BA03B0F0BD09
:1015D00013B504466A4600680821FFF7BFFF9DF86F
:1015E000003013F010037ED0206806236A460021E5
:1015F000FFF7F0FB002874D09DF801309DF8002023
:101600009DF80410DFED396A1B0203EB02439DF8DD
:1016100002201C021A4448BF02F17F429DF80330A9
:1016200007EE902A090201EB03419DF80530F8EE20
:10163000E77A0B44090287EEA66A48BF03F17F43AD
:1016400007EE903A2A4BB3F95C2005EE902AB3F9E5
:101650005E20F8EEE77A05EE102AB3F9702087EEE7
:10166000A67A06EE902AB3F96C2007EE902AF8EEDF
:10167000E66AF8EEE77AB3F96820E6EE267AD3ED6B
:10168000196AF8EEE66A26EE074AE6EE276AD3ED17
:10169000187AF8EEE77AB8EEC55AE6EE267A06EE44
:1016A000902AB3F96E20F8EEE66A04EE902AB3F9B8
:1016B0006A20E7EE267A06EE902AF8EEE44AF8EE83
:1016C000E66AF8EEE55AE6EE246A27EE057AE4EEDD
:1016D000267AC3ED1D7AF6EE007AA5EEA77A83EDA1
:1016E0001E7A02B010BD1846FBE700BF0000784824
:1016F000605D002030B5002385B00446C386836357
:101700000DF1070200680221FFF728FF18B9002534
:10171000284605B030BD9DF80730DB07F7D5062316
:1017200002AA03212068FFF755FB20680DF107028C
:101730000921FFF713FF05460028E8D09DF8073080
:1017400013F00C0FE3D1BDF808302068C3EB8333EE
:101750009B00E386BDF80A309B002387BDF80C3060
:10176000C3EB83339B00638701220A21FFF732F921
:10177000CEE71FB50446002300688DF807300DF151
:1017800007022721FFF7EAFE68B19DF8073013F042
:10179000080320D02068062302AA2821FFF71AFB9D
:1017A00018B9E086A06304B010BDBDF90830002B65
:1017B000B8BF03339B10E386BDF90A30002BB8BFD6
:1017C00003339B102387BDF90C30002BB8BF0333C4
:1017D0009B106387E7E71846E5E71FB5002104463D
:1017E000C18681630DF107020068FFF7B7FEC0B143
:1017F0009DF8073013F0080315D02068062302AACD
:101800000121FFF7E7FA60B1BDF808305BBAE38663
:10181000BDF80A305BBA2387BDF80C305BBA5B4277
:10182000638704B010BD1846FBE730B5002585B0CE
:101830000446C58685630DF1070200680621FFF79F
:101840008DFEA0B19DF8073013F0040311D020687D
:10185000062302AA2946FFF7BDFA40B1BDF80830B9
:10186000E386BDF80A302387BDF80C30638705B0E6
:1018700030BD1846FBE707B50DF10702FFF76EFE16
:10188000034B18709DF8070003B05DF804FB00BF20
:1018900010090020F8B5144E144F41F00102002148
:1018A0000446FFF7D5F93568C7F8205D13212046B7
:1018B000FFF7E1FF10F007000BD001220B212046BB
:1018C000FFF7C6F9002220461146FFF7C1F90120B3
:1018D00008E0D7F8242D002AE8D033689BB25B1BC0
:1018E0009A42E3D2F8BD00BF14260020586E0020B3
:1018F00010B50C460121FFF7BEFFC0F300132370A3
:10190000C0F3C003A370C0F380036370C0F38013FF
:10191000C0F3C010E370207110BD2DE9F047884678
:10192000502114460646FFF7A6FF01304000C0B222
:10193000208046213046FFF79EFF2D4F237801304F
:1019400080B27B434FF47A79A08003F5FA734FF4A9
:10195000FA6AB3FBF9F25121B3FBFAF300FB02334D
:101960003046B3FBF9F3E360FFF7E6FBC3B2C0F325
:101970000F22257803FA02F2013293B27D43E3800D
:1019800005F5FA723046B2FBF9F1B2FBFAF203FB4D
:1019900001227021B2FBF9F22282FFF76CFF0130C5
:1019A0004000C0B2608071213046FFF7C5FBC3B272
:1019B000C0F30F208340013398F803209BB22381AA
:1019C00012B1E2889B1A2381A37820897B4303F517
:1019D000FA734FF47A724FF4FA65B3FBF2F1B3FB8A
:1019E000F5F300FB0133B3FBF2F36382BDE8F0874C
:1019F000002F3A002DE9F047DA4FDFF87083DFF867
:101A000070934FF4FA738CB0044600268921006865
:101A1000C7F8243D88F86261FFF72DFF40F0010010
:101A2000C2B289212068FFF713F932462068882165
:101A3000FFF70EF9206801228021FFF709F92068DD
:101A40000122FF21FFF704F9324631462068FFF7F3
:101A5000FFF891212068FFF70EFF314687F8280D27
:101A600001222068FFF7F4F832462068FF21FFF7D3
:101A7000EFF8324620688021FFF7EAF860212068FD
:101A8000FFF7F9FE40F01200C2B260212068FFF7B4
:101A9000DFF8206820224421FFF729F92068FF227F
:101AA0000121FFF7D5F82568012280212846FFF79C
:101AB000CFF80122FF212846FFF7CAF83246314607
:101AC0002846FFF7C5F80622FF212846FFF7C0F891
:101AD00083212846FFF7CFFE40F00400C2B28321E5
:101AE0002846FFF7B5F80722FF212846FFF7B0F890
:101AF000012281212846FFF7ABF8012280212846E8
:101B0000FFF7A6F86B2294212846FFF7A1F832468A
:101B100083212846FFF79CF8D9F80060C7F8206DAC
:101B200083212846FFF7A7FE002800F050830122FA
:101B300028468321FFF78CF892212846FFF79BFE69
:101B40000022C0F3C716814681212846FFF780F89E
:101B500006222846FF21FFF77BF883212846FFF75E
:101B60008AFE832100F0FB022846FFF771F8284621
:101B70000122FF21FFF76CF8284601220021FFF720
:101B800067F828460022FF21FFF762F82846002266
:101B90008021FFF75DF8062305AAB0212068FFF732
:101BA00019F920680122FF21FFF752F8206800226E
:101BB0004F21FFF74DF820682C224E21FFF748F8FF
:101BC00020680022FF21FFF743F8B4222068B621E5
:101BD000FFF73EF80025002E18BF0C2609F07F09FC
:101BE0002A464FF0010C0CABC5F3C4005FFA85FE2A
:101BF0001844764510F81C3C05F0070102D89145C1
:101C000040F0F0820CFA01F123EA010300F81C3CD9
:101C10000135302DE7D1062305AAB0212068FFF752
:101C200047F8514B01221870FF212068FFF710F888
:101C3000002211462068FFF70BF820680022FF21E0
:101C4000FFF706F8206800220921FFF701F8206855
:101C500000221021FEF7FCFF206800221121FEF770
:101C6000F7FF206801222421FEF7F2FF2068FF22FF
:101C70002521FEF7EDFF206800227521FEF7E8FF21
:101C800020680122FF21FEF7E3FF20682C224E216D
:101C9000FEF7DEFF206800224821FEF7D9FF294623
:101CA00020682022FEF7D4FF20680022FF21FEF7E3
:101CB000CFFF294620680922FEF7CAFF20680022CC
:101CC0005421FEF7C5FF206804223121FEF7C0FF32
:101CD000206803223221FEF7BBFF206883224021C7
:101CE000FEF7B6FF206825224621FEF7B1FF2068E7
:101CF00000226021FEF7ACFF206800222721FEF7BA
:101D0000A7FF206806225021FEF7A2FF20680022CC
:101D10005121FEF79DFF206896225221FEF798FF81
:101D2000206808225621FEF793FF2A462068572193
:101D3000FEF78EFF206800226121FEF789FF2068F0
:101D400000226221FEF784FF206800226421FEF752
:101D50007FFF206800226521FEF77AFF2068A0221D
:101D6000662107E0586E002010090020605D002009
:101D700014260020FEF76CFF20680122FF21FEF7E9
:101D800067FF206832222221FEF762FF20681422BA
:101D90004721FEF75DFF2068FF224921FEF758FF2B
:101DA000206800224A21FEF753FF20680022FF210D
:101DB000FEF74EFF20680A227A21FEF749FF2068CD
:101DC00000227B21FEF744FF206821227821FEF7C4
:101DD0003FFF20680122FF21FEF73AFF20683422EE
:101DE0002321FEF735FF206800224221FEF730FF55
:101DF0002068FF224421FEF72BFF20682622452180
:101E0000FEF726FF206805224621FEF721FF40222B
:101E100011462068FEF71CFF206806220E21FEF7FF
:101E200017FF20681A222021FEF712FF20684022A7
:101E30004321FEF70DFF20680022FF21FEF708FF77
:101E4000206803223421FEF703FF20684422352155
:101E5000FEF7FEFE20680122FF21FEF7F9FE206852
:101E600004223121FEF7F4FE206809224B21FEF7FF
:101E7000EFFE206805224C21FEF7EAFE20680422CE
:101E80004D21FEF7E5FE20680022FF21FEF7E0FE6F
:101E9000206800224421FEF7DBFE20682022452135
:101EA000FEF7D6FE206808224721FEF7D1FE206803
:101EB00028224821FEF7CCFE206800226721FEF789
:101EC000C7FE206804227021FEF7C2FE20680122AE
:101ED0007121FEF7BDFE2068FE227221FEF7B8FEDA
:101EE000206800227621FEF7B3FE206800227721C9
:101EF000FEF7AEFE20680122FF21FEF7A9FE206852
:101F000001220D21FEF7A4FE20680022FF21FEF72A
:101F10009FFE206801228021FEF79AFE2068F822A9
:101F20000121FEF795FE20680122FF21FEF790FEB9
:101F3000206801228E21FEF78BFE206801220021FD
:101F4000FEF786FE20680022FF21FEF781FE206852
:101F500000228021FEF77CFE042220680A21FEF781
:101F600077FE256884212846FFF785FC842100F050
:101F7000EF022846FEF76CFE012220680B21FEF7D7
:101F800067FE2068019003A9FFF7B2FC019807AA39
:101F900003A9FFF7C2FC9DF80C30002B00F028814C
:101FA0000A9D05F684559DF80E30002B00F0238124
:101FB0000A9B03F2B22305EB43059DF80F3023B1D2
:101FC000BDF82C3003F525731D449DF8103023B166
:101FD000BDF82E3003F226231D442068C7F82C5D7F
:101FE000E8220121FEF734FE44F61F639D4203D927
:101FF0002068294648F0D1FA012220681146FEF7F0
:1020000027FE20684021FFF745FC002800F0E7800C
:10201000206801210222FEF71BFE20680021FFF745
:1020200039FC002800F0DB802068DFF8E491E8222A
:102030000121FEF70DFE202220684421FEF757FE05
:10204000256803A92846FFF753FC07AA03A92846D9
:10205000FFF763FC502257212846FEF7F9FD0822BE
:1020600056212846FEF7F4FD082250212846FEF7A7
:10207000EFFDBDF82C004FF47A7A48F20E660AFBA9
:102080000060B0FBF9F080B2FEF740FB5121024640
:102090002846FEF72CFE0A9A5C4B0AFB02669E421B
:1020A0009DBFB6FBF9F202F1FF32D2B2FF22462108
:1020B0002846FEF7CDFDD7F82C1D44F61F63994244
:1020C00002D9284648F069FA01212846FFF7D3FBD8
:1020D0000222064601212846FEF7BAFD00212846C5
:1020E000FFF7D8FB324601212846FEF7B1FD2468F0
:1020F00003A92046FFF7FCFB07AA03A92046FFF728
:102100000CFC482211462046FEF7A2FD082247217A
:102110002046FEF79DFD032232212046FEF798FD62
:10212000072230212046FEF793FD0122FF212046A1
:10213000FEF78EFD202230212046FEF789FD002289
:10214000FF212046FEF784FD062220467021FEF77F
:102150007FFDBDF82E304FF47A7246F6440002FB44
:1021600003004DF28803B0FBF3F09DF80F3080B20E
:102170001BB1BDF82230184480B2FEF7C7FA7121B6
:1021800002462046FEF7B3FDD7F82C1D44F61F6328
:10219000994202D9204648F000FA01212046FFF773
:1021A0006AFB0222054601212046FEF751FD00216F
:1021B0002046FFF76FFB2A4601212046FEF748FD27
:1021C0006423C7F8243D012388F8623107E0D9F879
:1021D00000309BB29B1BB3F5FA7F7FF6A1AC0CB02D
:1021E000BDE8F0870B41DB0744BF0132D2B20FE5F7
:1021F00040F63635D7E69DF80D30002B3FF4DDAEC6
:102200000A9B03F525731D44D7E600BF1B280D016B
:102210001C0C0100F8B53B4F97F862310446002BC7
:1022200037D0394D95F8306D012E33D0022E4FD076
:102230007EBB006801228021FEF70AFD2068012292
:10224000FF21FEF705FD206832463146FEF700FD0E
:1022500095F8282D20689121FEF7FAFC20680122CC
:102260003146FEF7F5FC20683246FF21FEF7F0FC10
:10227000206832468021FEF7EBFC206801223146BF
:10228000FEF7E6FC214B1B68C5F8203D012385F8CD
:10229000303DF8BD00680021FFF7EDFAC20711D507
:1022A000D5F8242D002AF4D0184BD5F8201D1B6832
:1022B0009BB25B1A9A42ECD2154B4FF0FF325A6038
:1022C0000023E4E7114B1B68C5F8203D0223DEE73D
:1022D00000681321FFF7CFFA4307E1D01E212068E1
:1022E000FEF72AFF012206460B212068FEF7B0FC0C
:1022F000074B0A20B6FBF0F6B6B25E60012387F802
:102300006331DDE7605D0020586E00201426002058
:1023100010090020F0B513238DB0054600222921B5
:102320000220FDF7C5F9524CC4F8EC01002800F07A
:1023300091800221FCF714FC02220021D4F8EC0168
:10234000FEF748FB002384F8F43184F8F05104F5DB
:10235000FC7304F5B7624FF0202143F8041B93424D
:10236000FBD1444E444F35683235D4F8EC01037943
:10237000012B71D0022B0FD183683F4ADB074FF04E
:1023800080015CBF3C4A8021FFF7C2F810B133687E
:102390009D42EAD8D4F8EC011024112213214FF009
:1023A000120E4FF0140C1527162617258DF80C4029
:1023B0008DF80E20182419228DF812101B210123EC
:1023C0008DF810E08DF814C08DF816708DF8186037
:1023D0008DF81A508DF81C408DF81E208DF82210B3
:1023E0004FF01A0E4FF01C0C1D271E261F254C24E3
:1023F000222203A98DF80D308DF80F308DF81130A1
:102400008DF813308DF815308DF817308DF81930A0
:102410008DF81B308DF81D308DF81F308DF820E0C1
:102420008DF821308DF823308DF824C08DF82530BB
:102430008DF826708DF827308DF828608DF82930BA
:102440008DF82A508DF82B308DF82C308DF82D40DA
:1024500048F039FD0DB0F0BD8268417C90F9100064
:1024600002F00102CDE900728022F8F7D3FA8DE77D
:10247000605D002014260020535F0020F0B5514C11
:10248000D4F8EC5185B015B194F8F2310BB105B028
:10249000F0BD012384F8F2312B79012B7CD0022B83
:1024A00037D128460DF10E028421FFF731F8D4F818
:1024B000EC5194F8F4212B79012B42F0040279D1EC
:1024C0008DF80F20AA6895F91000697C02F00102CE
:1024D00001920DF10F0200920422F8F775FA15E04F
:1024E000022B0ED1AB6813F0010F0DF10E024FF06D
:1024F0008401284602BF0DF10E0284212846FFF711
:1025000007F89DF80E3013F0040616D0D4F8EC51FD
:102510002B79012BE4D1AA68697C95F9100002F0AF
:10252000010201920DF10E0200928422F8F772FA74
:102530009DF80E3013F00406E8D1234D234884F8AB
:10254000F43131463C224FF006FA01273146A5F11D
:10255000460E05F5707635F8023F1A0A4FEA511C0F
:1025600003F0040322F02002134318BF5EF82C305E
:1025700001F01F0007FA00F01CBF18434EF82C00B2
:10258000B54201F10101E6D1FBF7DAFE0028FBD1EB
:1025900084F8F20105B0F0BDAA68697C95F91000D5
:1025A00002F0010201920DF10E0200928422F8F76E
:1025B00031FA7CE7022BACD128460421FEF7E5F97D
:1025C000A4E700BF605D0020565F0020105F002080
:1025D00010B52D4CD4F8EC0184B0E8B194F8F0318A
:1025E000012B32D0022B19D10823002104228DF8AF
:1025F0000C1003A984F8F3318DF80D308DF80E20FE
:102600008DF80F2048F05FFC20483C22FF214FF05E
:10261000A2F994F8F131D3B104B010BD0379012BC4
:1026200022D0022B1AD09DF80B3003F00503012BAA
:1026300009D013B9D4F8EC01D6E7154A126840F274
:10264000DC539A42E8D9D4F8EC014823CDE7FFF7F0
:1026500015FF012384F8F13104B010BD0DF10B0218
:10266000A021FEF755FFDEE7826890F910C0417C9B
:1026700002F0010201920DF10B0200926046A022CD
:10268000F8F7C8F9CFE700BF605D0020105F0020B9
:1026900014260020F0B53E4CD4F8EC5185B095B12D
:1026A00094F8F331180702D594F8F2316BB194F82D
:1026B000F13143B9FFF78CFF94F8F131002B3BD196
:1026C000002384F8F23105B0F0BD94F8F131012215
:1026D00084F8F221002BEDD02B79012B2FD0022B87
:1026E000E8D10DF10E0280212846FEF711FF0028E7
:1026F000E0D094F8F3219DF80E309A42DAD194F8A4
:10270000F051002DD8D1234B234E1F68D6F8343D0D
:10271000FB1AB3F57A7FCFD9A021D4F8EC010DF1E3
:102720000F02FEF71BFF9DF80F30590715D5C6F8AD
:10273000385DC6F8347DBFE7FBF702FEC0E7AA6844
:10274000697C95F9100002F0010201920DF10E0270
:1027500000928022F8F75EF9C9E703F00503012B28
:102760000ED0002BE5D194F8F3315B06E1D5D6F815
:10277000383D53B1FB1A642BDBD9FFF729FFD8E7AB
:1027800094F8F3315A06F2D5D3E7C6F8387DD0E78E
:10279000605D002014260020586E00202DE9F043D3
:1027A0008E4ED6F8EC4185B0002C6ED096F8F291A2
:1027B000B9F1000F00D0FEE796F8F3C101230CF049
:1027C000F70C86F8F3C186F8F2312379012B054620
:1027D0000F4600F0DF80022B00F097800DF10F080C
:1027E000B5F5807F00F0B4802379012B00F0BB8029
:1027F000022B07D1204650220821FEF7C6F8D6F852
:10280000EC412379764D012B1AD0022B0AD1424696
:102810002046A021FEF77CFE20B19DF80F4014F069
:10282000200451D0D5F81C32B5F820225969D6F8C9
:10283000EC410A4214BF5A831A832379012BE4D155
:10284000A268617C94F9100002F00102CDE90082D7
:10285000A022F8F7DFF8DFE7B9F1000F12D196F800
:10286000F341D6F8EC5104F0F70486F8F3412B79E4
:10287000012B00F0A580022B04D1224649462846B0
:10288000FEF783F8002386F8F23105B0BDE8F08347
:10289000022B16D162460A212846FEF776F8D6F8B2
:1028A000EC010379012B07EB040228D18568417CF8
:1028B00090F9100005F00105CDE90025C022F8F7D8
:1028C000A9F80134362CC7D0D6F8EC512B79012B5E
:1028D0005FFA84FCDCD1AA6895F91000697C8DF858
:1028E0000FC002F00102CDE900820A22F8F76CF86D
:1028F000D6F8EC010379012B07EB0402D6D0022BAA
:10290000DFD1C021FEF704FEDBE7494620466246E0
:10291000FEF73BF8D6F8EC41237981460DF10F081C
:10292000012BEAB22ED1A16894F9100001F0010C3C
:10293000617C8DF80F20CDF804C0CDF8008009220D
:10294000F8F742F8B5F5807FD6F8EC417FF44CAF4C
:10295000204640220A21FEF73DF8D6F8EC412379C3
:10296000012B7FF445AFA26894F91000617C02F05E
:102970000102CDE9008250228DF80F200822F8F7DD
:1029800023F83CE7022B7FF42BAF20460921FDF70B
:10299000FCFFD7E7A16894F9100001F0010E0DF1DA
:1029A0000F08617CCDF804E04A46CDF800808DF830
:1029B0000FC0F8F709F8D6F8EC4181462379AFE764
:1029C000A96895F9100001F001074A46697C8DF865
:1029D0000F40CDE90087F7F7F7FF53E7605D002070
:1029E000683900202DE9F04F5E4B93F8F251C7B0E3
:1029F00005B1FEE75B4A92F8F371012382F8F231E8
:102A000007F0F707D2F8EC3182F8F37103931B79E2
:102A1000012B04460E4600F09580022B40F090807A
:102A20000398836813F0010118BF29463A46FDF761
:102A3000ACFF05AD4B4BD3F8EC310393FF2C6C701E
:102A40004FF0090388BFA4082B708CBF04F0C008A6
:102A50004FF00008022200204FF00A090DF1150A7C
:102A60004FF00B0B10E0BEF5827F05F80290375C4B
:102A70000AF8023013D80130362805F804B002F104
:102A8000060C6F54724612D0941C48EA0003B4F549
:102A9000827F02F1040EDBB202F10301E3D90130BF
:102AA0006FF0004E3628DFF8C4C07246ECD1BCF59A
:102AB000827F9FBF08210DF1150305F80E10A0219C
:102AC00098BF03F80E10039894BF02326FF00042D3
:102AD000294648F0F8F9234B234DD3F8EC0103794C
:102AE000012B0DF1130419D0022B08D12246A0218D
:102AF000FEF70EFD18B1237813F020031AD0D5F895
:102B00001C32B5F8202259690A4214BF5A831A832D
:102B1000144BD3F8EC010379012BE5D18268417C99
:102B200090F9100002F00102CDE90042A022F7F76F
:102B300071FFDFE70B4A82F8F23147B0BDE8F08F52
:102B400005AD7BE7039881682A4601F0010501463F
:102B500090F91000497C019505AD2F700095F7F7AD
:102B600033FF67E7605D00206839002001000080C6
:102B7000024BD3F8EC3103B134E77047605D0020BD
:102B800010B5EFF31182102383F312884FF0E02386
:102B9000D2B29C69196911F4803F0D491EBF012012
:102BA000C1F80C0C9C690B4B1868D1F80C3C82F3F3
:102BB0001188094A11684FF47A72034402FB01F04C
:102BC000001BB0FBF1F00021E3FB020110BD00BFD0
:102BD000586E0020142600200C2E0020124B5B683B
:102BE000C3F3080330B4EBB9EFF31183D3B90F4B40
:102BF0000F484FF0E0251968AC691A688A42FAD18B
:102C0000D0F8081CA142F6D30A4B19684FF47A7326
:102C100003FB01F0001BB0FBF1F00021E2FB03011C
:102C200030BC704730BCABE700ED00E0142600205C
:102C3000586E00200C2E0020F8B506460D46FFF712
:102C4000CDFF04460F46FFF7C9FF031B61EB0702E8
:102C5000B34272EB0503F6D3F8BD10B50446013C50
:102C600000D210BD4FF47A700021FFF7E5FFF6E7C0
:102C700037B5054605249620FFF7EFFF0DF1070253
:102C800000212846FEF76AFC08B9013CF3D103B0E5
:102C900030BD38B500231A4635210120FCF708FD68
:102CA000164D0446C5F83C0D48B9154B85F8400D46
:102CB0001B781A2B04BF0123C5F8443D38BDFFF72C
:102CC000D7FF70B90E4B1B781A2B08BF0223204682
:102CD00008BFC5F8443DFBF736FF002385F8403DAB
:102CE000ECE70123002285F8403D85F8412D204680
:102CF0004021BDE83840FDF76DBE00BF586E002092
:102D0000F33B002008B5054B02463D211868FDF74E
:102D100061FEBDE8084019209FE700BFF048002091
:102D200084B070B590B014AC504E9DF8685084E8F3
:102D30000F0000244FF08070C6F8044C1CF026FDF4
:102D400028B9002010B0BDE8704004B070474FF4BF
:102D5000E133032290F904000294CDE900324FF0F0
:102D60008071434A23461CF0CDFEC6F8040C0028AF
:102D7000E7D001212046FDF713FD0520FFF76DFF89
:102D80003C4B93F87421012ADBD193F87521A02ADA
:102D9000D7D193F86D110029D3D13E200591FDF7CD
:102DA000F5FC1920FFF759FF0599002D54D03D205F
:102DB000FDF7ECFC14AC1920FFF74FFF0FCC0AAD68
:102DC0000FC5BDF95830BDF9562094E803008DF8C1
:102DD00020301B128DF82130BDF932308DF82230B1
:102DE0001B128DF82330BDF93430A9808DF82430C2
:102DF000BDF954108DF81C101B128DF82530BDF94B
:102E000036308DF81E2009121212BDF95050BDF94E
:102E100052408DF81D108DF81F2007A90C228DF847
:102E2000263055201B128DF82730FDF781FC192024
:102E3000FFF713FF8DF81C508DF81E4067202D12F0
:102E40002412042207A98DF81D508DF81F40FDF7AC
:102E50006FFC1920FFF701FF0C213D20FDF796FCC8
:102E60001920FFF7FAFE01206CE700BF586E002022
:102E700079E00008605D002013B5002204460A21B5
:102E80000068FDF7A7FD1420FFF7E7FE0F220A21D7
:102E90002068FDF79FFD0A20FFF7DFFE032301AA4C
:102EA00010212068FDF796FF0A20FFF7D6FE0022CA
:102EB0000A212068FDF78EFD0A20FFF7CEFE0DF1F6
:102EC000030220680221FEF749FB0DF1030220688E
:102ED0000921FEF743FB206801220A21FDF77AFD54
:102EE000012002B010BD10B5782204460021006810
:102EF000FDF770FD0520FFF7B0FE202201212068BC
:102F0000FDF768FD0520FFF7A8FE002202212068DA
:102F1000FDF760FD6420FFF7A0FE012010BD10B595
:102F20002422044641210068FDF754FD80B1206849
:102F300020223021FDF74EFD50B1206806223121BC
:102F4000FDF748FD20B1206800223421FDF742FD45
:102F50000520FFF782FE012010BD10B507220446B0
:102F60000A210068FDF736FD0520FFF776FE2422D2
:102F700041212068FDF72EFD0520FFF76EFEC022DF
:102F800042212068FDF726FD0520FFF766FE01209F
:102F900010BD10B50122044610210068FDF71AFD8E
:102FA00048B11420FFF759FE2068A022BDE8104068
:102FB0001121FDF70FBD10BD08B5006801220921E0
:102FC000FDF708FDBDE80840642046E680B50646EA
:102FD0000B25013D01D1FDF77BFC01210846FCF7E3
:102FE000F1FC00210846FCF7EDFC771C4FF032089D
:102FF00005240120FCF7D6FC0020FCF7D3FC0120BF
:10300000FDF72FFC4046FFF728FE0120FCF7CAFC25
:103010000020FCF7C7FCFDF724FC4046FFF71DFE2F
:103020007CB1013C05D14FF4FA70FFF716FE4FF06A
:10303000FA0854EA0703DCD14FF47A70FFF70DFE6B
:10304000C7E7013FF5E72DE9F043026B066890F80A
:103050002D30AF49B1FBF2FE0546AE488BB00246BB
:1030600007464FF0000C012492F80690A3EB0908E4
:10307000A3EB0C01B8F1000FB8BFC8F1000800299C
:10308000B8BF4942884502F1060204F10104BCBF01
:103090004FFA89FC1746102CE6D11FFA8EFE0278F3
:1030A00062450ED179884288AEEB0101AEEB020297
:1030B0000029B8BF4942002AB8BF52429142C8BF56
:1030C0000746013C00F10600E9D17A7904923A7989
:1030D00003927A8802923A780120CDE900E2032136
:1030E0008D4AF9F73FFD7A88894BB3FBF2F3AB6366
:1030F0002B689869A8B140F61503C3800472214675
:10310000FCF714F8854BAB612B6899690846FBF70F
:10311000EBFE002880F28C802B689869002840F034
:10312000E98000213046FBF71BFD80226B213046F1
:10313000FDF750FC9620FFF790FD032268213046F2
:10314000FDF748FC9620FFF788FD03226B213046EF
:10315000FDF740FC0F200021FFF76EFD10226A21D1
:103160003046FDF737FC0F200021FFF765FD0022F8
:103170006C213046FDF72EFC0F200021FFF75CFD8F
:103180007A7919213046FDF725FC0F200021FFF741
:1031900053FD18221B213046FDF71CFC0F20002197
:1031A000FFF74AFD18221C213046FDF713FC0F20C3
:1031B0000021FFF741FD102237213046FDF70AFCC0
:1031C0000F200021FFF738FD012238213046FDF79E
:1031D00001FC0F200021FFF72FFD3A791A2130461C
:1031E000FDF7F8FB01200021FFF726FD0321304603
:1031F000FBF7B6FC2868062308AA4321FDF7EAFD81
:1032000058B1BDF820305BBA2B84BDF822305BBAD0
:103210006B84BDF824305BBAAB8495F9223001335E
:1032200073D195F9203001336FD10620FFF7CEFE20
:10323000DFF8FC803A4A08EB000393F81C9405F190
:10324000180342F820300846FBF743FE02460846C2
:10325000FBF74AFE00F0FC0303F1804303F59C33C7
:1032600000F0030C4FEA8C0C98684FF00F0E0EFA2A
:103270000CFE20EA0E009860D3F808E0D0B200FA05
:103280000CF242EA0E029A6021B10846FBF72CFECE
:1032900001248440234B5C611A6822EA04021A600C
:1032A0005A6822EA04025A601F4AD2F8001C2143DD
:1032B000C2F8001C996821EA04019960D96821EAE2
:1032C0000401D960D2F8080C184B0443C2F8084C2A
:1032D00013F80920042A7FF61FAFC844042198F987
:1032E0002C0403F809100790F6F700F80798F5F793
:1032F000EFFF11E7FBF7F8FD012313FA00F01FBF02
:10330000084A1368184310600BE70BB0BDE8F08360
:1033100040420F0058220608F3AA060855D90008B3
:10332000F43B0020003C014000300140343C0020D0
:103330009C1E060818B103685B6803B11847FF209C
:10334000704718B103689B6803B1184700207047A5
:1033500070B450B106798E4207D34579954204D3B3
:103360000368DB680BB170BC184770BC704710B4C1
:1033700040B184798C4205D303681B6913B15DF8B1
:10338000044B18475DF8044B704718B103685B693C
:1033900003B11847704718B103681B6A03B1184797
:1033A0000020704730B560B1041D0A4600F11403D7
:1033B00020686168154603C508349C422A46F7D147
:1033C000012030BD10B50C4670B92D2300202375A7
:1033D000094B2061C4E90000C4E90200C4E90633D6
:1033E000302384F8203010BD0368DB6A002BECD05A
:1033F00098470028E9D0F6E7E7B0060838B5054D4C
:10340000441E14F8011F01B938BDD5F8640DFBF74F
:1034100089FBF6E7586E002013B50C4C01900C4860
:103420000091FFF7EBFFDDE900320A49D4F8640DA3
:1034300045F09AFDD4F8640DFBF768FB94F8683DFD
:1034400013B1012384F8693D02B010BD586E00200D
:103450002CAB060845EB000808B50648FFF7CEFF81
:10346000054BB3F86A0D18B1BDE80840FFF7F5BB8E
:1034700008BD00BFBAFC0608586E002010B5074C06
:1034800002460B46D4F8640D054945F06DFDD4F8AD
:10349000640DFBF73BFBBDE81040DDE7586E0020F4
:1034A00045EB000808B5FFF7A9FFBDE80840D3E7E2
:1034B00010B504460648FFF7A1FF2046FFF79EFF20
:1034C000044B93F8682D12B1012283F8692D10BDC9
:1034D0002CAB0608586E002010B504460348FFF7D1
:1034E0008DFF2046BDE81040DCE700BF38AB060882
:1034F0000CB4830607B500D551B9049805A901910C
:10350000FFF7BCFF012003B05DF804EB02B0704789
:103510000020F8E7024B0146D3F8640DFBF702BB2D
:10352000586E00200CB407B510F0400009D069B9FE
:103530002320FFF7EFFF049805A90191FFF79EFFF5
:10354000012003B05DF804EB02B070470020F8E7FB
:103550000FB413B5094C0A49D4F8640D04AB53F801
:10356000042B019345F000FDD4F8640DFBF7CEFA6F
:1035700002B0BDE8104004B0704700BF586E002094
:1035800045EB00080FB407B504A951F8040B0191ED
:10359000FFF774FF03B05DF804EB04B070470FB49D
:1035A00007B504A951F8040B0191FFF735FFFFF7A8
:1035B00053FF03B05DF804EB04B0704770B5837936
:1035C000164603F00F028EB00446062A50D8DFE8F4
:1035D00002F0041417191C1E4A000D7813F0C003E2
:1035E00048D0402B3DD12946204611F03BFD002814
:1035F0005BD00EB0BDE87040AAE791F90050EDE74E
:103600000D88EBE7B1F90050E8E70D68E6E791EDCA
:10361000000A03A8F9F788FE01462948FFF798FF3A
:10362000FEB1A37913F0C00F1BD1204611F067FC47
:1036300000EE100A03A8B8EEC00AF9F775FE0146BD
:103640002048FFF785FF204611F06AFC00EE100AC3
:1036500003A8B8EE400AF9F767FE01461948FFF7DC
:1036600077FF0EB070BD16480EB0BDE870406FE732
:103670000025B3E7042A0CBF134814482946FFF776
:1036800067FF002EEDD0A37913F0C00FE9D12046DB
:1036900011F035FC0190204611F042FC01990246E0
:1036A0000B480EB0BDE8704052E703A9204611F068
:1036B0004BFB084803AA2946FFF771FFD1E700BF7B
:1036C0001AAF06082FAF06088EAB0608F6EB060801
:1036D00085FE06083DAB06082DE9F04F8FB001F0DE
:1036E00020034D4C009381460F464FF000084B4B92
:1036F000D3F8640DFBF70AFA94F806B00BF0300328
:103700004B454BD1204611F099FBF9F7FFFF0646D8
:10371000204611F0B5FBD6F808A005460AEB0006D6
:10372000204611F0DFFB0BF00F02062A6CD8DFE811
:1037300002F0044045494E525E001AF80520007818
:10374000111A4A424A41009B03B13ABB03A92046E1
:10375000019211F0F9FA7B0615D5019A9AB9304811
:1037600003A9FFF7F5FE2F4903A847F0A1FC0028A5
:103770004CD11AF80530202B48D12B483146FFF7A1
:10378000E7FEFFF769FE294803A9FFF7E1FE0022E3
:1037900031462046FFF712FFFFF75EFE08F10108F1
:1037A00040F24623984504F10B04A0D10FB0BDE8C8
:1037B000F08F1AF9052090F90000C1E73AF80520CA
:1037C0000088BDE73AF90520B0F90000B8E75AF8DB
:1037D00005200068B4E796ED007AD0ED007AB4EEEB
:1037E000677AF1EE10FA0CBF01220022ABE70190DC
:1037F000204611F095FB0199421C30464EF0FAF834
:10380000B0FA80F252099EE700229CE7002231467E
:103810002046FFF7D3FEB4E718230608586E0020B1
:103820005AAB060857FE060865AB06085BAB0608F0
:1038300013B50446019111F055FB019A014620464B
:1038400002B0BDE81040B9E6F7B5847914F0C003C2
:10385000054603D0402B18D003B0F0BD04F00F0490
:1038600011F05EFB062C05D10146164803B0BDE8F9
:10387000F04087E60190284611F041FB019A01468D
:10388000114803B0BDE8F0407CE611F0DBFB0546D3
:103890000E480F4E0F4FFFF7B1FD00242B79A342C6
:1038A00003D803B0BDE8F040D6E514B13046FFF7C9
:1038B000A5FD2B68384653F82410FFF749FE013464
:1038C000ECE700BF6AAB06087AAB060891AB0608C6
:1038D000A1AB06082FAF060808B50548FFF78EFD17
:1038E000044BD3F8640DBDE80840FBF70FB900BFE7
:1038F00038AB0608586E0020004850E6A3AB060817
:1039000013460A460146014849E600BFAFAB060828
:1039100020B10078B0FA80F040097047012070476C
:103920002DE9F04F87B00346FFF7F2FF064618B1C6
:1039300007B0BDE8F04FDFE74649DFF84091DFF818
:1039400040A1DFF840B105AA18464DF0AAFF344661
:103950000546B0464FF0FF378DB97EB230461BF0BA
:1039600001FF10B14568002D5AD1B8F1000F36D1D2
:1039700039483946F9F7C4F807B0BDE8F08F012E91
:103980000ED0022E11D01EB92846F9F717FE0746B1
:10399000304905AA00204DF084FF01360546DBE7DB
:1039A0002846F9F70BFE8046F2E7494628464EF0D6
:1039B00058F820B9294928464EF053F808B144F088
:1039C0000104514628464EF04CF828B9594628467D
:1039D0004EF047F80028DBD044F00204D8E7002C72
:1039E00008BF03240023E4B2CDE9008402931A4601
:1039F000194630461CF086F8054610B91848394675
:103A0000B8E7184842463946F9F77AF83946164871
:103A1000F9F776F8154B2946D3F86C0D43F0A0F86A
:103A200013483946F9F76CF85CB16979A14208D0BE
:103A300010482246F9F764F82B68E1B29B692846E2
:103A40009847EB6A002BE1D00B48F9F759F80023AF
:103A5000EB62DBE78DAA0608CFAB0608DADA0608C8
:103A6000F7AB060816AC060881AC0608586E0020B5
:103A700033AC06084BAC06086BAC0608D2B9060896
:103A8000CCAB0608E1BF06082DE9F04F85B005462E
:103A9000FFF73EFF044630B10021012005B0BDE82C
:103AA000F04F43F0B7B885492846F9F743FA20B9F3
:103AB00005B0BDE8F04F3AF021B881492846F9F742
:103AC00039FA28B9012005B0BDE8F04F3AF00EB937
:103AD0007C492846F9F72EFA034688BB7A4A92F9C0
:103AE000D61F82F8D00F104692F89054012D08D0BE
:103AF000033D052D05D9002C00F0D28080F8D61F9B
:103B0000CEE092F8A654A52D03F1010313D10129AB
:103B10000ED16E4A80F8D13F002380F8D01F82F882
:103B2000703D80F8D63F05B0BDE8F04F3AF064B97B
:103B3000013949B20124782B02F11802D4D1DAE715
:103B40002846F9F73BFD614B93F9703D009303FA6A
:103B500080F6772E834600F2A7802846FAF700FF0A
:103B60000746002800F08980F9F728FD0124C5B236
:103B70003846FAF7F5FE0746002800F08180F9F78D
:103B80001DFD01340190E4B23846FAF7E9FE8046A3
:103B9000002877D0F9F712FD01340746E4B2404619
:103BA000FAF7DEFE814600286ED0F9F707FD0134F2
:103BB0000290E4B24846FAF7D3FE8246002865D068
:103BC000F9F7FCFC01340FFA80F9E4B25046FAF739
:103BD000C7FE824600285BD0F9F7F0FC01340FFAEB
:103BE00080F8E4B25046FAF7BBFE002852D00390AA
:103BF000F9F7E4FC03990FFA80FA0846FAF7B0FEE9
:103C00000346002857D004F0FD04F9F7D7FC042C34
:103C100046D1C3B2012D02D9E91E052940D81BB1F6
:103C2000A52B01D0482B3BD1274C0EB984F8D66F79
:103C3000182101FB0646019AC6F89424A52B029A86
:103C400086F89054C6F89874C6F89C24A6F8A094F8
:103C5000A6F8A284A6F8A4A486F8A6340AD10098EF
:103C60001A4B0130584483F8700D94F8D63F013355
:103C700084F8D63F05B0BDE8F08F0446054677E7E7
:103C8000019081E707468AE7029093E781469DE726
:103C90008046A7E75FFA88F382468046062CB9D0B3
:103CA00005B0BDE8F04F27E609487722214605B068
:103CB000BDE8F04F24E60134E4B2EFE7AFAC06080C
:103CC000B5AC0608D7B60608504D0020586E002047
:103CD000BAAC060808B50346FFF71AFE40B10C4B14
:103CE0000C480022A3F86A2DBDE80840FFF7DABBB4
:103CF0001846F9F763FC014630B1054BA3F86A0D8D
:103D0000BDE8084004483DE4BDE80840F4E500BFD4
:103D1000586E0020C3AC0608D9AC06082DE9F04F58
:103D2000DFF8B8A087B0074616460C4615464FF098
:103D3000000B4FF019094FF46178002E4BD0237817
:103D400028788342EB7844D161786A78914240D1F7
:103D5000A178AA7891423CD1E178CA1A51425141E6
:103D6000CDE9041310F03AFD059B049919FB038378
:103D70000393AB7819FB038302936B780193037A67
:103D8000009352465B463846FFF7CCFB04992078F7
:103D9000049110F023FDE378049919FB0383039346
:103DA000A37819FB0383029363780193037A00934A
:103DB00052465B4638460BF1010BFFF799FBBBF10E
:103DC000280F04F1040405F10405B6D107B0BDE8DD
:103DD000F08F0021C4E73146D9E700BFF0AC0608F8
:103DE000F7B50646FFF794FD054630B12549002298
:103DF000012003B0BDE8F04090E73046F9F7DEFB64
:103E00002728044636DC8700701C8DF80750FAF727
:103E1000A7FD1C4D064668B1F9F7D0FB002809DB69
:103E2000C0B210F0EDFC28B1037805F8243001236E
:103E30008DF807303046FAF793FD064650B1F9F792
:103E4000BDFB0D2806D8EB1958709DF807300133DB
:103E50008DF80730B91C0DF1070229443046FAF7F6
:103E60008CFD9DF80730042B02D0002345F8243048
:103E700003B0F0BD04482722294603B0BDE8F04056
:103E80003EE500BF04420020D5AD06082DE9F04F05
:103E900089B0374EDFF8E090069280460C46154612
:103EA00002F13C0B94F9041000230C22314F02FB69
:103EB00003F0C057884255D00133052BF6D10C359D
:103EC0005D4504F10C04EDD109B0BDE8F08F95F922
:103ED00004302A68687995F806C095F808E095F8E6
:103EE00007A099423CD12168914239D16179814240
:103EF00036D1A179614533D1217A714530D1E1794B
:103F0000A1EB0A077942794156F82A7056F8200049
:103F1000049756F82E70039756F82C700297CDE947
:103F200000204A4640460791FFF7FCFA0799E279DC
:103F300094F9043056F822200492227A56F822206E
:103F40000392A27956F822200292627956F8222032
:103F500001922268009240464A46FFF7C9FAAEE74E
:103F60000021D1E7069B002BB1D11946DFE700BF46
:103F70009C1D0608643C002003AD0608F0B585B022
:103F80000346FFF7C5FC30B143490022012005B0CC
:103F9000BDE8F0407AE718465E1CF9F70FFB0446CF
:103FA00040B21BF069FD054630B93C48214605B0DA
:103FB000BDE8F040FFF7F3BA0068696801AB03C3DE
:103FC000A86818603046FAF7CBFC0446002852D0A7
:103FD00003782B2B05D02D2B42D0F9F7EFFA019067
:103FE00009E001342046F9F7E9FA019B012202FABF
:103FF00000F003430193022600272046FAF7B0FCA5
:10400000044638B3F9F7DAFA254A0023114652F884
:1040100004EB70455FFA83FC04D00133112BF6D119
:104020004FF0000C51F82C30984213D1102200218F
:104030006046F7F735FF022F1FD0032F20D0012F46
:1040400014BF8DF809008DF80A0001370136042FDE
:10405000F6B2D2D1012E16D805B0BDE8F0404BE43F
:1040600001342046F9F7AAFA019B012202FA00F076
:1040700023EA0003BEE70126BEE78DF80C00E4E763
:104080008DF80B00E1E701AB03CB2860186869608D
:10409000A86005B0F0BD00BF9445002020AD060823
:1040A0009C1D06082DE9F04FDFF8C0B089B08046AE
:1040B00017460C46154600264FF0190A4FF4617951
:1040C000002F51D06979A8780791A1782B786A7868
:1040D00095F803C095F804E00693814242D1217817
:1040E00099423FD1617891423CD1E178614539D123
:1040F0002179714536D1079963795B1A5942594143
:10410000069B06911AFB0393CDE901031AFB029269
:10411000079B03920093CDE904CE33465A464046AE
:10412000FFF700FA069923790593E37804936378FF
:104130001AFB0393039323781AFB03930293A37848
:104140000193637900935A46334640460136FFF7A0
:10415000CFF9142E04F1060405F10605B0D109B01B
:10416000BDE8F08F0021CBE73946DCE733AD060828
:104170002DE9F3478246FFF7CBFB064630B13C49B9
:104180000022012002B0BDE8F0478BE75046F9F766
:1041900015FA1328054663DC062747430AF1010098
:1041A0008DF80760334CFAF7DBFB04F6715909EB25
:1041B0000708064648B1F9F701FA03289FBFE3193B
:1041C00083F8760D01238DF807303046FAF7C8FBE7
:1041D000064668B1F9F7F2F90D2809D8062303FB62
:1041E000054383F8730D9DF8073001338DF80730D0
:1041F0000DF1070241463046FAF7BFFBFAF7B0FB74
:10420000064668B1F9F7DAF93A2809D89DF8073077
:10421000062202FB0542013382F8740D8DF8073047
:104220003046FAF79DFB68B1F9F7C8F90D2809D8AF
:104230009DF80730062202FB0544013384F8750D12
:104240008DF807309DF80730062B06D0002349F87B
:104250000730A8F80430FFF74FFB02B0BDE8F08745
:1042600005481322314602B0BDE8F047FFF748BBCE
:10427000C97B0020586E0020D5AD06082DE9F04F0F
:104280002DED088BDFF814A197B0074690460C4639
:104290001546002694ED008AB5EE408AF1EE10FA3C
:1042A00073D0D4ED019A94ED029AD4ED038AB8F15B
:1042B000000F40D095ED000A95ED01BAD5ED02AAA8
:1042C00095ED03AAB4EE408AF1EE10FA62D1F4EE55
:1042D0004B9AF1EE10FA5DD1B4EE6A9AF1EE10FA53
:1042E00058D1F4EE4A8AF1EE10FA0CBF4FF00109F2
:1042F0004FF0000912A8F9F717F8B0EE4B0A834601
:104300000EA8F9F711F8B0EE6A0A05900AA8F9F7B5
:104310000BF8B0EE4A0A049006A8F9F705F8059BD9
:10432000049A0390CDE900B30292334652464946BF
:104330003846FFF7F7F8B0EE480A12A8F8F7F4FF8E
:10434000B0EE690A81460EA8F8F7EEFFB0EE490A12
:1043500083460AA8F8F7E8FFB0EE680A049006A8BA
:10436000F8F7E2FF049B0390CDE901B3CDF800908C
:1043700033465246002138460136FFF7B9F80C2E75
:1043800004F1100405F1100584D117B0BDEC088BC1
:10439000BDE8F08F4FF00009ACE700BF51AD060853
:1043A00070B50546FFF7B4FA064628B1BDE870407F
:1043B0002C490022012061E72B4905222846F8F705
:1043C0009DFD38B9274B002201300C2843F8102BF3
:1043D000FAD170BD2846F9F7F1F80B2804463AD80F
:1043E0002846FAF7BDFA064648B3F9F705F81D4B1B
:1043F00003EB041383ED000A01253046FAF7B0FA07
:10440000064638B1F8F7F8FF164B03EB041383EDBB
:10441000010A01353046FAF7A3FA064638B1F8F733
:10442000EBFF104B03EB041383ED020A013530461A
:10443000FAF796FA28B9BDE87040FFF75DBA05466D
:10444000DBE7F8F7D9FF0748032D00EB041484EDF0
:10445000030AABD0EFE731460448BDE870400B22B9
:10446000FFF74EBA447C0020AFAC0608D5AD060875
:104470002DE9F043DFF8649085B080460D4616467E
:104480000227002446B336F8242035F82430F05BA8
:1044900093421FD1EB5B191A4B424B411946CDE9B0
:1044A000002023464A4640460391FFF73BF8039914
:1044B000EB5B019335F8243000934A46234640468F
:1044C0000134FFF715F8042C07F10407DAD105B021
:1044D000BDE8F0830023E1E73146E9E765AD060872
:1044E000F8B50446FFF714FA054628B1BDE8F840D0
:1044F000294900220120BBE728492046F8F71AFD88
:10450000A8B9274B4FF47A714FF4FA62A3F8AC1EA6
:10451000A3F8AE2EA3F8B01EA3F8B22EA3F8B41ED3
:10452000A3F8B62EA3F8B81EA3F8BA2EF8BD2046FD
:10453000F9F744F80328074627D82046FAF710FA77
:10454000044670B1F9F73AF8012506462046FAF715
:1045500007FA10B1F9F732F82DB9BDE8F840FFF7C6
:10456000CBB90546F2E7A6F2EE2240F2DC539A42BE
:10457000F3D8A0F2EE229A42EFD8094B03EB87035F
:10458000A3F8AC6EA3F8AE0ED0E729460548BDE807
:10459000F8400322FFF7B4B9047D0020AFAC060851
:1045A000586E002076AD06082DE9F04FDFF800A127
:1045B00091B0834691460C461546002604F1150835
:1045C0000422414609A84DF029FA00238DF828302D
:1045D000D4E90232082B72F100010BAF56D23049F8
:1045E0001A463846F8F7A8FAB9F1000F55D02B78DB
:1045F0000793079A237893424DD1D4E90202D5E973
:1046000002139A4208BF884245D1227D2B7D9A42EF
:1046100041D1042205F1150140464DF072F9002800
:1046200039D121692B69CB1A594259411D4B059348
:1046300000230493B5F912300393B5F910300293B7
:10464000194B0193079B00935246334658460791F6
:10465000FEF768FF079909AB0593237D0493B4F92E
:1046600012300393B4F91030CDE9017314F8203BF4
:1046700000935246334658460136FEF739FF082E5E
:1046800005F120059AD111B0BDE8F08F07493846F1
:10469000F8F752FAA8E70021C8E74946DBE700BF70
:1046A000F6EB06089AC40608FBDE06087EAD06088F
:1046B00089AD06082DE9F74F0446FFF729F90746AB
:1046C00030B170490022012003B0BDE8F04F6BE724
:1046D0006D492046F8F72EFC014638B969484FF479
:1046E000807203B0BDE8F04F4DF035B92046F8F7C1
:1046F00065FF83B2072B054600F2BB802046FAF720
:104700002FF9804600284CD0F8F758FF01240FFA03
:1047100080FB4046FAF724F968B14FF0000A411EC9
:1047200000F1100C564611F8013F13F0DF0F3BD19A
:1047300001270134E4B2FAF713F9804600284CD07F
:10474000F8F73CFF01340FFA80F9E4B24046FAF77B
:1047500007F90346002842D00190F8F72FFF0134F3
:10476000019B0FFA80F8E4B21846FAF7F9F803460D
:10477000002836D00190F8F721FF0134019B41B2A7
:10478000E4B218460191FAF7EBF80199024650B3EA
:104790000134E4B2032C28D803B0BDE8F04FFFF792
:1047A000ABB804468346B4E76145C2D0A3F13002FA
:1047B000D2B2092A05D9A3F16102052A07D8573BCD
:1047C000DAB2360146EA1A7642EA0A1AABE7A3F1F0
:1047D0004102052AADD8373BF2E78146B6E780466D
:1047E000C2E70146CDE7294AD4E71FFA8BF3022B33
:1047F000D2D809F226239BB2B3F5E16FCCD808F2E8
:1048000026239BB2B3F5E16FC6D8CCB2062CC3D831
:104810001046019246F056FC0428BDD8002FBBD0AC
:104820001B4B019A2DB203EB451103F56C6303EBAF
:104830004510C0E902A60346164D81F8C0BEA1F896
:10484000D09EA1F8D28E81F8D44E1533511E03327A
:1048500011F8010F445D04F00304022C08BF203856
:1048600003F8010B087808B18A42F1D103B0BDE822
:10487000F08F09480722394603B0BDE8F04FFFF733
:104880003FB800BF187D0020AFAC06089AC40608E8
:10489000586E0020B9030708AAAD06082DE9F047B5
:1048A000DFF874A086B0814690460D461746002674
:1048B000B8F1000F2ED03B782A789A42D7E9010C44
:1048C00026D16A68824223D1AC68A4EB0C02544220
:1048D0005441CDE9010C21460093524633464846E7
:1048E0000594FEF71FFE0599AB6802936B68019370
:1048F00015F80C3B00935246334648460136FEF706
:10490000F7FD082E07F10C07D2D106B0BDE8F087FD
:104910000024DEE74146E7E7B7AD06082DE9F84396
:104920000446FEF7F5FF054628B1BDE8F8432E49D9
:1049300000220120B2E72D492046F8F7FBFA014694
:1049400028B9BDE8F843284860224DF004B8204655
:10495000F8F734FEC3B2072B064606D92946244889
:10496000BDE8F8430722FEF7CBBF2046F9F7F8FF72
:10497000074628B3F8F722FE051E18BF01250124BB
:104980003846F9F7EDFF0746E0B1F8F717FE0134B6
:104990008046E4B23846F9F7E3FF0746A0B1F8F7DE
:1049A0000DFE01348146E4B23846F9F7D9FF08B16B
:1049B0000134E4B2032C09D0BDE8F843FEF79CBFF4
:1049C0000446DDE78046E5E78146EDE7094B76B230
:1049D0000C2000FB063686F8C05FC6F8C48FC6F808
:1049E000C89FBDE8F88300BF187E0020AFAC060862
:1049F000CCAD0608586E00202DE9F04FDFF8689026
:104A00008FB007468846164600240DF1240A58F850
:104A100024300293514602A842F056F816B356F8D5
:104A20002430029D0393EB1A5D420DF1100B5D41A2
:104A3000594603A842F048F8CDF800B023464A464C
:104A400029463846FEF76EFD2346CDF800A04A46BB
:104A5000294638460134FEF74BFD202CD7D10FB044
:104A6000BDE8F08F3546EFE7DBAD06082DE9F04FE6
:104A700089B00546FEF74CFF044630B16549002277
:104A8000012009B0BDE8F04FB6E72846F8F796FDDB
:104A90001F28074600F3B6802846F9F761FF5D4BF3
:104AA000019443F827405C4BCDE902430546A046FC
:104AB000A146A24626464FF0010B039B05AA13F818
:104AC00001CB039396460023284615F8011B19B124
:104AD0008C4501D00A2B0CD108AD2B448C454FF0EE
:104AE000000503F80C5C08D009B0BDE8F04FFEF7F4
:104AF00003BF0EF8011B0133E6E7731E451C032BB1
:104B000003D8DFE803F0243A687705A8F8F756FDE4
:104B100001900136F6B2052ECFD1029B3F4803F03B
:104B20000F0343EA844343EA8A5343EA092343EAEF
:104B30000838019B1B0100EB8707DBB248EA03033F
:104B400047F8D83C09B0BDE8F04F2AF089BC05A869
:104B5000F8F734FD0290DCE74E2B13D0452B13D031
:104B6000532B13D0572B13D0552B13D0442B04D1D8
:104B700005230BFA03F34AEA030A12F8013B002B60
:104B8000EAD1C6E70023F4E70123F2E70223F0E7C6
:104B90000323EEE70423ECE7DFF888C0002001469A
:104BA0001CF8010B984204D0072901F10100F6D14D
:104BB0004946542B14D04F2B14D0422B14D04E2BDB
:104BC00014D0492B14D0572B04D105230BFA03F32F
:104BD00048EA0308894612F8013B002BDCD198E72C
:104BE0000023F3E70123F1E70223EFE70323EDE7D7
:104BF0000423EBE705A8F8F7E1FC10280446A8BF5A
:104C0000002486E706481F22214609B0BDE8F04F80
:104C1000FEF776BE787E0020CF220608507F002067
:104C2000D5AD0608D42206082DE9F047DFF870A0BC
:104C300086B0814690460D4616460027B8F1000F13
:104C40002BD033882A889A4225D16C887188621AC1
:104C500054425441F2780292B2780594CDE9003280
:104C600021463B4652464846FEF75CFC0599EB78E8
:104C70000293AB78019335F8043B009352463B46D0
:104C800048460137FEF734FC102F06F10406D5D153
:104C900006B0BDE8F0870024DCE74146E7E700BF47
:104CA000E5AD06082DE9F8430546FEF731FE04465A
:104CB00028B1BDE8F843254900220120B4E7284681
:104CC000F8F77CFC0F28064630DC2846F9F748FE4A
:104CD00020361F4FDFF8848005464FEA86092846B4
:104CE000F8F76CFC37F8023B984226DC012C08EB05
:104CF000090311D0022C12D023F8D80C28462C21FD
:104D00004CF040FE054668B1013501230134A3B1E2
:104D1000032CE4D1BDE8F88303F8D60CEEE703F8E2
:104D2000D50CEBE7A21E53425341EFE72146094859
:104D3000BDE8F8430F22FEF7E3BD074B002243F81E
:104D40002620BDE8F843FEF7D7BD00BFF87E00205F
:104D5000DC220608D5AD0608787E0020507F0020B2
:104D60002DE9F04F14462A4A85B0064689460027A9
:104D70004FF0060B0BFB07F5C0354FF0000819F894
:104D800005A0002C40D0635DAAEB030041424141E5
:104D9000CDE9008330463B460391FEF7C3FB039900
:104DA0001B4ACDE9008A3B46304608F10108FEF770
:104DB0009FFBB8F1060F164A05F10105DFD1013757
:104DC000062FD7D1124FE42519F805A0A5F1E40864
:104DD000E4B1635DAAEB030251425141CDE9008386
:104DE0003A46062330460391FEF79CFB0399CDE932
:104DF000008A06233A4630460135FEF779FBEF2D4F
:104E0000E2D105B0BDE8F08F2146CAE72146EEE7C2
:104E1000F7AD060870B586B00346FEF779FD044687
:104E200030B11A490022012006B0BDE8704097E772
:104E30001749174E02AA18464CF033FD03AD80B156
:104E4000032C03D1FEF758FD06B070BDF8F7B6FB92
:104E500002AA45F8040B3146002001344CF021FD34
:104E6000EDE7032CEED1DDE90345059B01931A46DE
:104E70002946E0B22AF00EFC0028E3D0019B054849
:104E80002A462146FEF77EFBDEE700BF787E002043
:104E90008DAA0608F7AD06082DE9F043DFF89890D3
:104EA00087B0804617460C4615460026002F41D095
:104EB000B5F90030B4F90010B5F90220B5F90400D5
:104EC00095F906C0994233D1B4F9021091422FD11D
:104ED000B4F9041081422BD194F90610A1EB0C0E09
:104EE000DEF1000141EB0E01CDE90032CDE9020C0B
:104EF00033464A4640460591FEF714FB059994F95E
:104F000006300393B4F904300293B4F902300193EC
:104F100034F9083B00934A46334640460136FEF7D3
:104F2000E7FA102E05F10805C0D107B0BDE8F083FF
:104F30000021D9E73946E2E70BAE06087FB5054602
:104F4000FEF7E6FC00285BD02E490022012004B0C9
:104F5000BDE87040A0E72D2B03D0A3F13002092A51
:104F600049D8042C04DD04B0BDE87040FEF7C4BC91
:104F70002846F8F723FB04AB621C03EB440424F837
:104F80000C0C15F8013F303B092BFAD914462B784D
:104F9000002BE0D1052CE6D1BDF80430BDF904604A
:104FA0000F2BE0D8BDF90610A1F5FA7292B2B2F556
:104FB000FA6FD8D8BDF90820A2F5FA7080B2B0F522
:104FC000FA6FD0D8BDF90A008142CCDC8242CADB3C
:104FD0009142C8DCBDF90C5005F17D04A4B2FA2C55
:104FE000C1D8084B23F8361003EBC6035A809880CB
:104FF0009D7104B070BD202BB5D101352246C5E7A7
:105000000446C4E79C3D00202DE9F04FDFF8B8B01E
:105010008FB0804617460C4615460026A388ADF88B
:105020002C3023780893B4F90290637820680693B3
:10503000237994F905A00A900793B9F1000F3CD0A9
:10504000002F3FD02868BDF828100C9080B2AB88A4
:10505000ADF8343081422A7895F801C0B5F90230B4
:1050600095F804E02CD14B452AD1BDF82C10BDF8A1
:105070003400081A41424141CDE901C30092CDE913
:1050800003EA33465A4640460991FEF74BFA09991E
:10509000079BCDF810A0CDE90293069B0193089BD6
:1050A00000935A46334640460136FEF721FA202E39
:1050B00004F1060405F10605B0D10FB0BDE8F08F8C
:1050C0000021D9E73946E3E720AE0608F0B589B0FC
:1050D000044645F0F7FF10F0FF0205D12A490120F0
:1050E00009B0BDE8F0408FE7284905222046F7F7D0
:1050F00005FF30B92448152109B0BDE8F04045F05E
:105100006BBB20462249224E01AA4CF0CAFB4FF04D
:10511000FF33079302AD002478B1062C02D1FEF7CD
:10512000EBFB2EE0F8F74AFA01AA45F8040B3146EA
:10513000002001344CF0B5FBEEE7042CEFDD029EBD
:105140001F2EECD8039D0F2DE9D8049C252CE6D802
:10515000059800F57A73B3F5FA6FE0D80699FF2940
:10516000DDD8079A531C402BD9D80A4B062707FBDA
:10517000063358831D7608485C7619775A77FFF70F
:10518000A5FF09B0F0BD00BF687F0020AFAC0608E6
:105190008DAA0608507F00209AC4060810B5114B4E
:1051A000014603F1180253F8044B41F8044B9342B3
:1051B000F9D11B880B800B4900F11A0351F8044BFD
:1051C00043F8044B9142F9D111881980054B3430D2
:1051D00053F8041B40F8041B9342F9D11B88038049
:1051E00010BD00BF1C3C06084F4B2DE9F04F1D7849
:1051F000854203D020B985F001051D70BDE8F08F10
:105200004A495A7CD1F80080CAB1A8F51C575968A0
:10521000103F4FF0640AB94216D30A2A71D04448AD
:105220005960A8EB0101A0FB0101C1F347115A74B9
:105230000029E0D098180132C1715A74DBE70122CD
:105240005A74C3F80480D6E7012A01D14146E2E747
:1052500093F808C0961E1AFB0C11B146002E4DD0D3
:10526000D01E02284FF000002CD96CF307006CF31D
:105270000F20D3F809406CF317406CF31F6084EAE9
:10528000000E00F07F3B6FEA0E0E44F080340EF00B
:10529000803EA4EB0B048EEA04049C60B408012C4D
:1052A0000CD0D3F80D406040C04344F08034A4EBF0
:1052B0000B0B00F0803080EA0B00D860B40726F0BA
:1052C00003001BD0461C03EB060E03EB000B9EF8FD
:1052D00008404E45A4EB0C048BF808400EDA02306F
:1052E0001E188145347AA4EB0C048EF8084005DDC5
:1052F0009BF80B00A0EB0C0C86F808C0013AD2B268
:1053000089E7187C63288AD808480068A0F51C50F3
:105310001038884283D893F808C04FF008091AFB68
:105320000C114E469CE700BF888400201426002004
:105330001F85EB51F8B5204C237D05460E463BB149
:10534000D4E90623904271EB030324BF00232375A5
:105350001A4FFB693846984710F0010325D0D7E96A
:1053600004315B19A3614FF0010346EB010684F899
:10537000203080F00203E661C3F340032375430746
:10538000A06A48BF0123A5EB000548BF84F821307F
:10539000002D03DD012084F82000F8BD94F82000E2
:1053A0000028FAD194F82100F8BD8207E7D5227DC4
:1053B000002AE4D0E2E700BF8884002040410020BA
:1053C0002DE9F04FDFF808A19DB0804617460C4646
:1053D00015460026A646BEE80F000DF1400CACE8CD
:1053E0000F0023780C939EE8030094F901300D938D
:1053F000A3780E93237B94F804B094F81490099248
:105400008CE803000A930B90002F5FD0AE46BEE8F5
:105410000F000DF1580CACE80F009EE80300109B44
:105420000F928CE8030023F07F4C169B95F804E064
:10543000287B2A69297D23F07F439C4544D1F3458D
:1054400042D1099B9C460F9B9C453DD10A9B8342C0
:105450003AD10B9B934237D1A9EB010359425941F1
:105460000B9B06930A9B0593099BCDF81C90CDE9F5
:1054700003B30E9B02930D9B01930C9B009352462A
:10548000334640460F91FEF74DF80F990B9B06935C
:105490000A9B0593099BCDF81C90CDE903B30E9BA5
:1054A00002930D9B01930C9B00935246334640465A
:1054B0000136FEF71DF8402E04F1180405F1180519
:1054C00088D11DB0BDE8F08F0021C9E73946DDE77E
:1054D00037AE06082DE9F04F164615461C4A87B030
:1054E00007460C464FF0000BD4E9009AD4F8088028
:1054F00066B3AB689845D5E9000125D1814523D134
:10550000AAEB010359425941CDE9019ACDF8008037
:105510005B4638460591FEF705F805990C4ACDF82B
:1055200000805B46CDE9019A38460BF1010BFDF78F
:10553000DFFFBBF1080F064A04F10C0405F10C056E
:10554000D2D107B0BDE8F08F0021DDE73146E6E7B4
:1055500058AE06082DE9F04FDFF804B1A1B080463F
:1055600017460C4615460026A646BEE80F000DF16C
:10557000480CACE80F0023790A93A3680B939EE8CC
:105580000700A38A0D93E38A0E93238B0F93638BFB
:1055900094F800A094F80C900C908CE807001093FD
:1055A000002F5BD0AE46BEE80F000DF1640CACE8F6
:1055B0000F009EE807002B7853458CE807004BD17D
:1055C0002B790A9A934247D1AB680B9A9A4243D1FE
:1055D0002B7B4B4540D10C9A82423DD1179A8A428F
:1055E0003AD118991F9BCB1A59425941109B0893E5
:1055F0000F9B07930E9B06930D9B05930C9B11919C
:10560000CDE903930B9B02930A9B5A46CDE900A375
:1056100040463346FDF786FF1199109B08930F9B78
:1056200007930E9B06930D9B05930C9BCDE903936B
:105630000B9B02930A9B5A46CDE900A34046334692
:105640000136FDF755FF042E04F11C0405F11C057D
:105650008AD121B0BDE8F08F0021C7E73946DCE7E9
:1056600069AE06082DE9F0418AB0044645F02AFDEE
:1056700010F0FF0205D1384901200AB0BDE8F04121
:105680009EE6364905222046F7F738FC38B93248FD
:105690004FF47E710AB0BDE8F04145F09DB8204658
:1056A0002F492F4E6A464CF0FCF801AD002478B12A
:1056B000092C02D1FEF720F94BE0F7F77FFF6A468D
:1056C00045F8040B3146002001344CF0EAF8EEE7CF
:1056D000092CEFD1DDF804E0BEF13F0FEAD8DDF888
:1056E00008C0BCF1010FE5D8039F7B1C402BE1D81B
:1056F000049E2E2EDED8059D062DDBD8069C194B68
:1057000004F5742202F510729A42D3D8079806283D
:10571000D0D8089901F5742202F510729A42C9D8BE
:10572000099AFF2AC6D8104B4FF0180808FB0E3311
:1057300083F83C0083F830C00C4883F8317083F85C
:10574000326083F834509C63196483F84420FFF777
:1057500089FF0AB0BDE8F081B8840020AFAC06082C
:105760008DAA060880841E00888400209AC406083A
:1057700070B586B0044645F0A5FC10F0FF0205D1D7
:105780002149012006B0BDE87040A3E61F4905226B
:105790002046F7F7B3FB38B91B4840F2FF3106B09B
:1057A000BDE8704045F018B820461949184E01AAC6
:1057B0004CF077F802AD002478B1042C02D1FEF74A
:1057C0009BF81FE0F7F7FAFE01AA45F8040B3146F3
:1057D000002001344CF065F8EEE7042CEFD1029A7A
:1057E000072AECD80B4B0C480C2101FB0233039A1F
:1057F000C3F83826049AC3F83026059AC3F834262D
:10580000FFF7B6FF06B070BDB88A0020AFAC06083F
:105810008DAA0608888400209AC406082DE9F04362
:105820008DB0044645F04EFC10F0FF0205D13E4914
:1058300001200DB0BDE8F0438CE63C49052220462E
:10584000F7F75CFB38B938484FF47E710DB0BDE80E
:10585000F04344F0C1BF20463549354E01AA4CF013
:1058600020F802AD002478B10A2C02D1FEF744F8EA
:1058700057E0F7F7A3FE01AA45F8040B31460020D4
:1058800001344CF00EF8EEE70A2CEFD1DDF8088079
:10589000B8F1030FEAD8DDF80CE0BEF1010FE5D84E
:1058A000DDF810C0BCF1060FE0D8059F214B07F5CD
:1058B000742202F510729A42D8D8069E062ED5D8C8
:1058C000079D05F5742202F510729A42CED8089C05
:1058D000B4F5004FCAD20998B0F5004FC6D20A9964
:1058E000B1F5004FC2D20B9AB2F5004FBED2124BA7
:1058F0004FF01C0909FB0833A3F8A60683F890E6CD
:105900000E4883F894C6C3F8987683F89C66C3F86B
:10591000A056A3F8A446A3F8A816A3F8AA26FFF752
:105920007DFF0DB0BDE8F083188B0020AFAC0608FA
:105930008DAA060880841E00888400209AC4060868
:1059400037B505460846019145F0BCFB0199044670
:1059500002462846F7F7D2FA68B92B5DA3F1300268
:10596000092A06D923F02003413B192B01D9013420
:10597000281903B030BD0020FBE72DE9F347374974
:10598000DFF8D89001AA4BF08CFF4FF0000A4FF0DF
:10599000FF3557465446D0462E4668B9BAF1040F33
:1059A00050D03ADCBAF1020F13DC2D492B463246B7
:1059B000012041F0B9F90EE0BAF1040F09D8DFE88F
:1059C0000AF0030D12171C00F7F7F8FD064603282E
:1059D0001BD9FDF791FF02B0BDE8F087F7F7EEFDA8
:1059E00005468728F4E7F7F7E9FD80463F28EFE70B
:1059F000F7F7E4FD04463F28EAE70378482B03D095
:105A0000562BE6D1012700E0002701AA49460020D5
:105A10000AF1010A4BF045FFBFE7BAF1050FD8D1F3
:105A2000882303FB0655A4010E4E04F47C6408F0A1
:105A30003F0844EA080406EB450544EA4734A5F864
:105A40000047C8E7882303FB0652064B03EB4203DB
:105A5000B3F80077C7F34037E2E700BF8DAA060826
:105A6000888B0020888400201FB5094B0293094BC6
:105A70000193094B0093094A094B0A490A48FDF76B
:105A800081FD0A490A4805B05DF804EBFDF77ABDCF
:105A900039A8060842A806084BA806085DA806080B
:105AA00057A8060805A806088BAE0608A3AE060888
:105AB000BDAE0608F8B50C480C4D0D4E0D4FFDF768
:105AC00061FD00246CB93268C2F50072920022B107
:105AD00057F824100848FDF755FD0134252CF1D165
:105AE000F8BD55F82420F2E7C6AE0608C4380020F9
:105AF000C0300020383C0608DCAE06082DE9F84F1F
:105B0000054645F0DFFADFF8EC800446D8F800904F
:105B1000C0B93048304D314FFDF770FC012655F8C3
:105B2000041B59B10B783BB106FA04F313EA090FD1
:105B300002D03846FDF70CFD0134F0E7BDE8F84F20
:105B4000FDF78ABC024626492846F7F7D7F978B907
:105B50002448214C214DFDF751FC54F8041B002929
:105B6000ECD00B78002BF8D02846FDF7F1FCF4E7D9
:105B70002B78DFF864B02D2B03BF013504F1FF341F
:105B80004FF0010A4FF0000A00265BF8047B1FB9B2
:105B9000BDE8F84F41F028B8224639462846F7F7C5
:105BA000ADF9A8B90120B040BAF1000F0AD0F7F75B
:105BB000A3FD0D48FDF722FC39460C48BDE8F84F1F
:105BC000FDF7E0BC40EA0900C8F800000848F1E72A
:105BD0000136DAE7EAAE0608CC3C0608F5FC060812
:105BE0009ABC0608F4AE060800AF06082FAF0608F8
:105BF00009AF0608643900202DE9F84F054645F045
:105C000061FA334F0446BE68C8B93248324DDFF8F6
:105C1000D880FDF7F3FB0127E3B205EB8302D2F84E
:105C2000341141B107FA03F3334202D04046FDF785
:105C30008FFC0134F0E7BDE8F84FFDF70DBC0246DC
:105C400026492846F7F75AF960B92548254C264DCC
:105C5000FDF7D4FB54F8041B0029ECD02846FDF7CF
:105C600077FCF7E72B78DFF87CB02D2B03BF0135ED
:105C700004F1FF344FF0010A4FF0000A4FF0000921
:105C80005BF8048BB8F1000F03D1BDE8F84F40F08A
:105C9000ABBF224641462846F7F730F9A8B90123A1
:105CA00003FA09F3BAF1000F0BD026EA03030F48F9
:105CB000BB60FDF7A3FB41460D48BDE8F84FFDF77B
:105CC00061BC33430B48BB60F3E709F10109D7E737
:105CD000EC460020EAAE06081C3C06089ABC060802
:105CE000F4AE0608503D0608F5FC060800AF0608AD
:105CF0002FAF060809AF0608F8B50C4C0C4E0D4F37
:105D00002D252068FDF77AFB616811B13046FDF75B
:105D10001FFCA16811B13846FDF71AFCFDF79CFB8A
:105D2000013D04F11004ECD1F8BD00BF783D060838
:105D300011AF060817AF06082DE9F047814645F078
:105D4000C1F94D4E0446376800BB4C484C4D4D4E92
:105D5000FDF7FEFB4FF00C0808FB04F35B5D5A1ED9
:105D6000012393403B4206D0204619F03BFB0146FD
:105D70003046FDF7EDFB0134182CEDD117B9424840
:105D8000FDF73CFBBDE8F047FDF766BB02463F4927
:105D90004846F7F7B3F8054678B93D48FDF72EFBBE
:105DA0002C46384D204619F01DFB0134014628468B
:105DB000FDF7CEFB1A2CF5D1E4E799F800302D2B36
:105DC00003BF09F1010904F1FF344FF0010A4FF05C
:105DD000000A4FF00008404619F004FB2246054631
:105DE00001464846F7F78AF800283BD1BAF1000F80
:105DF0001FD0B8F1180F0BD16FF07F4333602548E7
:105E0000FDF7FCFA29462448BDE8F047FDF7BABB88
:105E1000B8F1190F01D17368F0E7204B0C2202FB97
:105E2000083898F82C345A1E012393401F433760DA
:105E3000E5E7B8F1180F03D1C6F800A01848DFE76E
:105E4000B8F1190F01D17760F8E7144B0C2202FB6F
:105E5000083898F82C345A1E0123934027EA030788
:105E60003760EBE708F10108B8F11A0FB3D1BDE8CC
:105E7000F04740F0B9BE00BF143F00201DAF060838
:105E8000484006082EAF060827AF06089ABC060849
:105E900033AF060800AF06082FAF06081C3C060803
:105EA00009AF0608F0B585B0044645F00BF90428A3
:105EB0003DD1631E2546E11C13F8012FA2F16100BC
:105EC000192898BF203A8B421A70F5D11A4F261D17
:105ED00015F8011B019138464BF054FD20B1019992
:105EE00028464BF04FFD20B105B0BDE8F040FDF76E
:105EF00003BDB542ECD120461EF020FC0F48104CEB
:105F0000FDF77CFA0C4901231A5D11F8010B04AD71
:105F10002A440133052B02F8080CF5D10023094867
:105F20008DF80C3002A9FDF72DFB05B0F0BD00285F
:105F3000E4D0FDF7E1FCE1E7804106083EAF06084A
:105F40003C3C00201AAF06087FB5184B1A78012A8E
:105F500028D15B790D2B05D0154807B05DF804EB0F
:105F6000FDF74CBA1122002101A84BF0F4FCA62346
:105F70008DF8003041238DF80130EB238DF803308C
:105F80000C4B1B788DF80430B22315218DF80530A9
:105F9000684603238DF802108DF806301EF0C3FD0D
:105FA0000548DAE707B05DF804FB00BF3C3C002081
:105FB00044AF0608C009002053AF060810B5204CB6
:105FC0002048A17AFDF7DEFA1F48FDF76BFAA179A8
:105FD0001E48FDF7D7FAE1791D48FDF7D3FA217A7B
:105FE0001C48FDF7CFFA617A1B481C4CFDF7CAFA32
:105FF0001B48FDF757FAB4F91030B4F90E20B4F984
:106000000C101848FDF7BEFAB4F91C30B4F91A2088
:10601000B4F918101448FDF7B5FAB4F91420B4F91E
:106020001210B4F916301148FDF7ACFAB4F920207B
:10603000B4F91E100E48BDE81040FDF7A3BA00BF2A
:10604000B80101206DAF060886AF06089AAF0608B2
:10605000A2AF0608ABAF0608B3AF0608CC480020D5
:10606000BBAF0608CEAF0608DDAF0608EBAF0608EB
:10607000F9AF060808B51F4B1F4C1D68A06819F042
:10608000A7FD284619F0A4FDA06841798B0704D428
:10609000036841F002019B69984700210846F9F71F
:1060A00091FC00210120F9F78DFCA068FAF7A5FB0F
:1060B00070B101210020F9F785FCA068FAF7BEFB5A
:1060C00001462846FAF731FB00210846F9F77AFC29
:1060D0002846FAF792FB0028E7D001210846F9F795
:1060E00071FC2846FAF7AAFB0146A068FAF71DFBE7
:1060F000D7E700BFC47B0020983F0020F7B50546D6
:10610000FDF706FC044620B103B0BDE8F040FDF702
:10611000F3BB28461D491D4F01AA4BF0C2FB264682
:10612000254640B90B2D18D9014619480B22FDF719
:10613000E7FB03B0F0BD44B1012C0AD001AA3946F7
:10614000002001344BF0ADFBEBE7F7F737FA0546DB
:10615000F4E7F7F733FA0646F0E7022C0DD1A6F57F
:106160007A73B3F57A7F05D90A484FF4FA624FF48F
:106170007A71DCE7084B23F81560074B074833F9C1
:1061800015202946FDF7FEF9D3E700BF8DAA0608C2
:10619000D5AD060843BB0608E811012007B0060884
:1061A00070B50446FDF7B4FBC0B11F4B5E68013605
:1061B000304619F017F934460546E8B901341A2C6F
:1061C000A8BF0024204619F00DF90546A0B9B44235
:1061D000F4D1BDE870401548FDF764B92046F7F7E3
:1061E000EDF9044619F0FEF8054628B92146104895
:1061F000BDE87040FDF7C6B90B4B5C6019F0AEFF0F
:106200000C4821462A46FDF7BDF9192C9DBF0A48C6
:106210000C2101FB04000020BDE8704098BF90F8FD
:106220002C0419F0B7BF00BFC009002014B0060845
:1062300028B006083EB006081C3C060838B51749C9
:10624000052204464BF0B4FB58B9154A13781BB924
:1062500001211170134A1370BDE838401248FDF750
:1062600021B91249032220464BF0A2FB80B90C4D04
:106270000C4C2B7843B1237833B10D48FDF78FF9DF
:1062800000232B70237038BD0A48FDF70BF9F7E7A0
:10629000BDE838400848FDF782B900BF60B5060880
:1062A000C07B0020C17B002053B00608F8B606086A
:1062B00069B00608A0B00608B4B006082DE9F0439E
:1062C0004C498DB0F6F736FE044600284BD14A4DB6
:1062D0002B78012B4BD1FCF715FD4848162306AA55
:1062E00055210068FAF776FD0C20FCF70BFD2046DF
:1062F00001AB1C18C3B29A1DD2B20CA9CE1802333E
:1063000016F8177C16F8181CDBB241EA07219342F5
:1063100024F8021BF1D106301228E9D1BDF92A6018
:10632000BDF92C40BDF90490BDF90680BDF908E027
:10633000BDF90AC0BDF90C70BDF90E00BDF9101011
:10634000BDF91220BDF91430A5F81890A5F81A80EF
:10635000A5F81CE0A5F812C0AF82E882A981EA8105
:106360002B82EE832C840DB0BDE8F04326E6022B91
:10637000F9D101463D20FAF709FA1920FCF76DFC26
:1063800016215520FAF70CFA3220FCF766FC1C4A5D
:10639000204607AB1E18C3B2991DC9B2D41867783E
:1063A000D45C0233DBB244EA07248B4226F8024B6A
:1063B000F4D106301228ECD10C213D20B2F9126044
:1063C000B2F91440FAF7E2F91920FCF746FCBDF9DE
:1063D0001C90BDF91E80BDF920E0BDF922C0BDF9B9
:1063E0002470BDF92600BDF92810BDF92A20BDF999
:1063F0002C30A9E7C3B00608CC480020F0480020A4
:10640000D55E00202DE9F0478CB0074610F8013B1F
:10641000202BFAD00025204CDFF88480DFF8849010
:10642000DFF884A02E4601A920460EF08DFC3946E7
:1064300001A84BF016FBE0B101A94046FDF788F832
:10644000494601A844F034FE00BB20460EF04AFD48
:10645000124B0146007820280CBF50461846FDF725
:1064600077F8FCF7F9FF2046FDF7EEF9FCF7F4FFAB
:106470000136013540F246239D4204F10B04D2D18E
:106480000EB940F0B1FB0CB0BDE8F087002120460A
:10649000FDF7CEF9E5E700BF182306081AAF060896
:1064A0005FAB060857FE060865AB06082DE9F04FFE
:1064B0002DED028B8DB00678202E054600F10100EF
:1064C000F9D0284644F0FEFD044618B1012822D137
:1064D0002A2E20D18248834DDFF81C82FCF7E2FF90
:1064E000002640F24627284601A90EF02DFC01A9FE
:1064F0004046FDF72DF8013628462146FDF798F96C
:10650000FCF7AAFFBE4205F10B05ECD10DB0BDECC6
:10651000028BBDE8F08F3D2128464BF033FA00286E
:1065200000F0D6800346984613F8012D202AFAD0B1
:10653000A8EB05080130064610F8013B202BFAD0E5
:10654000684F4FF000095FFA88F840F2462B01A926
:1065500038460EF0F9FB01A844F0B4FD01A902464B
:1065600082462846F6F7CAFC5E4B044610BBC2457D
:1065700020D10B2202FB09339B7903F00F08B8F1FD
:10658000060F22D1584901A844F092FD0446304636
:1065900044F098FD0246B4B93378222B13D1331856
:1065A00013F8013C222B0ED1821E711C38460EF0CE
:1065B00065FDABE709F10109D94507F10B07C6D124
:1065C00040F012FBA2E73146F0E713F0C0030AD017
:1065D000402B4DD04548FCF76BFF3846FDF734F9AA
:1065E000FCF73AFF92E73378002BF3D0404930466E
:1065F0004BF027FA0446304644F064FD8442E9D16A
:106600003046F6F7F9FE3846B0EE408A0EF077FCD9
:1066100007EE900AF8EEE77AF4EEC87AF1EE10FA97
:10662000D8D838460EF07CFC07EE900AF8EE677A70
:10663000F4EEC87AF1EE10FACCDBB8F1050F0CD10C
:1066400018EE104A38460EF04DFCB8F1050F30D860
:10665000DFE808F02E2E38383A3CB8F1040F304607
:1066600003D1F6F791FF0446ECE7F6F7A7FFFAE748
:1066700038460EF0E7FC90F804B0814625462346E4
:10668000A246AB4500D91BB1BAF1000FA2D0D9E7A1
:10669000D9F80030314653F82500F6F74BFC0028B6
:1066A00005BF2C46012300234FF0010A0135E8E71E
:1066B000047001A90F48FCF74BFF00213846FDF795
:1066C000B7F823E70480F4E70460F2E70460F0E73A
:1066D00028460DB0BDEC028BBDE8F04F92E600BF3E
:1066E000C9B006081823060857FE0608F4B00608C5
:1066F000DBB00608E9B006085FAB06082DE9F04FED
:10670000BE4BBF481968BF4EBF4CDFF83893A7B0E7
:106710004FF47A73B1FBF3F1FCF734FF0BA8F6F7F3
:1067200009FDB6F9402B0BA91BA843F007F81BA9DC
:10673000B648FCF727FF1FF0DFFCB54B1B7804EBD6
:1067400083036422D3F86C350093B24BB0FBF2F1B3
:1067500002FB11021B78B04892B289B2FCF712FF1B
:10676000AE4BAF481968AF4BB1FBF3F1FCF7F0FE4D
:10677000AD4B1F68002504F27C5804F5B36A012371
:10678000AB403B420DD059060BD058F8253043B1F1
:1067900019F805205AF8251053F82220A348FCF7D1
:1067A000D7FE0135082DEAD1FCF756FEA0489D4DD5
:1067B000FCF778FE0EA8F3F751FC0E999D48B1FB4B
:1067C000F5F1FCF7DFFE0F999B48B1FBF5F1FCF703
:1067D000D9FE10999948B1FBF5F1FCF7D3FE119958
:1067E0009748B1FBF5F1FCF7CDFE964B1B78002BDB
:1067F00014BF0123022304EB8303D3F8C0150991CE
:106800001FF008FF04EB8000D0F8C02508921FF0AD
:1068100017FF04EB8000D0F8C03507931FF026FF68
:1068200004EB8000D0F8C0951FF030FF05461FF044
:106830007DFF07461FF062FF804618F0BDFD04EBA8
:10684000800004EB8808D0F8C005049004EB8707AB
:10685000D8F8C005039004EB8505D7F8C005029071
:10686000D5F8C0050999DDE90732CDE900907648F1
:10687000FCF788FE754B1B68DA031AD510F06CF82C
:106880000546B0B101467248DFF81C82DFF81C9261
:10689000FCF778FE0027B8F9022039464846013750
:1068A000FCF756FEFBB29D4208F11008F3D8FCF746
:1068B000D3FD684B684A1D88684B69491B68694865
:1068C000DFF8EC91DFF8EC81674FDFF8ECB1DFF82F
:1068D000ECA1C3F500739B00FCF754FE634A644BC4
:1068E0006448D31A644AADB229461288FCF74AFEBE
:1068F0006248FCF7D7FD002559F8041B6048FCF7F7
:1069000027FE5846FCF77AFD18F8011B002940F0D5
:1069100010815C48FCF772FD5B48FCF76FFD57F88F
:10692000041B002940F009815648FCF7BBFD0135E6
:10693000042DE1D1554B5648198BFCF709FE012077
:106940001EF034FB054658B107EE900ADFED516AA0
:10695000F8EEE77A86EEA77AFDEEC77A17EE905A40
:1069600003201EF023FB034658B107EE900ADFED2B
:10697000496AF8EEE77A86EEA77AFDEEC77A17EE57
:10698000903A002007931EF011FB079B58B107EEC9
:10699000900ADFED406AF8EEE77A86EEA77AFDEE20
:1069A000C77A17EE900A0090B6F8441B3A483B4E5F
:1069B000DFF80C812A46FCF7E5FD3948FCF71EFD9F
:1069C000356825F0004525F07F050127002D40F0B2
:1069D000B880FCF741FD33685B017CD512A80EF04E
:1069E000B5FA002877D1129B40F2452293429EBF10
:1069F0002C480B2505FB030064E000BF1426002093
:106A000004B10608888400201C3C06081EB1060854
:106A10005C4800205D4800202FB10608C00500201A
:106A200054B1060840420F00B401012064B10608C9
:106A30006CB1060881B1060893B10608A5B1060835
:106A4000B7B10608F4480020C9B10608B00101201A
:106A500025B20608082E002000000220C0300020C9
:106A60000018000059B20608605D00200080000890
:106A70000040000891B2060860390020CBB2060839
:106A8000DEB2060829AF0608FCB20608E8110120AC
:106A900006B306080024744916B30608A8010120AD
:106AA00053B30608182306084C3E00204AB20608D5
:106AB000EC410608203F0020E6B20608F5B20608C1
:106AC0002FAF060888BF28461BA90EF03DF92848BD
:106AD0001BA9FCF764FD274D2748FCF78FFC2868AD
:106AE000FCF72FFC00283FD012A92868FCF76AFCAD
:106AF0009DF85C109DF86830199A2048FCF728FD35
:106B0000169911B11E48FCF723FD149911B11D48C7
:106B1000FCF71EFDFCF7A0FC1B4B1B7833B104EB0C
:106B200083041A48D4F83C16FCF72CFD27B0BDE8C6
:106B3000F08F5046FCF70CFDEEE65046FCF722FDC8
:106B4000F5E695FAA5F3B3FA83F307FA03F2062BF9
:106B500025EA02057FF73AAF04EB83034046D3F8FA
:106B6000C415FCF7F5FC31E70948FCF747FCD1E711
:106B70006AB30608E44700207EB3060884B306081B
:106B8000A2B30608ABB30608343E0020C7B306081C
:106B9000BAB306082DE9F04F2DED028B43489FED67
:106BA000448A95B0FCF7EEFC00252F46A84608A9BC
:106BB000E8B21EF073F99DF82430002B54D0129CDB
:106BC0004CB107EE904AB8EEE77AC8EE077AFDEED0
:106BD000E77A17EE904ADDF830900D9B4FEAE47BA0
:106BE00009FB0BF1A9FB040604FB031141F28833F6
:106BF000C01841EB06014FF47A72002345F0A4F867
:106C0000DDE910A1614306460AFB0B1B41F2883304
:106C1000A4FB0A01C0184FF47A724FF000034BEB4B
:106C2000010145F091F8042D4FF47A720E9BB3FBED
:106C3000F2F306934FF00A0318BF3F1890FBF3F2EC
:106C400003FB1200CDE9042096FBF3F218BFB04419
:106C500003FB1266CDE90226CDE9009A089A154891
:106C600023462946FCF78EFC01351B2D9FD108A831
:106C70001EF000F90A9A08990F484FF47A73B2FB94
:106C8000F3F30C9AFCF77EFC0A2297FBF2F302FB6B
:106C9000137798FBF2F10948009702FB1182FCF789
:106CA00071FC15B0BDEC028BBDE8F08FE1B30608B6
:106CB0000024744928B406085DB406087FB40608A9
:106CC0002DE9FF471B481C4C1C4E1D4FDFF87480FC
:106CD000FCF758FC0025A379E27994F808A006EBAC
:106CE000830306EB8202DB69D2F8549603932046B5
:106CF000F8F7EFF800F1410120460291F8F7F4F8B7
:106D0000DDE902130246BAF1000F0CD0CDE900A96B
:106D10004046FCF737FC0135312D04F10C04DAD183
:106D200004B0BDE8F087CDF800903846FCF72AFCA7
:106D3000F1E700BFADB40608683900201C3C060826
:106D4000D9B40608C9B406082DE9F84FCA4D6B79C5
:106D50002DED028B002B3ED095F82830C74A03EB6F
:106D6000430002EB4000590090F8A606002800F00E
:106D70000482012800F0E081C81802EB400090F87E
:106D8000A706002800F0E381012802D1BC480024B6
:106D9000C483C81802EB400090F8A806002800F051
:106DA000C882012802D1B648002404840B4402EBB7
:106DB000430292F8A936002B00F0BE82012B40F06E
:106DC0001081B04B1B68D90440F1C78240F2DC50FF
:106DD000AB4B588405E1AA4CDFF8D4B2A36A13F494
:106DE000807F03F4807AB0EE408ABBF9023040F035
:106DF000EE81A54ED4F8C070D6F8488B96F84C0BAF
:106E000017F48079A3F2DC5214BF98F80DC098F8FB
:106E100008C012F5FA7FC0F29D81B2F5FA7F00F347
:106E2000AF8111B20029B8BF494289B2884240F30C
:106E300098829FED960A47F067FBA083BAF1000F96
:106E400040F09181BBF90A30B9F1000F00F00681E2
:106E5000A3F2DC5212F5FA7F98F80DC096F84C0BAD
:106E6000C0F20681B2F5FA7F40F3C7804FF4FA72A0
:106E700007EE90CADFED865A9FED860A9FED866A7F
:106E8000F8EE676A131ABBEE097A4FF4FA72C0F58E
:106E9000FA7002FB03F393FBF0F31BB207EE903A98
:106EA000F8EEE77A67EEA57AA7EEA77A67EE867A1C
:106EB000A7EE260A27EE800A47F026FBE083BBF9FF
:106EC0001200BAF1000F40F0AB80B9F1000F00F0F2
:106ED000B280A0F2DC5313F5FA7F98F80EC096F852
:106EE0004D1BC0F2B280B3F5FA7F00F378811AB27D
:106EF000002AB8BF524292B2914240F389829FED7C
:106F0000630A47F001FB404200B22084B9F1000F50
:106F100000F0D08098F8113098F80FC0A28B5F492C
:106F200013FB00F01CFB02F2E38B98F810C01CFB73
:106F300003F381FB00C8C017C0EB681881FB02C0D7
:106F4000D217C2EB6012A28381FB0321DB170FFA79
:106F500088F8C3EB6113A4F82080E38303201DF0BD
:106F60000DFC4F4BB3F810904FF4FA624946F4F71A
:106F700097FFA0EB090080B24FF47A72C9F5FA6965
:106F800000FB02F292FBF9F291B2B1F57A7F80F048
:106F90004D814248A0FB0131490904EB410392B203
:106FA000B3F9C4C0B3F9C6306FF0630EA3EB0C03A2
:106FB0000EFB012203FB02F280FB0230D317C3EB6E
:106FC000601363449BB22A791BB2638432B968F3BD
:106FD0000F0263F31F42E3692A63EB627A0600F152
:106FE0002881304B1B685B0732D5BDEC028B2E48E5
:106FF000BDE8F84F0021F8F77EB811B20029B8BFFC
:10700000494289B2884240F32C829FED200A47F022
:107010007BFAE083BBF91200BAF1000F3FF455AFE1
:1070200094F84030002B3FF450AFB4F94400B9F16C
:10703000000F7FF44EAFA0F2DC5313F5FA7F98F8FF
:1070400009C096F84D1BBFF64EAF9FED180A58E7E2
:10705000BDEC028BBDE8F84F0AF0A8BCA3F2DC52ED
:1070600012F5FA7F98F808C096F84C0BBFF6FAAE06
:107070009FED0E0ACBE700BFF84000201C3C06083D
:10708000E8110120AC0101208884002000000000EC
:107090000AD7233C00401C450AD7233D1F85EB51EE
:1070A0003C3C0020A8010120843B0020FFFFF9C3E5
:1070B00074410020C04FB4F91C003B78222B08BF5C
:1070C000BE4BB0EE480A08BF186000210FF034FB39
:1070D0003B78222B08BFB94B00B208BF5860A08391
:1070E00006BFB4F91E009860B4F91E00B0EE480A5D
:1070F00001210FF021FB3B78222B08BFAF4B00B2E0
:1071000008BFD860E08306BFB4F920001861B4F965
:107110002000B0EE480A02210FF00EFB3B78D4F8B5
:10712000C070222B08BFA54B0FFA80F8A4F820806E
:1071300008BFC3F8148011E7A14800248483C8184D
:1071400002EB400090F8A70600287FF41DAE9C4893
:10715000EC8D1DE69FED9B0A47F0D6F9A083BAF1AE
:10716000000F3FF46FAE94F83820BBF90A30002AC4
:107170003FF46AAEB4F93C3066E69148AC8DDDE789
:107180004FF4FA72131A4FF4FA72C0F5FA7002FB58
:1071900003F393FBF0F31BB207EE103ADFED995ABD
:1071A0009FED9A0AB8EEC77AFBEE096A27EE257AB8
:1071B00007EE90CAE7EE076AB8EE676ADFED927AEB
:1071C000E6EE867A27EE007A27EE870A33E694F811
:1071D0003020002A3FF40DAEB4F9343009E64FF404
:1071E000FA735B1A4FF4FA72C1F5FA7102FB03F3FA
:1071F00093FBF1F31BB207EE103ADFED825A9FEDDD
:10720000830AB8EEC77A07EE90CA27EE257ABBEE5E
:10721000096AA7EE076AF8EE676A27EE007ADFEDE3
:107220007A7AE6EE267A27EE270A6AE6664B1B880C
:10723000C9E6B4F9E030654ADD1782FB0323B6F8EE
:10724000582BC5EBA305AD1A2DB207EE905AB8EE38
:10725000E78ADFED5F7A28EE278AB0EE480AF4F776
:1072600063FBFDEEC87A17EE903A2033402B67D8C7
:10727000B42D0CDDDFED576A9FED577AF0EE487ABA
:10728000F4EEC77AF1EE10FA38EE668AF6DCDFED3E
:10729000537AB4EEE78AF1EE10FA0CD5DFED4D6AC1
:1072A0009FED4F7AF0EE487AF4EEC77AF1EE10FADD
:1072B00038EE268AF6D4DFED4B7AB4EEE78AF1EEAB
:1072C00010FA40DDDFED487A37EEC88A68EE087ABA
:1072D0009FED467A9FED466ADFED466AA7EE876A24
:1072E0009FED457AE7EE866A68EE275AA7EEA67A02
:1072F000A5EE878AB4F91E3007EE103AB4F91C30B7
:10730000B8EEC77A06EE903A68EE477AF8EEE66A8B
:10731000E6EE807A26EE888AFDEEE77AA7EE008A0E
:1073200017EE903ABDEEC88AA38318EE103AE383B5
:1073300057E623482C8E38E5214B6A8E5A8450E656
:107340009FED2E8AD6E7DFED2E7AB4EEE78AF1EED6
:1073500010FABBD5DFED217AB6E70FF0D3FA00B211
:1073600036E5002A3FF70EAF3FF463ADA3F57A731D
:107370004FF4FA7207EE90CAC0F5FA7002FB03F3FD
:10738000B3FBF0F3A3F5FA731BB2B8EE676A07EE2E
:10739000903A9FED1C5A9FED1C7ADFED1C5AF8EED7
:1073A000E77AFBEE096A67EE857AE7EEA76A67EE91
:1073B000A57AA6EE867A07E7F33B00209C7B0020A7
:1073C000E8110120FFFFF9C3203E002067666666D2
:1073D00035FA8E3CDB0FC940E4CB1641DB0F49C0C8
:1073E000E4CB16C1DB0FC93FDB0F49409A7C2E3638
:1073F000FAAF4FB93587083CA4AA2ABE00000000A6
:10740000DB0FC9BF0AD7233C00401C450AD7233DE8
:10741000002B3FF7E6AE3FF472ADA0F57A734FF460
:10742000FA72C1F5FA7102FB03F3B3FBF1F3A3F5B2
:10743000FA731BB207EE103A1FED0E5A5FED0D5AAC
:10744000B8EEC77A07EE90CA27EE057ABBEE096A56
:10745000A7EE076AF8EE676A27EE257A5FED167ADF
:10746000DFE6002A3FF704AD3FF4CFAD07EE90CA48
:10747000A3F57A734FF4FA72C0F5FA7002FB03F3C6
:10748000F8EE676AB3FBF0F35FED225A1FED220AB4
:107490001FED226ABBEE097AA3F5FA73FDE400BF83
:1074A0002DE9F04FDFF8289299F9D63F012B97B0DC
:1074B00002DD99F9D93FDBB97B4C23685F073FD5E3
:1074C000DFF810A279480021F7F715FEDAF800304E
:1074D0005E033DD4216821F0004323F07F03002B9D
:1074E00059D101F00403002B70D017B0BDE8F08F24
:1074F00099F9D81F89F8D13F4FF0180E4FF49262D6
:107500004E461EFB012E03F1FF3C002701E0782FC1
:107510000FD006EB0E050FCD06F592640FC495E86B
:107520000300BC4584E8030006F1180607F10107D3
:10753000EDD15D4C0023A9F8D83F23685F07BFD485
:10754000DFF890A10AF032FADAF800305E03C1D514
:1075500057482B21F3F77CFF0028BBD02168554BFF
:107560000B40002BB7D1544A544B127803EB420323
:107570005B78002BAFD011F0040340F06082504ED6
:10758000D6F8C020150440F1628221F0004222F0BA
:107590007F02E2B101E001F00403DFF83C8198F8DA
:1075A00011200A2A6CD0464EB26AD2079BD4002B17
:1075B0009BD141F20242FF230F20A8F8EC2D88F85E
:1075C000EE3D17B0BDE8F04F18F0E4BD3C4E00238F
:1075D0000DF157008DF8573036F02CFF9DF85730DD
:1075E000002B46D1DAF80030DFF8EC8043F40003DA
:1075F000CAF80030236843F00C032360002488F8A5
:10760000644B08F6683308F668521C601C71083336
:107610009A42FAD11AF07CFEB6F9E030294A2A4D96
:1076200082FB0312DB17C3EBA2031BB2A8F8583B83
:10763000A6F8E4300023C6F8E8302B6818034DD4D0
:1076400099F80730D3B1DAF80030D90716D50720FA
:1076500018F0A0FD1D4B1B68C8F8DC3D36F080F922
:10766000D8F8E83DC8F8E00DC8F8E43D17B0BDE82B
:10767000F08FDAF8003043F48043B5E70620E7E7FF
:1076800098F81020632A8ED8104AD8F8040012689F
:10769000A2F51C52103A904285D3064A0A40002AAD
:1076A0003FF421AF7FE700BFA8010120843B002009
:1076B000E48F00208006FF7F147A0020091C060852
:1076C000E811012067666666AC01012014260020DF
:1076D000504D0020B0010120888400209B4B802069
:1076E0001C7040F0A7FE044670B1994F3B68984269
:1076F00000F07281D7F8DC309C4200F06481D7F84A
:10770000B8319C4200F05681924B1B78012B97D1E7
:10771000914C278827B1B4F802B05F45C0F064816E
:107720001A466380237922800BB1002323718020C5
:1077300018F02CF80746002800F06181802118F02D
:1077400087F9FA79854B88F8680D53F8223097F954
:1077500004000093B3F5613F0CBF022300230293A2
:1077600002220023019280211A4618F0CBF97C4BAB
:10777000C8F86C0D5B8807467A4803EB4303A0FB0F
:107780000330400940220121F4F78AFB88F8700D8C
:10779000002F00F03481DAF8003061882F682588E6
:1077A00003F01002704B93F808E0A3688D422CBFE1
:1077B00000210121C3F3800C002A0CBF6046002089
:1077C00009916A49089014BF604600200D7807901F
:1077D0006749684A09781091AEF1010017F4006F0B
:1077E000B0FA80F04FEA501008BF002062490690BE
:1077F00007F0020014681190604AC6F8F8200020D3
:10780000C8F8740DC1E90100C1E90300B8F88A1D88
:10781000A8F8881D14F0080F02F5C67102F546722B
:10782000C6F80021C3F3C00208BF02460592C3F3A5
:10783000C0120E92C3F380120F92C3F340120D9246
:10784000C3F300120C92C3F34002C6F8FC1098F880
:10785000907DC8F88C0D0B9203F0010203F4807345
:107860000493C4F3001304F0200683460A92129393
:1078700004F0040401215FFA8BF21F2A19D8DFE813
:1078800002F011412727272727272727458724216B
:10789000518F8B4D491E35353583106194187F5DAE
:1078A000595535B1D8F88C3D01FA0BF00343C8F8AF
:1078B0008C3D202A00F0A7800BF1010BDBE7002FA5
:1078C000F0D1F6E7002EF7D0ECE7002CF4D0E9E792
:1078D00013920FF041F80BF1FF338342139A4FF0EC
:1078E0000101E6DC049B002BDCD1E2E7139211F0EE
:1078F000FFFA00EBCB00139A30F89C3C0121002BDF
:10790000D0D1D6E7049B002BD6D0CBE7109B002B21
:10791000C8D1D1E7089B002BC4D1CDE7079B002B32
:10792000C0D1C9E7119B002BC6D0BBE70E9B002B33
:10793000B8D1BEE70F9B002BB4D1BAE70D9B002B4B
:10794000B0D1B6E70A9B002BACD1B5E7BC30002024
:10795000282E0020F8460020EC4600209C1D06083A
:10796000C4460020D34D6210243F0020F33B00208A
:107970001E3E0020B4010120FC910020EC120120E9
:107980000C9B002B8ED194E7099B002B94D089E7A8
:10799000059B002B86D18FE7129B002B8CD081E7B3
:1079A000069B002B7FF47EAF86E70B9B002B7FF4BA
:1079B00079AF7EE7204618F0F3F8DC220021384842
:1079C00049F0C9FFA0E6204618F0EAF8DC220021C1
:1079D000344849F0C0FF92E618F0E2F8DC220021BA
:1079E000384649F0B8FF85E659463846F4F71AFAA2
:1079F00097FBF0F29BFBF0F392B29BB291E62A4A1E
:107A0000002313701CE698F8A53D274A003B18BFD9
:107A1000012388F8913D0023C8F8C43DA8F8C83D6B
:107A2000A8F8CA3D88F8D83D02231370D8F8D02DA5
:107A3000D8F85C3BC8F8CC2DC8F8D43D00E621F05E
:107A4000004222F07F02002A3FF44FADA5E5174D1A
:107A500015232A698DF857306B69A86802FB03F378
:107A6000834213D06B68E8680DF15701184449F060
:107A700039FD6B682A69A868216813446A69013274
:107A80006A61B3FBF0F200FB12336B6041F004015A
:107A90004FF40040216017B0BDE8F04F42F0C0BC89
:107AA000E02F0020042F0020F8460020187A002044
:107AB0002DE9F04F964D974FD5F8A8253B78D2F891
:107AC000289089B033B9944B1B685B0672D409B017
:107AD000BDE8F08F914CD4F80C3E04F60460984752
:107AE0000028F0D08E4E737F002B40F09180D6F8A6
:107AF0001E30C4F82A3E0223B6F9220085F8AC35C0
:107B0000B6F91E20B6F92030A4F82E0EB4F9241EC2
:107B1000844EDFF82082DFF820B2891AB4F9262ECD
:107B20000591D21AB4F9283E069205A91B1A94F8B9
:107B3000402E079308461EF039FD05A81EF0E6FC0E
:107B4000DDED057A784B794C93ED076AF8EEE76A3C
:107B5000DDED067AB8EEE77ADDED077AF8EEE77A42
:107B600066EE866A27EE067A67EE867AC7ED026AC7
:107B700087ED037AC7ED047A04F10C0A0BE008F1F3
:107B800004083046D5F878369847A24506F1240611
:107B900004ED010A97D09BF80030B4EC010A012BE8
:107BA000EDD18DED030A46F0AFFC9DED030A48F8D8
:107BB000040BE6E7594C94F8703E002B87D04FEA4F
:107BC000E9752946484644F029F804F6486207EE6C
:107BD000900AD2ED0F6A92ED107AD7ED025A97ED26
:107BE000036AD4F8903ED4F8941EE7EEA56A13EB2E
:107BF000090345EB0105A6EE277AC4F8903EC4F8C8
:107C0000945EC2ED0F6A82ED107A09B0BDE8F08F84
:107C100095F8AC35012B73D1B4F9243E07EE903AB8
:107C2000B4F9263EF8EEE77A05F2AC58CDED057AC8
:107C300007EE903AB4F9283EF8EEE77A05A9CDEDC3
:107C4000067A07EE903AF8EEE77A4046CDED077AED
:107C5000F4F77CF995F8AC35012B09D10023C4F871
:107C60002A3EA4F82E3E0023BB60FB603B612AE75E
:107C7000022B25D0002200230593069307939646F6
:107C80001346114610469446CDE900E2A4F82C0EA6
:107C9000A4F82E1E3084718401200421244AA4F803
:107CA0002ACEA6F81EC0F4F75DFFD5F8A83500204F
:107CB0000021C3E90C01C3E91001C3E90E01D2E7B9
:107CC00098ED065AD8ED0C5A98ED126A8DED055ACA
:107CD000FDEEC56ABDEEE57A16EE903AFDEEC67A87
:107CE0000FFA83FC17EE103A18B217EE903A19B259
:107CF000CDED065A8DED076A634686460A46C3E710
:107D0000B4F92A2EB4F92C3EB4F92E0EFEE600BFCB
:107D1000E8110120C8010120B4010120888400205D
:107D2000C4460020F41701208C920020D0010120CD
:107D300044C406089C7B0020F33B00202DE9F04F53
:107D40008FB01CF0C5FCDFF8F881794BA3EB08027B
:107D5000CDE901234FF00309102200210AA849F0C0
:107D6000FAFD019B0993029B0893724BCDF81C808E
:107D70001A69002ABFBF704A5A6002F188325A60FD
:107D80000124F322DA604FF0000A7E23224604A980
:107D900007A88DF83440CDF830A08DF81030F5F7F5
:107DA00085FC504515DA0023B9F1010900F0B980CE
:107DB000002BD1D098F800307E2B40F0B580F5F73D
:107DC00044FC002800F0B0800FB0BDE8F04F1CF07C
:107DD00099BC224604A95046F5F72CFC574CDFF815
:107DE00064B1ADF812005C453CD30024022205A921
:107DF00007A8ADF81440F5F759FCA042D3DBBDF855
:107E00001200022205A9F5F715FC0222ADF81200B6
:107E10000DF1120107A8F5F749FCA042C3DB0B984E
:107E200088B1079B089A03449342BCD80AABC0F1BF
:107E300004022146184449F08EFD0AA907A8F1F76B
:107E4000A4F9CDE90B400C9B002BACDB9DF8342052
:107E500022B138490A6942F000420A61B3FA83F359
:107E60005B09A1E762888DF819A0C2F30B06B31D68
:107E7000ADF814302388C3F30B011B0B8DF81830B9
:107E80001304ADF8161020D4062205A907A8F5F7AB
:107E90000DFC002887DBBDF81200062205A9F5F7C6
:107EA000C9FB6168ADF81200324607A8F5F7FEFB82
:107EB0000028FFF678AFBDF8120061683246F5F78A
:107EC000B9FBADF8120014348DE700273D460135AB
:107ED000EDB2062205A907A88DF81950F5F7E6FBC3
:107EE0000028FFF660AFBDF81200062205A9F5F7DD
:107EF000A1FB6168ADF812003944324607A803912E
:107F0000F5F7D4FB0028FFF64EAFBDF81200039939
:107F10003246F5F78FFB032DADF812003744D6D16A
:107F2000D1E7002B7FF446AF0520FBF74FF800BFE9
:107F300000800008003C024023016745BC0407089C
:107F400000400008A809070870B50C4E35782D1AB6
:107F500018BF01250328044634BF044600242046E8
:107F6000F5F71CFC064B347003F56A601A2204FB1B
:107F70000200C3F8480B284670BD00BFDD3B00205F
:107F800088840020022810B50C4614D8FFF7DCFFC7
:107F90000948FBF7A1FA094B094819780131FBF7A9
:107FA000F1FA21461020FBF797FB21462020BDE87F
:107FB0001040FBF791BB10BD11BC0608DD3B002053
:107FC00008B5060838B5164C164DAC4215D300203E
:107FD000F5F7E4FB14481CF0B1FB144A136843F4B2
:107FE00080031360124B2F221A70124B1878FFF780
:107FF000ABFFBDE8384027F033BAB4F90230002BAC
:108000004FF00001204607DAF5F7B8FB01212046C2
:10801000F5F7B4FB02212046F5F7B0FB1434D4E7A2
:10802000BC040708A8090708E7B40608643900205B
:10803000643F0020DD3B002010B5064B5C78241A1D
:1080400018BF0124032828BF002058701EF016F81E
:10805000204610BDDD3B0020022810B50C4610D88C
:10806000FFF7EAFF0748FBF737FA074B074859784D
:108070000131FBF787FA21463020BDE81040FBF7BD
:108080002BBB10BDF0B40608DD3B002000B5060890
:108090002DE9F04F0D468DB0B7490446FDF750FC71
:1080A0000646002840F0BE80B4492046FDF748FC53
:1080B0000646002840F0B880B1492046FDF740FC54
:1080C0000646002840F0B2802046AE49FDF738FC55
:1080D0000028064612BF1024264601240DB144F0A4
:1080E0002004A94DA94F95F8009095F80180DFF87C
:1080F00018A35745C0F09C80FFF764FF4846FFF780
:1081000023FF4046FFF798FFA1493046FDF718FCD2
:1081100008B144F0400414F01103009300F0898288
:108120009C48FBF7D9F90020FDF79EFC9A48FBF725
:10813000D3F99A48FBF7B6F904F03003302B02D19B
:108140009748FBF7C9F9974E9748DFF8C092FBF7BD
:10815000C3F99648FBF7C0F9D6ED007A944AF5EEDC
:10816000407AF1EE10FA0CBF012100212046FBF706
:10817000BFF931468F4A904E2046FCF77FF88F4872
:10818000FBF7AAF9B6F902108D4AB1FA81F1490953
:108190002046FBF7ADF931468A4A2046FCF734FF0A
:1081A0008948FBF799F9894A89492046FCF774FE0A
:1081B0008848FBF791F9884A88492046FCF76EFB0E
:1081C0008748FBF789F9874B874A1E68874B1F68EA
:1081D00067EA0603CB464FF0000A01935BF8043BC5
:1081E000002B32D01978D1B1019902934FF00108D8
:1081F00008FA0AF811EA080F14BF012100212046ED
:10820000FBF790F966EA070111EA080F764A029B2C
:1082100014BF012100212046FBF76AF9724A0AF1D6
:10822000010ADBE7012459E7022457E7042455E754
:108230007B88C3F30B021B04D7E9011048BF02EB94
:10824000420249F04FF9143753E79846684A67EA03
:108250000603019359F804BBBBF1000F27D09BF82C
:10826000001009B34FF0010A0AFA08FA17EA0A0FD8
:108270000BD066EA070111EA0A0F5B4614BF012121
:1082800000212046FBF74EF9594A16EA0A0F0BD097
:10829000019B13EA0A0F18BF01215B4608BF0021AA
:1082A0002046FBF725F9524A08F10108D2E7514868
:1082B000DFF85CA1FBF710F94F4AD2F800904F4A63
:1082C00012685E4689EA0208DFF848B16FEA0808DA
:1082D0000127B74018EA070F14BF0121002119EA4E
:1082E000070714BF52465A4630460391019217F0D1
:1082F00079F8019A039902900346204601910136CC
:10830000FBF710F9002F14BF5A465246029B019901
:108310002046FBF7EDF8182EDAD13948DFF8F8A03F
:10832000DFF8F880DFF8F890FBF7D6F8354B9F6858
:108330000026F3B20AEB8302D2F834B1BBF1000F8E
:1083400070D00121994039405B460CD04A4600214B
:108350002046FBF7CDF85B464A4600212046FBF756
:10836000E1F80136E5E7424620460191FBF7C0F807
:1083700001995B464246F1E72AB5060811BC06089A
:10838000F0B4060831B50608DD3B0020BC04070840
:1083900035B5060866BF060842B506085AB5060890
:1083A00066B506084883002057BC0608B6B506081F
:1083B000A1B50608447C002028800020B0B506083E
:1083C000BCB50608687F0020C9B506089C3D0020A2
:1083D00010490020CFB50608187E0020D881002063
:1083E000D8B50608944B0020E0B506086439002093
:1083F000ECB50608B3B9060894490020143F0020E4
:10840000F7B50608144C0020A8090708CC3C06085C
:1084100015B506081FB506081C3C06080CB606086C
:1084200000B606088A48FBF757F801238948DFF8A9
:10843000DCC2DFF8DCE28DF820B08DF810B08DF8EA
:1084400021B08DF811B08DF822B08DF812B08DF8F2
:1084500023B08DF813B01F4613F80C2010F8016BF1
:108460000CA911440DF1300801F8206C13F80E101E
:10847000884408F8106C17B1561A774277410133D7
:10848000052BE9D1744A002608AB394620468DF801
:108490001460FBF747F804AB6F4A39462046FBF7F8
:1084A00027F86E48FBF718F86D4A6E492046FBF72F
:1084B000EDFC6D48FBF710F86C4A6D492046FCF75F
:1084C0009BFA6C48FBF708F86B4A6C492046FCF7AE
:1084D000ABFB6B48FBF700F8644A65492046FCF7A4
:1084E0003FFC6848FAF7F8FF674A68492046FBF7FF
:1084F00015FC6748FAF7F0FF664A67492046FBF724
:10850000D1FD6648FAF7E8FF654A66492046FBF761
:10851000AFFF6548FAF7E0FF644A65492046FCF77B
:1085200043F86448FAF7D8FF634920463EF072FBEF
:108530006248FAF7D1FF4FF0FF331A4660492046F0
:108540003EF0F2FB5F48FAF7C7FF5F4A5F492046FB
:10855000FCF736FF5E48FAF7BFFF5E4A5E492046E9
:10856000FCF7B8FF5D48FAF7B7FF5D4A5D49204662
:10857000FCF7F0FF5C48FAF7AFFF30462146FBF707
:10858000ABF8E0064BD52146304695F800806F7871
:10859000FFF7F8FC21460120FFF7F4FC21460220FA
:1085A000FFF7F0FC21463046FFF756FD214601203B
:1085B000FFF752FD21460220FFF74EFD4046FFF730
:1085C000C3FC3846FFF738FD4848FAF785FF4848AE
:1085D00008F10101FAF7D6FF4648791CFAF7D2FFF5
:1085E000A10703D528782146FFF7CCFC620703D505
:1085F00068782146FFF730FD009B13B13E48FAF73B
:108600006BFF2EB13D48FAF767FF3D48FAF74AFF86
:108610003C4C3D4DAC420ED30DB0BDE8F08F2878F8
:108620002146FFF7AFFC68782146FFF715FD0126CC
:10863000D6E7009ED4E76388C3F30B021B04D4E99A
:10864000010148BF02EB420248F04CFF1434E1E75D
:1086500019B60608804106081DB606081CBD0608A6
:1086600094450020A84C00200DAF0608787E00201D
:10867000E880002029B60608F87E002068810020E6
:1086800024B606082FB6060804420020E849002058
:1086900033B60608C97B0020088400203CB60608D3
:1086A000047D00203883002044B60608187D002091
:1086B0003882002050B606087893002053B606088A
:1086C000B89E00205EB60608B8840020F8A20020FC
:1086D00064B60608B88A0020F8A8002070B606081C
:1086E000188B002058A900202AB506088DB6060868
:1086F000B8B60608B0B60608C3B60608DCB6060863
:10870000F2B60608BC040708A8090708184D00209F
:108710003C3C00200021BBE40121B9E42DE9F74FE6
:108720001BF0D6FFB64CB74B9C42C0F00F81B64C45
:108730002078FFF709FC6078B44CFFF77DFC94F8D3
:10874000603394F86123B2489A4224BF002384F82E
:108750006033F4F7D1FFAF4B1A68AF4B93431FD18F
:1087600000212A20F0F797FE0646C8B100212920F3
:10877000F0F791FE002800F01881056830682B1A88
:108780005D425D4100211220F0F785FE18B10268BC
:1087900033689A4200D01DB14FF48030F4F7ACFF3B
:1087A00000269E4F35464FF0FF0848F2BC3957F877
:1087B00026004308810801F0333103F077330B447E
:1087C000C10801F01131C31A5B1A03EB131310F047
:1087D000010203F00F33B3FBF8F1C1EB012118BF25
:1087E0000135A3EB010318BFEDB2012B08D9022B11
:1087F0000CD112B110EA090F02D141F039F928B1B8
:1088000003360F2ED3D1013D022D03D983480D210C
:1088100041F0E2FF824A138DD18C643B8B42A8BFAA
:108820000B46D38400BF7F4B9A780AB908229A700E
:1088300000200CF08BFB7C4A1368002800F0B78006
:1088400023F080631360794BD3F8486B0EF05AF82D
:10885000774B31781D88DFF8E8E183B22D1A642266
:10886000009305FB01F393FBF2F313FA80F0A4F8F5
:10887000640396F80180C1F16E0301EB8107A2EB5E
:10888000080B9BB24A42C1F1640C7F0092B2019383
:108890005FFA8CFC4FF00A0A4FF47A7916B2002E78
:1088A00040F38880604606FB06F308FB03F310FBE9
:1088B00000F093FBF0F0584406FB00F3009893FBA4
:1088C000FAF33B441BB26B4393FBF9F303442EF8DA
:1088D000023B0A32019B92B29342DFD11DF0E8FBCA
:1088E00030220021534849F036F80CF099F994F8F9
:1088F0009A13514BC820642212FB0101996094F82D
:108900009B1312FB0102DA600022C3E90422C3E9CF
:108910000622C3E9082283F8292083F82A20DA6294
:108920004FF07A7294F89D131A6383F828101DF0A3
:1089300097F81DF0BBF80CF055FD10F0A9F835F0D4
:1089400047FE03B0BDE8F04F1BF0DCBEB4F90230C7
:10895000DFF8F090002BADBF002703274FF0010890
:10896000B846002608EB0601C9B28F4201D2143482
:10897000D9E6324A02F1060ACA453CD21588D5B377
:108980005019484537D2052D35D9B4F800C0B2F892
:1089900002E0CCF30B0CE64505D192F805C00CF0D3
:1089A000030C8C450AD00246E4E70546EAE643F0AC
:1089B000806347E714BF0846012074E7314620462C
:1089C00092F804B0F4F7DAFE2188BBEB113F10D126
:1089D000B4F802C06068CCF30B01AA1F8A42A8BF9A
:1089E0000A461CF4004F18BF01FB0600514648F030
:1089F00079FD0136B6E731462046F4F7BFFEF8E7C9
:108A0000BC040708A8090708DD3B002078A6002061
:108A100020631406643900204000010094450020C2
:108A2000E4450020B4480020A801012088840020EB
:108A3000203E0020E0A90020F8400020014000086E
:108A4000AC1201200080000808B5FFF777F9FFF7A6
:108A500065FEBDE80840012017F0DABB10B50446FA
:108A6000FFF772FA18B1FFF769F9FFF757FE601CBC
:108A7000C0B2BDE8104017F0CBBB38B50C4D044672
:108A80002046FAF745FF38B10A4B0B481978BDE884
:108A900038400131FAF776BD2046F4F78FFD0138F2
:108AA000022804D8C0B2FFF7D9FF2C46E8E738BD4A
:108AB0009AC40608DD3B0020B8B6060810B5044687
:108AC000FFF7BAFA18B1FFF739F9FFF727FE601C74
:108AD000C0B2BDE8104017F09BBB38B50C4D044642
:108AE0002046FAF715FF38B10A4B0B485978BDE814
:108AF00038400131FAF746BD2046F4F75FFD0138F2
:108B0000022804D8C0B2FFF7D9FF2C46E8E738BDE9
:108B10009AC40608DD3B0020B0B60608174B10B516
:108B20001C68620705D5164B1B78022B01D001206B
:108B300010BD230703D5134B1B68D805F7D5A10635
:108B400003D5114B1B7E022BF1D139F0ADFB002870
:108B5000EDD00E4B93F87C26012A01D1A207E7D471
:108B60000B4A10780028E3D00A4A507F0028DFD053
:108B700093F8AC05023818BF012010BDB4010120E4
:108B800004470020B001012038470020E8110120EF
:108B9000C8010120C4460020034B1B685B0700D4BA
:108BA000704709F0BFB800BFA80101202DE9F04FC0
:108BB000DFF894A29FED997ADAF8A8359C6A984B71
:108BC00007EE904AF8EEE77A2DED088B67EE877A8C
:108BD000C3F8444B0AF2DC63C3ED007A914B1B6887
:108BE000ADB0CDE90A01590740F136818E4B0493AF
:108BF0001B68DA0600F18C82DFF85092DFF850B281
:108C0000DFF85082DBF8B033D8ED076AD8ED0F7A81
:108C100098ED117A98ED136A1B19CBF8B033DBF895
:108C2000B43343EBE473CBF8B433DBF8B8331B193C
:108C3000F4EEE67ACBF8B833D8ED107ADBF8BC3333
:108C400043EBE473F1EE10FAF4EEE67AD8ED087A2D
:108C5000C8BFC8ED0F6AF1EE10FAB4EEE77A98EDEE
:108C6000127A48BFC8ED106AF1EE10FAB4EEE77A56
:108C7000C8BFC8ED117AF1EE10FA48BFC8ED127AFC
:108C800067EEA77A98ED097ACBF8BC33E6EEA67AC0
:108C9000664BB4EEC76AE7EE077A1B7898ED146A64
:108CA000F1EE10FAB4EEC76AC8BF88ED137AF1EEA0
:108CB00010FA48BF88ED147AB1EEE77A98ED156A9C
:108CC000B4EEC76AF1EE10FA48BF88ED157A002BB2
:108CD00040F0D380564B1B689F0700F1AD850A9B7F
:108CE000CBF8903A534B0B9A5A600023C8F81C30CB
:108CF000C8F82030C8F824304F4B504C93ED000A90
:108D0000FEF722F8217E002940F037859BF80C3BC6
:108D1000002B40F0EB844A4F9BF8C23B00228BF8BB
:108D20000C2B002B00F09584F9F758FF05460C46F4
:108D300039F018FC284621463EF0F5F92846214630
:108D400039F0C2FAF9F74AFFBB790022022B064636
:108D50008846ABF8102D00F05E8426232E22CDE944
:108D600008320E212A23CDE9063122230A24059355
:108D70000623CDE902344FF0240E2C244FF00C0CC6
:108D8000282220230821042502200190787A022835
:108D900009D1019BABF8103DDDE908E4DDE9062CC3
:108DA000DDE90251059BF8790228387C01BFABF858
:108DB000105D22467346614610B1ABF8101D134694
:108DC000BA7A0498022A08BFABF8103D154B016827
:108DD0001B6821F0800213F00403026000F0C383DB
:108DE0003B78184A03EB830302EBC30311F4C01F63
:108DF000B3F8CA464FF00003BB8040F0C381CB06F6
:108E000041F17E85E50601F13586200702F1938662
:108E100032464346204636F083FAB8E1BD37863500
:108E200088840020A8010120B0010120C801012090
:108E3000B401012008B10020C41801203C3C0020EE
:108E4000504D00201C3C0608E8110120E0220120C2
:108E500078A60020C8180120BB4BDFF81CB3049390
:108E600000220023CBE9EE23DFF810930AF5DC683B
:108E7000B64B1B78002B3FF42DAFB54A0192B54A93
:108E80000992B24AB44EB54B0C930832CDE9023286
:108E900006F5E2730693DFEDB28A9FEDB29A9FED7D
:108EA000B28AB24C06F5F47306F180050D93059372
:108EB0000027039BAE48B3EC010A0393019B1B7888
:108EC0000F2B01BFFDEEC07A029A17EE903A1360A5
:108ED000A84BF9B21B689847019B1B780F2B02BF68
:108EE000FDEEC07A029A17EE903A304608BFD36082
:108EF00059F8D03C98479AF8B437002B40F0E280FC
:108F000005F16C03099A127F002A42D1039A02EDFF
:108F1000010A029A043202921D46069A059B013705
:108F20000C320433032F04F5117406F12406069263
:108F30000593BED19AF8B437002B3FF4CBAE9BF823
:108F40008C3A00228AF8182F9BB99AF82C290D9E8A
:108F5000501C00F03F008AF82C0906EB82003568AF
:108F6000056106EB82007468B168C0F81041C0F872
:108F70001012013303F001038BF88C3A9AF8303C5D
:108F8000032B03F23080DFE813F07B142E15630E01
:108F90000714A28C07EBC70007EB001010440BEB83
:108FA000800181EDFA0AD4ED8D7AD4ED8E6A94EDCC
:108FB0008C7A70EE677A4A3067EEA77A0BEB800006
:108FC000C0EDF17AB4F84012013292B29142A2841B
:108FD0004FEAC7003CBF0022A2841146C21907EB2A
:108FE00002120A440BEB820191EDFA6A30EE077A25
:108FF0004A3237EE467A0BEB820284ED8C7A92EDA0
:10900000F16A019A77EEA67AD4ED8F6A127877EE3C
:10901000C67A27EE267AC4ED8E7A84ED8D7A27EE15
:10902000A67AB5EEC07AF1EE10FAA8BFF1EEC77AD3
:1090300084ED087AACBF27EE887AB0EE497A152A1B
:1090400084ED017A76D0D4ED046AD4ED057A76EE1B
:10905000A66A76EEE75A77EEE67AF5EE405AF1EE3A
:1090600010FA14BFD4ED074A94ED065AC4ED055A20
:109070001EBF84EEA56AB7EE005A35EE465AD4ED0F
:10908000004A94ED026A18BFB0EEC55AA4EE856A94
:1090900018BF84ED065A36EE077A77EE807A86EEB0
:1090A000075AF7EE006AE5EE275A76EEC57AB0EE7B
:1090B000650A67EE867A84ED035AC4ED045AC4ED5E
:1090C000027A23E7059B83ED000A019B1B78122B94
:1090D00001BFFDEEC07A029A17EE903A1360069A2D
:1090E00005F16C0352F8041B089328460792884741
:1090F000089B079A2435AB42F4D1019A1278122AC0
:1091000001BFFDEEC07A029917EE902ACA60F9E617
:109110000E200BF033FCDFF86490002801F09384FC
:1091200099F87436032B3FF669ADDFF84CB0DFF8E1
:1091300050809DE6D4ED037A029A67EEA87AFDEEA0
:10914000E77AC2ED007A7EE7B0010120C801012074
:10915000F33B0020C4460020201901209C7B002006
:1091600000007A44000000001F852B3F38AA002031
:10917000A4020120DC01012078A60020E0220120C9
:10918000C818012032464346204639F0CFFABE4D7A
:109190003B790BB10023BB707B790BB10023FB70D3
:1091A000FB7A2BB1BBF8103D43F04003ABF8103D08
:1091B0003B7B2BB1BBF8103D43F08003ABF8103D77
:1091C0007B7B2BB1BBF8103D43F48073ABF8103DB3
:1091D00097EDFF0A45F098F9AC4BCBF8380D93EDBD
:1091E000000A45F091F995ED000ACBF83C0D45F0E9
:1091F0008BF9049BCBF8400D1A68D40640F1BA8174
:10920000DBF8442DDBF8483D134300F00381F9F708
:10921000E5FCDBF8503D0390C31A022008EE903ABB
:109220000591F5F722FC9A4D9A4C05FB00F09A4DFA
:10923000A5FB0035B4F90630401B05EB500503EBE8
:109240008303ED0A03EB830305EB850200209D00F9
:10925000C5EB4205B4F9043095FBF3F5F5F705FCD1
:1092600021888E4CA1FB0031D81841EB0102C018B7
:1092700041EB0202D20042EA5072C000C01841EB3A
:1092800002014B01420143EAD063801841EB030124
:109290008900834A41EA90710023800042F054FD26
:1092A0002DB286B205FB06F384FB03247D4ADBF86E
:1092B000441DDB17C3EB641302935468DBF8503D85
:1092C00006932343A5EB010540F0758792ED027AE2
:1092D000DFED757ABBF85C2DDFED745A019125EA5C
:1092E000E573B8EEE88A724D28EE278AD5ED017A4B
:1092F00095ED000A85ED028A78EE277A02FB03F3EA
:1093000088EE276A07EE903AF8EEE77AF0EE406AC8
:10931000D7EEA56A36EE877AA6EE070A85ED000A33
:1093200045F0F2F89BF8743D01998046002B40F01F
:109330002087BAF922000190002900F00E811FFA5F
:1093400088F8A0EB0808B8F57A7F019AB8BF4FF407
:109350007A78904580F20181002B01F052830FFA58
:1093600088F30193029BDBF8485D581B069B23435F
:1093700040F0D4864F4B93ED007A4F4CBBF85C3DE8
:10938000D4ED017A94ED000ADFED4C5A84ED028AA7
:1093900078EE277A20EAE07088EE276A03FB00F077
:1093A000B0FBF6F007EE900AF8EEE77AF0EE406ACE
:1093B000D7EEA56A36EE877AA6EE070A84ED000A94
:1093C00045F0A2F89BF8A08D0646B8F1000F40F0DA
:1093D0008886BAF922000246002D00F0B880B6B2A5
:1093E000861BB6F57A7FB8BF4FF47A76964280F244
:1093F000AE80B8F1000F01F0158332B2294B059908
:109400005960019B9342A8BF1346AAF82230039BE0
:10941000CBF8503D19F8244C002C78D059ED067A41
:1094200019ED077A59ED046A254B67EEA77AB0EE7D
:10943000006AE7EE077AB7EE007AA7EEC67AD3EDB8
:10944000008AF4EEC76AF1EE10FA00F3FB86049B83
:109450001B680393DA0601F1B9853B78194A03EBDF
:10946000830302EBC303B3F8CA361B0641F1EB8654
:109470007B7B002B41F0AA85BAF92030DAF8C08056
:109480000593022300F0E7BE545100205051002004
:1094900010090500243F0020010110001F85EB5139
:1094A000187C3E00C8B30020BD3786356F12833A62
:1094B000DCB3002004B4002008B40020CDCCCC3DA7
:1094C000C41801201C3C060807EE903AC84ABAF9B5
:1094D000DC3082FB0312DB17C3EBA2031BB207EEE7
:1094E000103AB8EEC77AF8EEE77AB0EEC77AB4EE83
:1094F000E77AF1EE10FA02F3DF82002389F82935CA
:10950000B0EE680AD9F868362046022198470DF077
:10951000EBFDB84B1B78002B40F0D385B64B1B7886
:10952000002B40F0AD85B54B1B78002B40F0A48597
:10953000049B1A68910200F15B859BF8D03D002BDB
:1095400000F028852DB0BDEC088BBDE8F08F00231E
:10955000236000238BF8A03D50E700232B600023FD
:109560008BF8743DFEE6D406A7F8113087F8EC3F7F
:109570003FF546AE3B78A24A03EB830302EBC303FD
:10958000B3F8CA36D80541F12D86F7EE008A0DF002
:10959000B9F907EE900ABAF92240B8EEE78A0DF061
:1095A000B1F9241A07EE904AF8EEE76A59ED067A07
:1095B00019ED077A9FED936A67EEA77AE7EE077ACF
:1095C000F4EEC67AF1EE10FA02F39D82B7EE007A5D
:1095D000F0EE005AB0EE476AA7EEE56AC7EE067AEB
:1095E00077EEC77AB7EE007AA8EEA77AF0EE487A5F
:1095F000E6EE877AFDEEE77A17EE904A0DF082F9F3
:10960000814B84421B8803DBA342A8BF2346184634
:10961000AAF82200F4E501232F25ABF8103D2723FB
:10962000CDE908354FF00F0C2B23CDE9063C232361
:109630000B2205930723CDE902322D244FF0250E8E
:109640004FF00D0C29222123092105250320FFF7C6
:109650009CBB6E4B9FED6E7AD3ED0F7A6D4B6E4CCB
:109660005A7F77EE877A002300200021C4E9280181
:10967000C4E90201C4E90C01C4E91401C4ED467A4D
:10968000C4ED477AC4F82831C4F82C31C4F830311D
:10969000C4F83431C4F8C430002A41F0A5819FEDEC
:1096A0005F8A5F4884ED2D8AB7EE000AF0EE480A23
:1096B00084ED408A84ED438A84ED2E8A84ED418ACC
:1096C00084ED448A84ED2F8A84ED428A84ED458AB4
:1096D000F1F70CFF5348F0EE480AB7EE000AF1F735
:1096E00005FF01238BF8C23BFFF71EBB34F042F8A5
:1096F0004D4B4E4C1A682368DBF8B41BCBF8B43BD7
:10970000500701F15B814A4F34F088FE20B19BF88D
:10971000B83B002B02F02F80BB7B1620002B41F0C2
:10972000EF850BF02BF9B87335F05CF932F0E8FDFA
:1097300034F03CFC3B78324A03EB830302EBC30377
:1097400041F6B800D3F8CC5620EA050040F05AFEA6
:10975000284640F065FE2E200BF010F920B1DAF813
:10976000C030190542F10F80FB7C002B41F09D8633
:109770007B78ABF8C03BFFF7CFBA9BF80C3B002BD4
:1097800001F0FC809BF80D3B2A4E002B01F09C85DC
:1097900007EE901A96ED007AF8EEE77AF4EE477A43
:1097A000F1EE10FA41F0908506F19407BAF91C30F9
:1097B00007EE903ABAF91E30F8EEE77AC7ED007A74
:1097C00007EE903ABAF92030F8EEE77AC7ED017A61
:1097D00007EE903ABAF92230F8EEE77AC7ED027A4E
:1097E00007EE903AF8EEE77AC7ED037A01F0CBB8CE
:1097F000676666661E3E00201D3E0020B3480020BE
:109800001C3C0608CCCC4C3E203E00207040002082
:109810006F12833AC446002040B2002000000000CE
:1098200078B2002098B20020A80101201426002060
:10983000504D002088B10020DAF8E836E348984718
:109840000446002800F03383E14B1B780D2B01F018
:109850000181BAF9EE3649F8C83CBAF9F03649F850
:10986000C43CBAF9F23649F8C03C049B1B689D051C
:1098700000F1E6819AF87C36012B40F0E1813DF061
:109880009BF8051EC0F2DC810BEB050393F8983AB8
:10989000002B02F0D1829BF8983A002B00F0D08187
:1098A0009BF8993A002B00F0CB819BF89A3A002B59
:1098B00000F0C6819BF89B3A002B00F0C1819BF819
:1098C0009C3A002B00F0BC819BF89D3A002B00F0E5
:1098D000B781C04E00231C931D931E931F931893B2
